:100000000C94D2030C94EF030C94EF030C94EF03C5
:100010000C94EF030C94EF030C94EF030C94EF0398
:100020000C94EF030C94384B0C94EF030C94EF03F7
:100030000C94EF030C94EF030C94EF030C94EF0378
:100040000C94EF030C94EF030C94EF030C94EF0368
:100050000C94EF030C94545A0C94EF030C94EF039C
:100060000C94EF030C94EF030C94EF030C94EF0348
:100070000C94EF030C94EF030C94EF030C94EF0338
:100080000C94EF030C94EF030C94EF030C94EF0328
:100090000C94EF03BD4C084DCC4DF24D6A4E8F4E83
:1000A000BA4EBE4EDA4EDD57DD57DD57DD57DD5710
:1000B000DD57DD57DD57DD57DD57DD57DD57DD57A0
:1000C000DD57DD57DD57DD57DD57DD57DD57DD5790
:1000D000DD57A84FF64E124FC74FD84F4D51A6517E
:1000E0004A528C52C8523B53DD57DD57DD57DD571E
:1000F000DD57DD57DD57DD57DD57DD57DD57DD5760
:10010000DD57DD57DD57DD57DD57DD57DD57DD574F
:10011000DD5708504D50A953C253F2530954DD57CF
:10012000DD57DD57DD57DD57DD57DD57DD57DD572F
:10013000DD577D50D55016549654155557551E57BA
:100140002D57CE55E2553C574E576257DD577357E2
:10015000BA50E2500A51A757C2579855B355F655B1
:100160002A564D56AD56C856F356CE03C103B303B7
:10017000A30390037A036103470329030803E602FC
:10018000C2029E0276024F02280203026C01B801ED
:1001900096017501560139011F010601EF00DA00D1
:1001A000B5008200A5009600000043414E203100BA
:1001B00000000000000000000043414E203200001B
:1001C000000000000000000043414E20330000000A
:1001D0000000000000000043414E203400000000F9
:1001E00000000000000043414E20350000000000E8
:1001F000000000000043414E2036000000000000D7
:100200000000000043414E203700000000000000C5
:1002100000000043414E20380000000000000000B4
:10022000000043414E2039000000000000000000A3
:100230000043414E2031300000000000000000006B
:1002400043414E2031310000000000000000004317
:10025000414E203132000000000000000000434108
:100260004E20313300000000000000000043414EEA
:1002700020313400000000000000000043414E2007
:10028000313500000000000000000043414E2031E5
:100290003600000000000000000043414E203137CE
:1002A00000000000000000000043414E20313800F3
:1002B000000000000000000043414E2031390000E2
:1002C0000000000000000043414E203230000000DA
:1002D00000000000000043414E20323100000000C9
:1002E000000000000043414E2032320000000000B8
:1002F0000000000043414E203233000000000000A7
:1003000000000043414E2032340000000000000095
:10031000000043414E203235000000000000000084
:100320000043414E20323600000000000000000073
:1003300043414E203237000000000000000000431F
:10034000414E203238000000000000000000434110
:100350004E20323900000000000000000043414EF2
:1003600020333000000000000000000043414E2018
:10037000333100000000000000000043414E2033F4
:1003800032000000000000000000466C617368202D
:10039000310000000000000000466C6173682032EC
:1003A0000000000000000000466C6173682033000C
:1003B00000000000000000466C61736820340000FB
:1003C000000000000000466C6173682035000000EA
:1003D00000000000005357495443482031000000FA
:1003E00000000000535749544348203200000000E9
:1003F00000000053574954434820330000000000D8
:1004000000005357495443482034000000000000C6
:1004100000535749544348203500000000000000B5
:100420005357495443482036000000000000005351
:10043000574954434820370000000000000053573C
:100440004954434820380000000000000053574939
:10045000544348203900000000000000535749541D
:1004600043482031300000000000005357495443F6
:10047000482031310000000000004348414E4E4505
:100480004C20310000000000004348414E4E454CD6
:1004900020320000000000004348414E4E454C20F1
:1004A000330000000000004348414E4E454C2034CC
:1004B0000000000000004348414E4E454C203500EE
:1004C00000000000004348414E4E454C20360000DD
:1004D000000000004348414E4E454C2037000000CC
:1004E0000000004348414E4E454C203800000000BB
:1004F00000004348414E4E454C20390000000000AA
:10050000004348414E4E454C203130000000000071
:100510004348414E4E454C2031310000000000431D
:1005200048414E4E454C2031320000000000434807
:10053000414E4E454C2031330000000000434841FD
:100540004E4E454C20313400000000004348414EDF
:100550004E454C20313500000000004348414E4ECE
:10056000454C20313600000000004348414E4E45C6
:100570004C20313700000000004348414E4E454CAE
:1005800020313800000000004348414E4E454C20C9
:10059000313900000000004348414E4E454C2032A6
:1005A0003000000000004348414E4E454C2032319F
:1005B00000000000004348414E4E454C20323200BE
:1005C000000000004348414E4E454C2032330000AD
:1005D0000000004348414E4E454C2032340000009C
:1005E00000004348414E4E454C203235000000008B
:1005F000004348414E4E454C20323600000000007A
:100600004348414E4E454C20323700000000004325
:1006100048414E4E454C203238000000000043480F
:10062000414E4E454C203239000000000043484105
:100630004E4E454C20333000000000004348414EF0
:100640004E454C20333100000000004348414E4EDF
:10065000454C20333200000000004348414E4E45D7
:100660004C20333300000000004348414E4E454CBF
:1006700020333400000000005649525455414C20AC
:10068000310000000000005649525455414C2032C0
:100690000000000000005649525455414C203300E0
:1006A00000000000005649525455414C20340000CF
:1006B000000000005649525455414C2035000000BE
:1006C0000000005649525455414C203600000000AD
:1006D00000005649525455414C203700000000009C
:1006E000005649525455414C20380000000000008B
:1006F0005649525455414C20390000000000005624
:1007000049525455414C20313000000000005649F8
:10071000525455414C2031310000000000564952DE
:100720005455414C203132000000000056495254CB
:1007300055414C20313300000000005649525455B9
:10074000414C2031340000000000564952545541BC
:100750004C20313500000000005649525455414CA0
:1007600020313600000000005649525455414C20BB
:10077000313700000000005649525455414C203199
:100780003800000000005649525455414C20313980
:1007900000000000005649525455414C20323000B0
:1007A0000000000011241FBECFEFD0E1DEBFCDBF9F
:1007B00011E0A0E0B1E0EEE2FDED00E00BBF02C011
:1007C00007900D92A43BB107D9F71FE0A4EBB1E06D
:1007D00001C01D92A931B107E1F70C94D23C0C94F1
:1007E0000000282F277099279695879596958795CD
:1007F0009695879533272330310529F1243031052B
:100800004CF421303105B9F022303105C4F4232BEA
:1008100071F02CC025303105F1F025303105BCF0E8
:1008200026303105E1F027303105E9F01FC0A098EE
:10083000A198A2981BC0A09AA198A29817C0A098AE
:10084000A19AA29813C0A09AA19AA2980FC0A098AA
:10085000A198A29A0BC0A09AA198A29A07C0A098AA
:10086000A19AA29A03C0A09AA19AA29A80628093A8
:100870007C0020E02F5F2A3FE8F380917A008061BE
:1008800080937A0080917A00806480937A008091CE
:100890007A0086FDFCCF209178008091790099271D
:1008A000880F991F880F991F2295269526952370EA
:1008B000820F911D0895282F277099279695879567
:1008C000969587959695879533272330310529F19D
:1008D000243031054CF421303105B9F02230310596
:1008E000C4F4232B71F02CC025303105F1F02530F4
:1008F0003105BCF026303105E1F027303105E9F053
:100900001FC0A098A198A2981BC0A09AA198A298D5
:1009100017C0A098A19AA29813C0A09AA19AA298D1
:100920000FC0A098A198A29A0BC0A09AA198A29AD1
:1009300007C0A098A19AA29A03C0A09AA19AA29ACD
:10094000806280937C0080917A00806480937A003A
:1009500080917A0086FDFCCF80917A00806180933F
:100960007A00809179009927089540E050E0FC01D9
:100970000296259134916217730760F44B5F5F4FC5
:10098000FC010296259134916217730718F44639D9
:100990005105A4F3CA010895FC0180910001813042
:1009A000B1F410920001F093BD01E093BC01F0930B
:1009B000BB01E093BA01F093B901E093B801F09361
:1009C000B701E093B601F093B501E093B4016091F3
:1009D000BA017091BB017093BD016093BC0140915D
:1009E000B8015091B9015093BB014093BA012091D5
:1009F000B6013091B7013093B9012093B8018091CD
:100A0000B4019091B5019093B7018093B601F09332
:100A1000B501E093B401E80FF91FE20FF31FE40FF3
:100A2000F51FCF01860F971F65E070E00E94DE6D15
:100A3000CB01089580E10E94F1030E94CC04BC0127
:100A40008AE691E00E94B5049927089583E10E9407
:100A50005B049091B30D989F90011124232F3327AD
:100A60002F3F310519F010F04FEF01C0422F809158
:100A7000BE01882339F44093C0014093BF014093E5
:100A8000BE0118C08091C001280F311D9091BF0197
:100A9000290F311D8091BE01280F311D9093C00197
:100AA0008093BF014093BE01C901969587959695A5
:100AB0008795482F842F9927089580E280937C00A2
:100AC00087E880937A00989A999A9A9AA098A19820
:100AD000A298089590E0892F8295807F8093ED0001
:100AE0001092EE001092EF001092F0001092F100C0
:100AF0001092F2001092F3001092F4001092F500A0
:100B00001092F6001092F70080E01092FA008F5FCA
:100B10008830D8F39F5F9F30F0F208953091ED0058
:100B200090E020EC892F8295807F8093ED0080916A
:100B3000EF00822329F43093ED00892F992708953F
:100B40009F5F9F3078F33093ED008FEF90E0089532
:100B50008091EE0086FF03C080E090E008958091D0
:100B6000EE0085FF03C081E090E008958091EF00E2
:100B7000807C19F48FEF90E0089582E090E0089572
:100B8000BC0140E08091EF0099278F709070892B15
:100B900089F0FB01E40FF11D8091FA0080834F5F23
:100BA000242F33278091EF0099278F70907028179A
:100BB00039077CF3089589EB9CE00E94143A60E6C3
:100BC0007DE080E00E94513A67E17DE081E00E9493
:100BD000513A61ED7CE082E00E94513A81E08093DD
:100BE000C2018091B90C813061F48091BA0C90916E
:100BF000BB0C6AE070E00E94DE6D7093B70C6093EE
:100C0000B60C8091610D813061F48091620D9091FC
:100C1000630D6AE070E00E94DE6D7093B20C609329
:100C2000B10C8091180D813061F48091190D909173
:100C30001A0D6AE070E00E94DE6D7093B50C60934F
:100C4000B40C8091D20C813061F48091D30C9091DE
:100C5000D40C6AE070E00E94DE6D70935F0D6093CB
:100C60005E0D0895CF93DF93CDB7DEB7CE55D0405C
:100C70000FB6F894DEBF0FBECDBF19828CE0888F0F
:100C800084E690E09B838A831D821C821E821F82E1
:100C9000188619861A861B8689819E01245F3F4F1C
:100CA000F901E80FF11D10828F5F8C30C8F3CE017F
:100CB00001960E94043AA895198E1A8E84E690E057
:100CC0009C8F8B8F1E8E1D8E898D9E012F5F3F4FB7
:100CD000F901E80FF11D168E8F5F8034C8F3CE0145
:100CE00049960E94243AA89581E0898F1A8E84E65D
:100CF00090E09C8F8B8F1E8E1D8E8A8D9E012F5FA4
:100D00003F4FF901E80FF11D168E8F5F8034C8F355
:100D1000CE0149960E94243AA89582E0898F1A8EC6
:100D200084E690E09C8F8B8F1E8E1D8E8A8D9E0197
:100D30002F5F3F4FF901E80FF11D168E8F5F803452
:100D4000C8F3CE0149960E94243AA895C25ADF4FB3
:100D50000FB6F894DEBF0FBECDBFDF91CF910895DF
:100D600099278832910509F440C08932910594F49D
:100D70008532910559F18632910534F4833291051B
:100D8000D9F08497F1F04FC08632910521F1879711
:100D900039F149C08B329105B9F18C32910534F4A7
:100DA0008932910539F18A9751F13DC08C32910514
:100DB00081F18D9799F137C080EC0E94024A992702
:100DC000089581EC0E94024A9927089582EC0E94BE
:100DD000024A9927089581ED0E94024A99270895B1
:100DE00084EC0E94024A9927089585EC0E94024AE9
:100DF0009927089586EC0E94024A9927089587EC66
:100E00000E94024A9927089583EC0E94024A99277A
:100E1000089582ED0E94024A9927089583ED0E9469
:100E2000024A9927089580E090E00895DF92EF92BA
:100E3000FF920F931F93CF93DF93CDB7DEB76597E4
:100E40000FB6F894DEBF0FBECDBF8091B20D8823E0
:100E5000C4F480915D0D833620F48F5F80935D0D27
:100E600010C010925D0D19821A821B821C8282E0D2
:100E70008D8381E08E838AE08F83CE0101960E946C
:100E800085478091B00D9091B10D01978F5F97408C
:100E900008F0A0C49091AF0D992309F49BC48091F0
:100EA000B30C8F5F8093B30C891708F493C410922E
:100EB000B30C88E08D8300E0CE010696FC01E00FC4
:100EC000F11D10820F5F0830C8F38091B80C99278C
:100ED0008630910509F4B3C287309105BCF48330A4
:100EE000910509F4E8C18430910544F481309105FD
:100EF00009F46FC1029709F4A5C122C0843091059D
:100F000009F434C2059709F465C21AC08930910505
:100F100009F44DC38A30910544F48730910509F4F2
:100F2000C3C2089709F413C30BC08B30910509F4B1
:100F3000B4C38B3091050CF487C30C9709F41FC41C
:100F40008091B00D9091B10DAA27BB2789839A8318
:100F5000AB83BC8301E00093B80C10E080EC0E94EE
:100F6000024A8111102F81EC0E94024A8111126005
:100F700082EC0E94024A8111146081ED0E94024AB3
:100F80008111186084EC0E94024A8111106185EC85
:100F90000E94024A8111106286EC0E94024A81116D
:100FA000106487EC0E94024A811110681E8310E0D1
:100FB00083EC0E94024A811111E082ED0E94024AF4
:100FC0008111126083ED0E94024A811114601F8317
:100FD00010E081E00E94A95D811111E082E00E9491
:100FE000A95D8111126083E00E94A95D81111460E6
:100FF00084E00E94A95D8111186085E00E94A95DCE
:101000008111106186E00E94A95D8111106287E064
:101010000E94A95D8111106488E00E94A95D811180
:101020001068188710E089E00E94A95D811111E025
:101030008AE00E94A95D811112608BE00E94A95D87
:10104000811114608CE00E94A95D811118608DE00F
:101050000E94A95D811110618EE00E94A95D81113D
:1010600010628FE00E94A95D8111106480E10E94EE
:10107000A95D81111068198710E081E00E94381382
:10108000811111E082E00E9438138111126083E027
:101090000E9438138111146084E00E94381381117A
:1010A000186085E00E9438138111106186E00E946B
:1010B00038138111106287E00E9438138111106487
:1010C00088E00E943813811110681A8710E089E0C7
:1010D0000E943813811111E08AE00E9438138111B7
:1010E00012608BE00E943813811114608CE00E9422
:1010F0003813811118608DE00E943813811110613E
:101100008EE00E943813811110628FE00E94381324
:101110008111106480E10E943813811110681B87CF
:1011200010E081E10E943813811111E082E10E94F8
:1011300038138111126083E10E9438138111146009
:1011400084E10E9438138111186085E10E943813F0
:101150008111106186E10E9438138111106287E1CC
:101160000E9438138111106488E10E9438138111A4
:1011700010681C8710E089E10E943813811111E08A
:101180008AE10E943813811112608BE10E943813AA
:10119000811114608CE10E943813811118608DE177
:1011A0000E943813811110618EE10E943813811161
:1011B00010628FE10E9438138111106480E20E9456
:1011C0003813811110681D87CE0101960E94854752
:1011D00001C38091B00D9091B10D0196AA27BB2754
:1011E00089839A83AB83BC8382E08093B80C00E050
:1011F000802F8F5F0E944732DC01FC01878580FFD2
:1012000002C014E613C0FD01878583FF02C015E606
:101210000DC0FD01878586FF02C016E607C0FD01EF
:101220008181807F11F011E001C010E0FE01E00F2C
:10123000F11D16830F5F0830D8F2CE0101960E948F
:101240008547C8C28091B00D9091B10D0296AA2732
:10125000BB2789839A83AB83BC8383E08093B80CDC
:1012600000E0802F875F0E944732DC01FC01878508
:1012700080FF02C014E613C0FD01878583FF02C012
:1012800015E60DC0FD01878586FF02C016E607C082
:10129000FD018181807F11F011E001C010E0FE01AD
:1012A000E00FF11D16830F5F0830D8F2CE010196D2
:1012B0000E9485478FC28091B00D9091B10D039629
:1012C000AA27BB2789839A83AB83BC8384E080935E
:1012D000B80C00E0802F8F5E0E944732DC01FC01D9
:1012E000878580FF02C014E613C0FD01878583FF58
:1012F00002C015E60DC0FD01878586FF02C016E617
:1013000007C0FD018181807F11F011E001C010E074
:10131000FE01E00FF11D16830F5F0230D8F2083096
:1013200000F50F2EF6E0EF2EFF24F02DEC0EFD1E43
:10133000802F8F5E0E944732DC01FC01878580FF91
:1013400002C014E607C0FD018181807F11F011E029
:1013500001C010E0F701E00FF11D10830F5F0830AE
:1013600038F3CE0101960E94854734C28091B00DBA
:101370009091B10D0496AA27BB2789839A83AB83EA
:10138000BC8385E08093B80C00E00F2EF6E0EF2ED2
:10139000FF24F02DEC0EFD1E802F875E0E94473249
:1013A000DC01FC01878580FF02C014E607C0FD0157
:1013B0008181807F11F011E001C010E0F701E00FA2
:1013C000F11D10830F5F083038F3CE0101960E94A3
:1013D000854700C28091B00D9091B10D0596AA2766
:1013E000BB2789839A83AB83BC8386E08093B80C48
:1013F00000E00F2EF6E0EF2EFF24F02DEC0EFD1E88
:10140000802F8F5F0E944732FC018181807F59F0DD
:101410009701200F311D80899189019696958795B6
:10142000F901808304C0F701E00FF11D10820F5F06
:10143000083030F3CE0101960E948547CBC18091E0
:10144000B00D9091B10D0696AA27BB2789839A8388
:10145000AB83BC8387E08093B80C00E00F2EF6E0EE
:10146000EF2EFF24F02DEC0EFD1E802F875F0E94D3
:101470004732FC018181807F59F09701200F311D97
:1014800080899189019696958795F901808304C09A
:10149000F701E00FF11D10820F5F083030F3CE012D
:1014A00001960E94854796C18091B00D9091B10D33
:1014B0000796AA27BB2789839A83AB83BC8388E0DE
:1014C0008093B80C00E00F2EF6E0EF2EFF24F02DF5
:1014D000EC0EFD1E802F8F5E0E944732FC01818141
:1014E000807F59F09701200F311D808991890196E5
:1014F00096958795F901808304C0F701E00FF11DEF
:1015000010820F5F023030F30830E0F40F2EF6E067
:10151000EF2EFF24F02DEC0EFD1E1FE0802F8F5EBE
:101520000E944732FC018181807F29F0F701E00FA2
:10153000F11D108304C0F701E00FF11D10820F5F51
:10154000083060F3CE0101960E94854743C1809127
:10155000B00D9091B10D0896AA27BB2789839A8375
:10156000AB83BC8389E08093B80C00E00F2EF6E0DB
:10157000EF2EFF24F02DEC0EFD1E1FE0802F875E66
:101580000E944732FC018181807F29F0F701E00F42
:10159000F11D108304C0F701E00FF11D10820F5FF1
:1015A000083060F3CE0101960E94854713C18091F7
:1015B000B00D9091B10D0996AA27BB2789839A8314
:1015C000AB83BC838AE08093B80CCE010E960E9458
:1015D0002D328889282F3327C901880F991F880F3A
:1015E000991F880F991F820F931F280F391F832F70
:1015F00099278E832F838989282F33278091B50DD2
:1016000088235CF488EC90E0289FA001299F500D6E
:10161000389F500D11249A010AC084E690E0289F5B
:10162000F001299FF00D389FF00D11249F01832FA9
:101630009927888729871A861B861C861D86CE01D6
:1016400001960E948547C6C08091B00D9091B10D62
:101650000A96AA27BB2789839A83AB83BC838BE036
:101660008093B80CCE010E960E942D321E821F82EE
:10167000188619868E859F859C012F5F3F4F369572
:101680002795832F99278A872B8781E08C871D8652
:10169000CE0101960E9485479DC08091B00D90912A
:1016A000B10D0B96AA27BB2789839A83AB83BC8392
:1016B0008091C101882331F081508093C101109243
:1016C000B80C06C089E08093C1018CE08093B80C0F
:1016D00010E081E10E94A95D811111E082E10E9488
:1016E000A95D8111126083E10E94A95D81111460DE
:1016F00084E10E94A95D811118601E8381E20E942D
:101700004732DC01FC01878580FF02C014E60DC072
:10171000FD01878583FF02C015E607C0FD018181B9
:10172000803F11F411E001C010E01F83113019F463
:101730008FE0898701C0198682E20E944732DC016E
:10174000FC01878580FF02C014E60DC0FD0187857E
:1017500083FF02C015E607C0FD018181803F11F4BF
:1017600011E001C010E01887113019F48FE08A876A
:1017700001C01A86CE0101960E9485472BC0809138
:10178000B00D9091B10D0C96AA27BB2789839A833F
:10179000AB83BC831092B80C809180018E838091C2
:1017A00081018F83FE013896A6E0B0E082E090E0F0
:1017B00021E08030920719F40E94816E03C0182E38
:1017C0000E94816E1A861B861C861D86CE0101969C
:1017D0000E9485478091B60C9091B70C009709F450
:1017E00072C001979093B70C8093B60C892B09F0C7
:1017F0006AC08091BA0C9091BB0C6AE070E00E94C4
:10180000DE6D7093B70C6093B60C8091BC0C909118
:10181000BD0CAA27BB2789839A83AB83BC8388E04E
:101820008D838091C2018E838091BE0C0E94DB3239
:101830000196969587958F838091BF0C0E94DB322D
:1018400001969695879588878091C00C0E94DB321F
:1018500001969695879589878091C10C0E94DB320D
:101860000196969587958A878091C20C0E94DB32FB
:101870000196969587958B878091C30C0E94DB32E9
:101880000196969587958C872091C20189EB9CE003
:10189000FC01E20FF11D82850E94DB3201969695D4
:1018A00087958D878091C201982F9F5F9093C20189
:1018B0008091D00C891718F481E08093C201CE0189
:1018C00001960E9485472091640D3091650D8091AD
:1018D0001B0D90911C0D2817390719F4DD24D394A2
:1018E00001C0DD248091B10C9091B20C009709F4F5
:1018F00004C201979093B20C8093B10C892B09F02C
:10190000FCC1CE010E960E942D328091620D909105
:10191000630D6AE070E00E94DE6D7093B20C60931C
:10192000B10C8091640D9091650DAA27BB27898326
:101930009A83AB83BC8388E08D83EE240F2EF0E87E
:10194000FF2EF02D0E2D802F9927FC01E05AF24F2B
:101950001681133238F4812F0E94E731882379F001
:10196000EF280DC01E3238F4812F0E94B006882364
:1019700031F0EF2804C01E3211F4A499EF28F69438
:101980000F5F083000F3DD2029F10F2EF0E8FF2E65
:10199000F02D00E0802F9927FC01E95EF24F1681BF
:1019A000133238F4812F0E940D32882379F0EF280A
:1019B0000DC01E3238F4812F0E94B006882331F00A
:1019C000EF2804C01E3211F4A499EF28F6940F5F9B
:1019D000083000F3EE82EE240F2EF0E8FF2EF02DFB
:1019E0000E2D802F9927FC01E05AF24F16851332F5
:1019F00038F4812F0E94E731882379F0EF280DC059
:101A00001E3238F4812F0E94B006882331F0EF286F
:101A100004C01E3211F4A499EF28F6940F5F083029
:101A200000F3DD2029F10F2EF0E8FF2EF02D00E06D
:101A3000802F9927FC01E95EF24F1685133238F4A6
:101A4000812F0E940D32882379F0EF280DC01E32BD
:101A500038F4812F0E94B006882331F0EF2804C0AB
:101A60001E3211F4A499EF28F6940F5F083000F3AA
:101A7000EF82EE240F2EF0E8FF2EF02D0E2D802F9A
:101A80009927FC01E05AF24F1689133238F4812F5E
:101A90000E94E731882379F0EF280DC01E3238F418
:101AA000812F0E94B006882331F0EF2804C01E3237
:101AB00011F4A499EF28F6940F5F083000F3DD20AD
:101AC00029F10F2EF0E8FF2EF02D00E0802F99274E
:101AD000FC01E95EF24F1689133238F4812F0E941F
:101AE0000D32882379F0EF280DC01E3238F4812F93
:101AF0000E94B006882331F0EF2804C01E3211F492
:101B0000A499EF28F6940F5F083000F3E886EE24DE
:101B10000F2EF0E8FF2EF02D0E2D802F9927FC01BF
:101B2000E05AF24F168D133238F4812F0E94E731BC
:101B3000882379F0EF280DC01E3238F4812F0E94DF
:101B4000B006882331F0EF2804C01E3211F4A499A6
:101B5000EF28F6940F5F083000F3DD2029F10F2EF7
:101B6000F0E8FF2EF02D00E0802F9927FC01E95EC0
:101B7000F24F168D133238F4812F0E940D328823D4
:101B800079F0EF280DC01E3238F4812F0E94B00684
:101B9000882331F0EF2804C01E3211F4A499EF28F5
:101BA000F6940F5F083000F3E986EE240F2EF0E87C
:101BB000FF2EF02D0E2D802F9927FC01E05AF24FB9
:101BC00016A1133238F4812F0E94E731882379F06F
:101BD000EF280DC01E3238F4812F0E94B0068823F2
:101BE00031F0EF2804C01E3211F4A499EF28F694C6
:101BF0000F5F083000F3DD2029F10F2EF0E8FF2EF3
:101C0000F02D00E0802F9927FC01E95EF24F16A12C
:101C1000133238F4812F0E940D32882379F0EF2897
:101C20000DC01E3238F4812F0E94B006882331F097
:101C3000EF2804C01E3211F4A499EF28F6940F5F28
:101C4000083000F3EA86EE240F2EF0E8FF2EF02D88
:101C50000E2D802F9927FC01E05AF24F16A5133262
:101C600038F4812F0E94E731882379F0EF280DC0E6
:101C70001E3238F4812F0E94B006882331F0EF28FD
:101C800004C01E3211F4A499EF28F6940F5F0830B7
:101C900000F3DD2029F10F2EF0E8FF2EF02D00E0FB
:101CA000802F9927FC01E95EF24F16A5133238F414
:101CB000812F0E940D32882379F0EF280DC01E324B
:101CC00038F4812F0E94B006882331F0EF2804C039
:101CD0001E3211F4A499EF28F6940F5F083000F338
:101CE000EB868E859F856AE070E00E94DE6D6C87D2
:101CF0001D86CE0101960E9485478091B40C90917B
:101D0000B50C009709F414C1DD2009F011C1019749
:101D10009093B50C8093B40C892B09F009C1809184
:101D2000190D90911A0D6AE070E00E94DE6D7093BB
:101D3000B50C6093B40C80911B0D90911C0DAA27DB
:101D4000BB2789839A83AB83BC8388E08D83ED2C8A
:101D50000F2EF0E8FF2EF02D0D2D802F9927FC017E
:101D6000E95EF24F1681133238F4812F0E940D3252
:101D7000882379F0EF280DC01E3238F4812F0E949D
:101D8000B006882331F0EF2804C01E3211F4A49964
:101D9000EF28F6940F5F083000F3EE82EE240F2E4A
:101DA000F0E8FF2EF02D0E2D802F9927FC01E95E23
:101DB000F24F1685133238F4812F0E940D3288239A
:101DC00079F0EF280DC01E3238F4812F0E94B00642
:101DD000882331F0EF2804C01E3211F4A499EF28B3
:101DE000F6940F5F083000F3EF82EE240F2EF0E838
:101DF000FF2EF02D0E2D802F9927FC01E95EF24F6A
:101E00001689133238F4812F0E940D32882379F01D
:101E1000EF280DC01E3238F4812F0E94B0068823AF
:101E200031F0EF2804C01E3211F4A499EF28F69483
:101E30000F5F083000F3E886EE240F2EF0E8FF2E47
:101E4000F02D0E2D802F9927FC01E95EF24F168DA3
:101E5000133238F4812F0E940D32882379F0EF2855
:101E60000DC01E3238F4812F0E94B006882331F055
:101E7000EF2804C01E3211F4A499EF28F6940F5FE6
:101E8000083000F3E986EE240F2EF0E8FF2EF02D47
:101E90000E2D802F9927FC01E95EF24F16A1133217
:101EA00038F4812F0E940D32882379F0EF280DC07D
:101EB0001E3238F4812F0E94B006882331F0EF28BB
:101EC00004C01E3211F4A499EF28F6940F5F083075
:101ED00000F3EA86EE240F2EF0E8FF2EF02D0E2DF3
:101EE000802F9927FC01E95EF24F16A5133238F4D2
:101EF000812F0E940D32882379F0EF280DC01E3209
:101F000038F4812F0E94B006882331F0EF2804C0F6
:101F10001E3211F4A499EF28F6940F5F083000F3F5
:101F2000EB8688898C871D86CE0101960E948547A5
:101F300080915E0D90915F0D009709F488C1019723
:101F400090935F0D80935E0D892B09F080C1809185
:101F5000D30C9091D40C6AE070E00E94DE6D709317
:101F60005F0D60935E0D8091D50C9091D60CAA27E1
:101F7000BB2789839A83AB83BC8388E08D83EE245F
:101F80000F2EF0E8FF2EF02D0E2D802F9927FC014B
:101F9000EF52F34F1681133238F4812F0E94E7314C
:101FA000882319F1EF2821C01E3238F4812F0E94B6
:101FB000B0068823D1F0EF2818C01E3440F4812FDA
:101FC0008D520E943813882381F0EF280EC01236FC
:101FD00040F4812F8D520E94025E882331F0EF2859
:101FE00004C0123611F4A499EF28F6940F5F08305C
:101FF00060F2EE82EE240F2EF0E8FF2EF02D0E2D73
:10200000802F9927FC01EF52F34F1685133238F4D5
:10201000812F0E94E731882319F1EF2821C01E3259
:1020200038F4812F0E94B0068823D1F0EF2818C021
:102030001E3440F4812F8D520E943813882381F082
:10204000EF280EC0123640F4812F8D520E94025E9E
:10205000882331F0EF2804C0123611F4A499EF2838
:10206000F6940F5F083060F2EF82EE240F2EF0E856
:10207000FF2EF02D0E2D802F9927FC01EF52F34FEC
:102080001689133238F4812F0E94E731882319F121
:10209000EF2821C01E3238F4812F0E94B006882319
:1020A000D1F0EF2818C01E3440F4812F8D520E94C9
:1020B0003813882381F0EF280EC0123640F4812FA8
:1020C0008D520E94025E882331F0EF2804C0123640
:1020D00011F4A499EF28F6940F5F083060F2E886B7
:1020E000EE240F2EF0E8FF2EF02D0E2D802F9927D5
:1020F000FC01EF52F34F168D133238F4812F0E94FA
:10210000E731882319F1EF2821C01E3238F4812FDE
:102110000E94B0068823D1F0EF2818C01E3440F486
:10212000812F8D520E943813882381F0EF280EC032
:10213000123640F4812F8D520E94025E882331F0C6
:10214000EF2804C0123611F4A499EF28F6940F5F1B
:10215000083060F2E986EE240F2EF0E8FF2EF02D15
:102160000E2D802F9927FC01EF52F34F16A1133249
:1021700038F4812F0E940D32882331F0EF2804C0FB
:10218000133211F4A499EF28F6940F5F083048F346
:10219000EA86EE240F2EF0E8FF2EF02D0E2D802F74
:1021A0009927FC01EF52F34F16A5133238F4812F13
:1021B0000E940D32882331F0EF2804C0133211F44D
:1021C000A499EF28F6940F5F083048F3EB86EE24CD
:1021D0000F2EF0E8FF2EF02D0E2D802F9927FC01F9
:1021E000EF52F34F16A9133238F4812F0E940D32AB
:1021F000882331F0EF2804C0133211F4A499EF289A
:10220000F6940F5F083048F3EC86EE240F2EF0E8CA
:10221000FF2EF02D0E2D802F9927FC01E15FF24F4C
:102220001081133238F4812F0E940D32882331F04F
:10223000EF2804C0133211F4A499EF28F6940F5F2D
:10224000083048F3ED86CE0101960E9485476596D9
:102250000FB6F894DEBF0FBECDBFDF91CF911F91B7
:102260000F91FF90EF90DF9008958091A60D9091CF
:10227000A70D885E934031F084EF91E09093A70D15
:102280008093A60D8FE090E09093A90D8093A80D08
:1022900089E999E09093AB0D8093AA0D1092AC0D53
:1022A0001092AD0D1092AE0D1092AF0D1092B10DB7
:1022B0001092B00D84E18093B50DE6EAFDE0A0E850
:1022C000B0E080E190E021E08030920719F40E94B4
:1022D000926E0895182E0E94926E0895BF92CF922A
:1022E000DF92EF92FF920F931F93CF93DF93CDB7BF
:1022F000DEB7AE970FB6F894DEBF0FBECDBFBB24DE
:10230000BE016F5F7F4F8B2D0E943A388B2D99272E
:102310009C0122953295307F3227207F3227B901E8
:102320006E527E4F9981492F4170DB018C91887FDD
:102330009670842B892B8C930F2EF3ECCF2EF1E02B
:10234000DF2EF02DC20ED31E8A819B81F601918370
:1023500080838C819D81938382834E815F815583AD
:1023600044838885998597838683D901A553BE4F79
:102370002A858B85982F9295907F822F8F70892B3D
:102380008C938C8581878D8582878E8583878F85C9
:1023900084878F8D8170982F990F990F990FFB016A
:1023A0008081877F892B808388A1F601858789A119
:1023B00086878AA18170982F9295907FFB018081FA
:1023C0008F7E892B80838C918F70833090F5CA012A
:1023D000AA2797FDA095BA2FBC01CD010E94F66AED
:1023E000DC01CB0128A539A54AA55BA5BC01CD011F
:1023F0000E94106A7B018C018CA5992787FD90951E
:10240000A92FB92FBC01CD010E94F66ADC01CB01D6
:102410009C01AD01C801B7010E94DB69DC01CB0161
:10242000BC01CD010E945C68DC01CB01F601958303
:1024300084838B2D99279C0122953295307F3227FA
:10244000207F3227F901E553FE4F808182958F70FE
:102450008330D8F50F2EF3ECCF2EF1E0DF2EF02DE8
:10246000C20ED31E88859985AA2797FDA095BA2FFD
:10247000BC01CD010E94F66ADC01CB0128A539A57B
:102480004AA55BA5BC01CD010E94106A7B018C01AD
:102490008CA5992787FD9095A92FB92FBC01CD0157
:1024A0000E94F66ADC01CB019C01AD01C801B701B5
:1024B0000E94DB69DC01CB01BC01CD010E945C689C
:1024C000DC01CB01F601978386838B2D99278295BA
:1024D0009295907F9827807F9827FC01EE52FE4FBF
:1024E000808186958370813011F0833041F48B2D8B
:1024F0009927FC01ED53FC4F81E0808306C08B2DB2
:102500009927FC01ED53FC4F10822B2D3327C90175
:1025100082959295907F9827807F9827FC01EE52B4
:10252000FE4F80818F798083C901820F931FFC0148
:10253000EE50FC4F11821082B394FFE1FB1508F0BE
:10254000DFCEFE01BD96A3E3B8E082E090E021E09B
:102550008030920719F40E94816E03C0182E0E94E9
:10256000816E8DA58093F0038EA58093F103109268
:10257000E4031092E303AE960FB6F894DEBF0FBEED
:10258000CDBFDF91CF911F910F91FF90EF90DF9022
:10259000CF90BF9008951F93CF93DF93CDB7DEB751
:1025A000AE970FB6F894DEBF0FBECDBF10E0A89572
:1025B0008981887F89831B821A821D821C821F82E7
:1025C0001E82198618861A861B861C8681E08D87D6
:1025D0001E868F871F8E18A219A21AA280E090E093
:1025E000A0E8BFE388A799A7AAA7BBA71CA685E078
:1025F000FE01B39611928A95E9F78FE0FE0170967D
:10260000DF01282F1D922A95E9F7189FC001112498
:1026100086559E4FBC01CF010E94816DBE016F5F48
:102620007F4F812F0E9402381F5F103208F4BFCF06
:102630001EA61DA6FE01BD96A3E3B8E082E090E0D1
:1026400021E08030920719F40E94926E03C0182E88
:102650000E94926EA895AE960FB6F894DEBF0FBE9C
:10266000CDBFDF91CF911F9108958093E30308952B
:102670000F93CF93DF93CDB7DEB721970FB6F894C2
:10268000DEBF0FBECDBF89838150803270F000E085
:1026900021E0AE014F5F5F4F63E171E081E091E0C7
:1026A0000E94233480E090E007C089819927FC01D3
:1026B000EE53FC4F8081992721960FB6F894DEBF28
:1026C0000FBECDBFDF91CF910F9108958091F003A0
:1026D0008823E1F08091F1030E94024A8823B1F43B
:1026E000482F83EC93E0FC01E40FF11D10824F5F53
:1026F0004032C8F31092880010928A0080918000C6
:102700008F758093800085B18F7985B98091BD0DDB
:10271000882359F081508093BD0D882331F4809136
:1027200080008F7D809380002E988091B70D882344
:1027300059F081508093B70D882331F48091800047
:102740008F77809380002D9840E062EF73E0A3ECD8
:10275000B3E051E0242F3327C901820F931FFC01FE
:10276000E60FF71F80819181009791F10197918386
:102770008083892B69F5C90182959295907F98276E
:10278000807F9827FC01EE52FE4F808186958370F2
:1027900099278130910551F08130910514F004970B
:1027A0004CF0FD01E40FF11D108204C0FD01E40FA7
:1027B000F11D5083842F992782959295907F9827B9
:1027C000807F9827FC01EE52FE4F80818F798083B5
:1027D0004F5F403208F4BECF08958091E303882311
:1027E00099F08091E403882379F084EE93E0AC01C2
:1027F0004C5F5F4F6091E7038091E5039091E603A2
:102800000E9423581092E40308958F929F92AF92F2
:10281000BF92CF92DF92EF92FF920F931F93CF93CD
:10282000DF938C01EE24FF2499248091F003882308
:1028300039F08091F1030E94024A882309F4DAC238
:102840006091CF0D683070F58091CD0D9091CE0DD7
:102850009C0144275527F80180819181A281B38191
:1028600082179307A407B507E9F4E60FF11D8581E8
:1028700080938A0080918A00882351F08091B80D5E
:10288000882331F08091800080628093800006C0B0
:10289000809180008F7D809380002E988091A80D7C
:1028A0008093BD0D6091D20D683070F58091D00D90
:1028B0009091D10D9C0144275527F8018081918189
:1028C000A281B38182179307A407B507E9F4E60F45
:1028D000F11D85818093880080918800882351F0C4
:1028E0008091C90D882331F08091800080688093A9
:1028F000800006C0809180008F77809380002D98A3
:102900008091A80D8093B70D8091AA0D9091AB0D89
:102910009C0144275527F80180819181A281B381D0
:1029200082179307A407B50799F48091AC0DE80FBF
:10293000F11D85819091AD0D8923891749F40E947D
:102940009B590E9406261092E10D82E280931101AC
:1029500060E07091E3030F2EF3ECAF2EF3E0BF2E97
:10296000F02D88248394C090A80DD090A90D862FB7
:10297000992782959295907F9827807F9827EC01E0
:10298000CD53DE4F88819981AA27BB27F80120818A
:1029900031814281538182179307A407B50749F01B
:1029A0008A819B81AA27BB2782179307A407B507B3
:1029B000C1F4462F5527CA01840F951FFC01EE5024
:1029C000FC4FD182C082872F733048F099279C0139
:1029D0002F733070CA0103962817390711F4992410
:1029E00093948F8583FF09C08D85F801E80FF11D51
:1029F0009E858581981709F0AAC128813981211502
:102A0000310509F4A4C144275527F801808191813B
:102A1000A281B381281739074A075B0709F0C3C0B1
:102A200091E08985882379F0E80FF11D8481E82EF3
:102A3000FF24FE2CEE248A85F801E80FF11D848125
:102A4000E80EF11C14C08A85882381F0F801E80F94
:102A5000F11D8481E82EFF248F8584FF08C0EE20BD
:102A600034F420E03FEFE22AF32A01C090E09923FA
:102A700009F499C088858F7099278330910509F4EE
:102A800055C0843091054CF481309105E9F08230D5
:102A900091059CF5892B69F086C08530910509F474
:102AA0005BC0853091050CF44CC0069709F45EC0FC
:102AB0007AC08C819D818E159F0509F074C0F50147
:102AC000E60FF11D80826FC08F8584FF0BC08C8163
:102AD0009D818E159F050CF066C0F501E60FF11D76
:102AE000808261C08C819D818E159F0508F05BC03E
:102AF000F501E60FF11D808256C08F8584FF0BC063
:102B00008C819D81E816F9060CF04DC0F501E60FA9
:102B1000F11D808248C08C819D81E816F90608F07D
:102B200042C0F501E60FF11D80823DC08C819D8180
:102B30008E219F21892BB9F1F501E60FF11D8082CD
:102B400032C08C819D818E219F21892B61F5F501F9
:102B5000E60FF11D808227C08C819D818E159F0517
:102B600011F1F501E60FF11D80821DC08C819D8160
:102B70008E219F21892BA1F08F85982F907285FD42
:102B800012C080628F87F501E60FF11D80818130D0
:102B900011F4908308C0F501E60FF11D808203C097
:102BA0008F858F7D8F878A819B819C014427552744
:102BB000F80180819181A281B381281739074A07E2
:102BC0005B0709F0C4C091E08B85882379F0E80F9A
:102BD000F11D8481E82EFF24FE2CEE248C85F80163
:102BE000E80FF11D8481E80EF11C14C08C85882348
:102BF00081F0F801E80FF11D8481E82EFF248F8514
:102C000084FF08C0EE2034F420E03FEFE22AF32AEC
:102C100001C090E0992309F49AC0888582958F704D
:102C200099278330910509F455C0843091054CF4FF
:102C300081309105E9F0823091059CF5892B69F08E
:102C400086C08530910509F45BC0853091050CF490
:102C50004CC0069709F45EC07AC08E819F818E15A4
:102C60009F0509F074C0F501E60FF11D10826FC0D9
:102C70008F8584FF0BC08E819F818E159F050CF080
:102C800066C0F501E60FF11D108261C08E819F8143
:102C90008E159F0508F05BC0F501E60FF11D10824F
:102CA00056C08F8584FF0BC08E819F81E816F90680
:102CB0000CF04DC0F501E60FF11D108248C08E8169
:102CC0009F81E816F90608F042C0F501E60FF11DF4
:102CD00010823DC08E819F818E219F21892BB9F169
:102CE000F501E60FF11D108232C08E819F818E2189
:102CF0009F21892B61F5F501E60FF11D108227C098
:102D00008E819F818E159F0511F1F501E60FF11D52
:102D100010821DC08E819F818E219F21892BA1F061
:102D20008F85982F907486FD12C080648F87F5017F
:102D3000E60FF11D8081813011F4908308C0F50108
:102D4000E60FF11D808203C08F858F7B8F876F5FB9
:102D5000603208F40CCE8091E303882309F44AC062
:102D6000992019F4823009F045C08091E403823043
:102D700009F440C08091E5039091E6039C0144274B
:102D80005527F80180819181A281B38128173907E5
:102D90004A075B0799F49091E7038481981771F4CF
:102DA000892F992798012B5F3F4FAC01B90184EE21
:102DB00093E004960E94886D892BC9F082E080938D
:102DC000E403F80124812093E703808191819093AB
:102DD000E6038093E503822F992798012B5F3F4FED
:102DE000AC01B90188EE93E00E94956D03C081E0CB
:102DF0008093E403DF91CF911F910F91FF90EF90AB
:102E0000DF90CF90BF90AF909F908F9008950E94D9
:102E10006A058091D80082608093D8000895CF938E
:102E2000DF93EC018981833089F48985882309F453
:102E300003C188818295807F8093ED008091EF00AF
:102E40008F738093EF0018821986F6C00E948E055A
:102E5000982F81E089879F3F09F4EBC09883892FE1
:102E60008295807F8093ED001092EE001092EF002B
:102E70001092F7001092F6001092F5001092F400F4
:102E80001092F000898199278130910509F46BC077
:102E9000823091051CF4892B29F0C9C0029709F4EE
:102EA000BBC0C5C08A8581FF30C08D81982F990F26
:102EB000990F990F8C81829586958770890F8093E1
:102EC000F3008C81982F990F990F990F8B81829520
:102ED00086958770890F8093F2008B81982F990FC8
:102EE000990F990F8A81829586958770890F8093B3
:102EF000F1008A81880F880F880F8093F0008091FD
:102F0000EF0080618093EF0012C08B81982F929523
:102F1000990F907E8A81869586958695890F8093F4
:102F2000F3008A818295880F807E8093F20020E0F2
:102F30008E81181660F48F819885FC01E20FF11DD7
:102F400080818093FA002F5F8E812817A0F39091E3
:102F5000EF008E81892B8093EF008091EF008064D9
:102F60008093EF0069C08A8581FF35C08D81982FDD
:102F7000990F990F990F8C81829586958770890F8B
:102F80008093F3008C81982F990F990F990F8B8163
:102F9000829586958770890F8093F2008B81982F98
:102FA000990F990F990F8A81829586958770890F5D
:102FB0008093F1008A81880F880F880F8093F0003A
:102FC0008091EF0080618093EF008091F000846039
:102FD0008093F00015C08B81982F9295990F907E69
:102FE0008A81869586958695890F8093F3008A81DC
:102FF0008295880F807E8093F20084E08093F000B9
:103000009091EF008E81892B8093EF008091EF00EB
:1030100080648093EF0010C08091EF008F738093E5
:10302000EF008091EF0080688093EF0005C0198663
:1030300003C08FEF90E002C080E090E0DF91CF917D
:103040000895CF93DF93EC018985882319F482E0FA
:1030500090E082C088818295807F8093ED000E94FD
:10306000A805813009F06CC019868091EF008F703F
:103070008E838F8198850E94C0058091F0009927EA
:10308000847090709595879595958795982F9170F8
:103090008A85282F2E7F292B2A878091EF0084FF95
:1030A00031C0822F82608A878091F3008695869551
:1030B00086958D838091F200982F9695969596959A
:1030C0008091F3008295880F807E890F8C83809198
:1030D000F100982F9695969596958091F20082959D
:1030E000880F807E890F8B838091F000982F9695B2
:1030F000969596958091F1008295880F807E890F34
:103100008A8316C08A858D7F8A878091F300829595
:10311000869587708B838091F200982F9295969573
:1031200097708091F300880F880F880F890F8A832A
:103130008091EF008F738093EF0080E090E00CC0EF
:10314000882349F489878091EF008F738093EF0083
:1031500080E090E001C09927DF91CF910895982FEA
:103160008F3F19F481E090E00895805C843128F469
:10317000892F0E94024A99270895892F8150803211
:1031800028F4892F0E94381399270895892F815296
:10319000843128F4892F0E94025E99270895892F8F
:1031A00087538C3028F4892F0E941F269927089571
:1031B00080E090E00895982F8F3F19F481E090E02F
:1031C0000895805C843128F4892F0E94E148992772
:1031D0000895892F8150803228F4892F0E94381356
:1031E00099270895892F8152843128F4892F0E94CC
:1031F000025E99270895892F87538C3028F4892FF0
:103200000E941F269927089580E090E008958091FC
:10321000BF0D9091C00D01969093C00D8093BF0D8E
:103220008091CB0D9091CC0D01969093CC0D809315
:10323000CB0D8091BB0D9091BC0D01969093BC0D70
:103240008093BB0D8091CA0D833008F46DC08F5FF1
:103250008093CA0D843029F441E061E40E948341E7
:1032600063C08091BF0D9091C00D8035910598F499
:103270008091CA0D853031F441E061E484E00E9420
:103280000E4252C08091CA0D883009F04DC083E0D3
:103290008093CA0D49C08091BF0D9091C00D803AB6
:1032A000910590F48091CA0D853031F441E061E4DC
:1032B00084E00E940E4238C08091CA0D8730A0F190
:1032C00083E08093CA0D30C08091BF0D9091C00DF6
:1032D0008856914090F48091CA0D863031F441E0D7
:1032E00061E484E00E940E421FC08091CA0D8730C5
:1032F000D8F083E08093CA0D17C08091BF0D9091E4
:10330000C00D8E5F914068F48091CA0D873060F0E7
:1033100041E061E484E00E940E4283E08093CA0DA4
:1033200003C081E08093CA0D8091BA0D833008F408
:103330006DC08F5F8093BA0D843031F440E061E45A
:1033400086E00E94834162C08091CB0D9091CC0DAC
:103350008035910598F48091BA0D853031F440E0C4
:1033600061E486E00E940E4251C08091BA0D88301F
:1033700009F04CC083E08093BA0D48C08091CB0D1A
:103380009091CC0D803A910590F48091BA0D8530E2
:1033900031F440E061E486E00E940E4237C0809143
:1033A000BA0D873098F183E08093BA0D2FC08091D9
:1033B000CB0D9091CC0D8856914088F48091BA0D38
:1033C000863029F440E061E40E940E421FC08091E3
:1033D000BA0D8730D8F083E08093BA0D17C0809182
:1033E000CB0D9091CC0D8E5F914068F48091BA0D19
:1033F000873060F040E061E486E00E940E4283E0A6
:103400008093BA0D03C081E08093BA0D8091BE0D08
:10341000833008F46DC08F5F8093BE0D843031F42B
:1034200041E061E486E00E94834108958091BB0DF4
:103430009091BC0D8035910598F48091BE0D85303A
:1034400031F441E061E486E00E940E4208958091EB
:10345000BE0D883009F04CC083E08093BE0D089506
:103460008091BB0D9091BC0D803A910590F48091B4
:10347000BE0D853031F441E061E486E00E940E42E9
:1034800008958091BE0D873098F183E08093BE0D42
:1034900008958091BB0D9091BC0D8856914088F4A1
:1034A0008091BE0D863029F441E061E40E940E4215
:1034B00008958091BE0D8730D8F083E08093BE0DD3
:1034C00008958091BB0D9091BC0D8E5F914068F482
:1034D0008091BE0D873060F041E061E486E00E949B
:1034E0000E4283E08093BE0D089581E08093BE0D6F
:1034F00008958091C20D0E94AF18882321F085E0C5
:103500008093B90D46C08091C70D0E94AF188823E3
:1035100041F08091C80D8093EE0983E08093B90D4E
:1035200038C08091C10D0E94AF18882321F084E03B
:103530008093B90D2EC08091C30D0E94AF188823CF
:1035400069F08091B90D873049F0863039F086E016
:103550008093B90D8AE08093ED091BC08091B90D6D
:10356000853021F482E08093B90D13C08091B90DAC
:10357000833041F48091EE09882321F481E0809327
:10358000B90D07C08091B90D843019F481E08093A2
:10359000B90D8091B90D8150823058F48091C40DDD
:1035A0000E94DB189091C50D981719F41092B90D6F
:1035B00017C08091ED09882399F48091B90D863068
:1035C00079F48091C40D0E94DB189091C50D981775
:1035D00039F487E08093B90D8091C60D8093EC0992
:1035E0000E94051D08951F93CF93DF9310E0812F54
:1035F00099279C01220F331FE901C80FD91FFE0133
:10360000EB52F24F8181882359F00E94AF18882332
:1036100039F0FE01E952F24F80818F78808304C136
:10362000812F99279C01220F331FE901C80FD91F51
:10363000FE01EB52F24F8081882309F4E8C00E941A
:10364000AF18882309F4E3C0FE01E952F24F8081EC
:1036500083FDEAC088608083877099278230910556
:1036600089F1833091051CF4019749F0DDC0833066
:10367000910509F467C0049709F4BAC0D5C0212F99
:103680003327C901880F991F820F931FFC01E9524C
:10369000F24F9081892F82958F70877021F0892F4A
:1036A0008F788083C1C0212F3327C901880F991FCC
:1036B000820F931FFC01E952F24F80818F78806165
:1036C0008083B2C0212F3327C901880F991F820F31
:1036D000931FFC01E952F24F808182958F708770B1
:1036E0009927009719F0019781F01EC0212F3327E9
:1036F000C901880F991F820F931FFC01E952F24FF5
:1037000080818F78806180838FC0212F3327C9010A
:10371000880F991F820F931FFC01E952F24F80819D
:103720008F788062808380C0212F3327C901880F62
:10373000991F820F931FFC01E952F24F80818F780D
:10374000808372C0212F3327C901880F991F820FF0
:10375000931FFC01E952F24F808182958F70877030
:10376000992781309105C1F0823091051CF4892B95
:1037700021F030C00297F9F02DC0212F3327C90165
:10378000880F991F820F931FFC01E952F24F80812D
:103790008F788061808348C0212F3327C901880F2B
:1037A000991F820F931FFC01E952F24F80818F789D
:1037B0008062808339C0212F3327C901880F991F68
:1037C000820F931FFC01E952F24F80818F78806352
:1037D00080832AC0212F3327C901880F991F820FA8
:1037E000931FFC01E952F24F80818F7880831CC0C7
:1037F000212F3327C901880F991F820F931FFC01C6
:10380000E952F24F80818F78806180830DC0212F33
:103810003327C901880F991F820F931FFC01E952BA
:10382000F24F8081877F80831F5F143008F4DFCEE2
:103830000E94DA260E940B250E94782810E085E27B
:10384000189FC0011124EC01C95CDB4F8C899D8954
:10385000009719F001979D8B8C8B8C85882384F0C1
:103860008D859E85009761F001979E878D8799854C
:103870009F3F31F085E0989FC00111249B878A8784
:103880002A853B852115310561F089858F3F49F0F7
:10389000C90101979B878A87892B19F48F858062DC
:1038A0008F878A8D9B8D009779F001979B8F8A8FE8
:1038B000892B51F48F8586FD04C0812F8F5F0E9474
:1038C00003378F8580648F878F81882311F0815023
:1038D0008F831F5F123208F4B2CFDF91CF911F9117
:1038E00008958091ED09882319F081508093ED09A6
:1038F0008091B90D8730B9F48091EC09882321F0CB
:1039000081508093EC090FC08091C30D0E94AF18C5
:10391000882339F086E08093B90D8AE08093ED0921
:1039200002C01092B90D8091EE09882319F08150E0
:103930008093EE09A49B23C02091E9092F3710F44E
:10394000220F01C02FEF8091AE0D8A30D0F0909100
:10395000B60D981710F0921730F48091B60D8F5F66
:103960008093B60D0EC08091E10D882351F48F5FD6
:103970008093E10D0E949B590E94062602C010927E
:10398000B60D90915B09809160099817E0F420E0F2
:1039900040E659E065E270E0FA01E20FF11D828134
:1039A000823268F49927869FF001879FF00D969FD9
:1039B000F00D1124E55CFB4F8081816080832F5FD7
:1039C0002C3050F3089590915B098091610989171B
:1039D000D8F420E040E659E065E270E0FA01E20F39
:1039E000F11D8281823268F49927869FF001879FBA
:1039F000F00D969FF00D1124E55CFB4F80818E7FCA
:103A000080832F5F2C3050F30895CF92DF92EF9296
:103A1000FF920F931F93CF93DF93809133048823FA
:103A200009F030C1F82E0F2EFAE0EF2EF02D8F2D79
:103A3000992782959295907F9827807F9827EC010F
:103A4000C756D64F00E08A818F3F11F401E045C090
:103A50009A81892F805C843128F4892F0E94024A40
:103A6000082F3BC09A81892F8150803228F4892FFA
:103A70000E943813082F31C09A81892F81528431D6
:103A800028F4892F0E94025E082F27C08A8183367E
:103A900071F49091B90D892F8350823020F09130CC
:103AA00011F0963011F401E018C000E016C08A81D0
:103AB000843651F48091B90D853011F0823011F4C3
:103AC00001E00BC000E009C09A81892F87538C3038
:103AD00020F4892F0E941F26082F89819927813081
:103AE0009105C9F1823091051CF4892B29F0C5C0DC
:103AF000029709F4BFC0C1C0013009F0BEC08F8178
:103B00008E9DC00111249C838B8389858E9DC0016D
:103B100011249E838D8388818460888310E025E250
:103B200030E0FE01E10FF11D82858F3F71F0992792
:103B3000829FA001839F500D929F500D1124FA0186
:103B4000E55CFB4F8081846080831F5F163048F303
:103B500081E0898392C08B819C81009709F48DC09C
:103B600001979C838B83892B81F5288122FF17C0C5
:103B70008F818E9DC00111249C838B83822F8B7F2C
:103B8000888310E0FE01E10FF11D82858F3F19F05F
:103B900060E00E944B1E1F5F1630A0F316C08885A0
:103BA0008E9DC00111249C838B83888184608883CF
:103BB00010E0FE01E10FF11D82858F3F19F061E0F9
:103BC0000E944B1E1F5F1630A0F38881282F2270A1
:103BD00081FD28C08D819E81009709F44EC0019718
:103BE0009E838D83892B09F048C082E08983122F40
:103BF00025E230E0FE01E10FF11D82858F3F71F07B
:103C00009927829FA001839F500D929F500D1124F0
:103C1000FA01E55CFB4F80818B7F80831F5F16304C
:103C200048F32BC0002349F5102F0F2EF5E2CF2EBD
:103C3000DD24F02DFE01E10FF11D22852F3F99F0CB
:103C4000822F99278C9DA0018D9D500D9C9D500D1C
:103C50001124FA01E55CFB4F80818B7F808361E05A
:103C6000822F0E944B1E1C821B821F5F163010F396
:103C7000198203C0002309F40983F39454E05F150B
:103C800008F0D5CEDF91CF911F910F91FF90EF906B
:103C9000DF90CF900895DF92EF92FF920F931F93E2
:103CA000CF93DF93CDB7DEB721970FB6F894DEBF81
:103CB0000FBECDBF8983162FDD24833260F00D2D1A
:103CC00021E0AE014F5F5F4F6BE173E082E191E075
:103CD0000E9423344EC0998185E2989F700111247F
:103CE00087E394E0E80EF91EF701858D9927807F20
:103CF0009070803A910529F40F2EF1E4DF2EF02D1B
:103D000018C0F701858D9927807F9070803B9105C1
:103D100029F40F2EF2E4DF2EF02D0BC000E021E09D
:103D2000AE014F5F5F4F67E273E082E191E00E9476
:103D30002334112379F483E0F701878380EF8183B3
:103D400087858F7B8787858D41A16D2D8F700E9420
:103D500083410FC0113069F4F70117828FE081832E
:103D6000878586798787858D41A16D2D8F700E940B
:103D70000E4221960FB6F894DEBF0FBECDBFDF9185
:103D8000CF911F910F91FF90EF90DF90089520E069
:103D90004EE659E065E270E08170382F330FFA018A
:103DA000E20FF11D8181823270F49927869FF00124
:103DB000879FF00D969FF00D1124E55CFB4F8081ED
:103DC0008D7F832B80832F5F243148F3089520E07B
:103DD0004EE659E065E270E08170382F330FFA014A
:103DE000E20FF11D8789823270F49927869FF001D6
:103DF000879FF00D969FF00D1124E55CFB4F8081AD
:103E00008D7F832B80832F5F243148F30895809129
:103E100035049091360408958091340499270895CB
:103E2000EF92FF921F93CF93DF937A018093600903
:103E30006093610910E0C12FDD27F701EC0FFD1F32
:103E400080810E942130823220F4FE01E05AF64F38
:103E500082831F5F1C3078F3DF91CF911F91FF9019
:103E6000EF9008955F926F927F928F929F92AF92A0
:103E7000BF92CF92DF92EF92FF920F931F93CF9357
:103E8000DF93CDB7DEB722970FB6F894DEBF0FBE33
:103E9000CDBFAA240E945532109259091092580998
:103EA000A0925A09A0925C09A0925D09A0925E09B5
:103EB000A0925F0982E1E1E2F9E011928A95E9F7C7
:103EC00043E359E028EB31E08A2D9927880F991FA9
:103ED000FC01E40FF51F31832083A39461E16A158F
:103EE00098F7AA2429E939E08A2D99278295929595
:103EF000907F9827807F9827FC01E20FF31F1182A3
:103F00001482138216821582FC01E756F64F8081D7
:103F100084608083A39474E07A1530F70E94923A0B
:103F2000803221F487E68093100103C08EE68093EF
:103F300010010F2EF7E38F2EF4E09F2EF02D41E0BD
:103F40004093370428EC30E030934A04209349042E
:103F500052EA5093540462EB609355041092580453
:103F60009FEF909356045093570483E08093590435
:103F700084010B5D1F4F40935C04F40130AF27AB0D
:103F8000F801558F668F41A3978F0F2EF7EAEF2E1A
:103F9000F02DE0A20F2EFFE0BF2EF02DB2A2F40113
:103FA000E65BFF4F40938104338B228B0F2EF3EAA5
:103FB000DF2EF02DD58E83EB868F41A3978F90A3B4
:103FC00089E082A3F401E159FF4F4093A604338BAB
:103FD000228BE58E0F2EF7EBCF2EF02DC68E41A350
:103FE000978F90A38BE082A3F401EC56FF4F409390
:103FF000CB04338B228B11EA158F0F2EF1EBFF2EA2
:10400000F02DF68E41A3978F90A38EE082A3F4014A
:10401000E754FF4F4093F004338B228B55EA558FC2
:1040200005EB068F41A3978F90A38DE082A30F2EFF
:10403000F6E0AF2EF02DF401E252FF4F409315054C
:10404000338B228B60EA658F70EB768F11A2978F8E
:1040500050A3A2A2F401ED5FFE4F40933A05338BCB
:10406000228B558F068F11A2978F90A384E082A395
:10407000F401E85DFE4F40935F05338B228B658F23
:10408000768F41A3978F60A38AE082A3F401E35B5C
:10409000FE4F40938405338B228B758F54EB568FE4
:1040A00075E071A3978F90A382E182A3F401EE588B
:1040B000FE4F4093A905338B228B64EA658F568FA0
:1040C00041A3978FD0A288E082A3F401E956FE4F66
:1040D0004093CE05338B228B56EA558F86EB868F25
:1040E00011A2978F60A342A30F2EFCE0AF2EF02DFC
:1040F000F401E454FE4F4093F305338B228B558F2C
:10410000868F41A3978F10A3A2A2F401EF51FE4F17
:1041100040931806338B228BE58EC68E11A2978FA3
:1041200090A382E082A3F401EA5FFD4F40933D0635
:10413000338B228B158FF68E11A2978F90A387E079
:1041400082A3F401E55DFD4F40936206338B228B21
:10415000F58E068F71A3978F2B2D3327A40185E24F
:1041600090E0289FB001299F700D389F700D112499
:10417000FB01E80DF91D9FEF90A381E182A3F401FB
:10418000E05BFD4F61E06093870628EC30E0338B05
:10419000228B0F2EF4EA6F2EF02D658E0F2EF4EB8E
:1041A000FF2EF02DF68E11A2978F0F2EF6EAEF2E2E
:1041B000F02DE0A285E082A3F401EB58FD4F60935F
:1041C000AC06338B228B8D2CD58E03EB068F11A280
:1041D000978F90A312A2FA01E656FD4F70E47093F8
:1041E000D1062FEF3FEF338B228B0F2EF7EADF2E16
:1041F000F02DD58EF68E63E061A3E78E90A392A397
:10420000FA01E154FD4F7093F606338B228BE58E55
:1042100015EB168F61A3E78E90A392A3FA01EC51E0
:10422000FD4F70931B07338B228B0F2EF5EACF2E99
:10423000F02DC58E0F2EF6EB7F2EF02D768E61A31E
:10424000D78E90A392A3FA01E75FFC4F70934007CB
:10425000338B228B658E87EB868F61A3D78E90A3DD
:1042600092A3FA01E25DFC4F70936507338B228BBA
:1042700080EA858F068F61A3C78E90A392A3FA016F
:10428000ED5AFC4F70938A07338B228B0F2EF1EA85
:10429000BF2EF02DB58E0F2EF2EBAF2EF02DA68E89
:1042A00061A3C78E90A392A3FA01E858FC4F7093C4
:1042B000AF07338B228B0F2EF2EA9F2EF02D958EB7
:1042C0000F2EF1EB5F2EF02D568E61A3678E90A31B
:1042D00092A3FA01E356FC4F7093D407338B228BE1
:1042E000858E0F2EF0EBCF2EF02DC68E61A3678E3C
:1042F00090A392A3FA01EE53FC4F7093F907338B0E
:10430000228B858F068F82E081A3178F90A392A3C3
:10431000FA01E951FC4F70931E08338B228BB58E46
:10432000A68E81A3178F90A392A3FA01E45FFB4F9F
:1043300070934308338B228B958E568E81A3F78E14
:1043400090A392A3FA01EF5CFB4F70936808338B44
:10435000228B858EC68E81A3F78E90A392A3FA013D
:10436000EA5AFB4F70938D08338B228BD58EF68ED5
:1043700081A3778E90A392A3FA01E558FB4F709327
:10438000B208338B228BE58EFA01E558FB4F168F6E
:104390009A01FA01E558FB4F52E051A3778E4FEF97
:1043A00040A342A3F901E056FB4FB72F7093D70803
:1043B0006FEF7FEF738B628B85EA858F768E51A3CB
:1043C00097EB978F40A342A3F901EB53FB4FB093B8
:1043D000FC08738B628B658E968F51A3978F40A3D9
:1043E00042A3AA24790105E210E07FE06A2D0F2E96
:1043F000F1E2BF2EF02D0F2EFEE19F2EF02D8A2D23
:104400009927809F9001819F300D909F300D11243E
:104410006901CE0CDF1CF601158A148AA901455CDE
:104420005B4FDA018C918C7D8C931786168A718391
:1044300014A213A2168615862D5B3B4FF9016083EB
:10444000F6011386128661878C918B7F8C93678B24
:104450006783B086968280E185837283118E108E89
:10446000138E128E648FA394F1E2FA1540F6229611
:104470000FB6F894DEBF0FBECDBFDF91CF911F9175
:104480000F91FF90EF90DF90CF90BF90AF909F90F3
:104490008F907F906F905F900895E1E2F9E082E164
:1044A000DF011D928A95E9F7CF010E94C43920E00F
:1044B00063E379E048EB51E0822F9927880F991F39
:1044C000FC01E60FF71F518340832F5F2231A0F3D9
:1044D00083E399E00E94E4390895AF92BF92CF92AE
:1044E000DF92EF92FF920F931F93CF93DF93CDB79D
:1044F000DEB7C15DD0400FB6F894DEBF0FBECDBFB2
:1045000010E00F2EF5E6EF2EFF24F02DEC0EFD1E31
:10451000012FD7011C9288ECF70181838AE0828306
:1045200015821482168280E1838317828FE0189FA0
:10453000C001112486589B4FBC01C70108960E94F8
:10454000816DF701078B008F1F5F612FC7010E94EC
:10455000E238A8951232E8F28E0102581F4F84E625
:10456000D8018C9388E7F80181834CE050E06FEF2D
:1045700070E0C80102960E94A26DC8010E944237F5
:104580008E0104571F4FF80181EC819344E150E004
:104590006FEF70E0CF010E94A26DF801158A8AE0EA
:1045A000868B44E150E06FEF70E0C80147960E94AF
:1045B000A26DC8010E947037A89510E00F2EF4E19B
:1045C000CF2EF02D7E010894E11CF11C0F2EFFE090
:1045D000DF2EF02D01E0D701EC2D1D92EA95E9F7D1
:1045E0001D9DC00111248B529C4FBC01C7010E942C
:1045F000816D088B1F5FB701812F0E947939A895C3
:104600001B3048F310E00F2EF3ECAF2EBB24F02D3F
:10461000AC0EBD1E0F2EFFE0CF2EF02D0F2EF7EBB0
:10462000EF2EFF24F02DEC0EFD1EDD24D3940FEFB2
:10463000D501EC2D1D92EA95E9F71C9DC0011124CE
:1046400086579C4FBC01C7010C960E94816DD70113
:104650001C92F70111821282D382D4828AE0858370
:104660008081F701E80FF11D06838F5F8630C8F364
:10467000BE0169547F4F812F0E949037A8951F5F1C
:104680001530B0F2EDECFDE088E0DF011D928A9577
:10469000E9F7A5ECBAE088E090E021E080309207ED
:1046A00019F40E94926E03C0182E0E94926E8FEF32
:1046B0008093CF0D8093D20DA895E1ECFDE088E0CA
:1046C000DF011D928A95E9F781E08093C50D8EE1A7
:1046D0008093C60D82E38093C80DAEEABEE088E009
:1046E00090E021E08030920719F40E94926E03C09E
:1046F000182E0E94926E9E012B5E3F4F80E5D901DD
:104700001D928A95E9F78CE0A0E2B1E0FE0178966F
:10471000982F0D9001929A95E1F7ACE2B1E0FE017D
:10472000BC96982F0D9001929A95E1F7A8E3B1E01D
:10473000FE01E05CFF4F982F0D9001929A95E1F7F2
:10474000A4E4B1E0FE01EC5AFF4F0D9001928A956E
:10475000E1F7F901AEECBEE080E590E021E08030C9
:10476000920719F40E94926E03C0182E0E94926E56
:104770008CE0E5EDFDE011928A95E9F7A895CF521E
:10478000DF4F0FB6F894DEBF0FBECDBFDF91CF91E4
:104790001F910F91FF90EF90DF90CF90BF90AF905F
:1047A0000895EF92FF920F931F93CF93DF93CDB7AE
:1047B000DEB7E7970FB6F894DEBF0FBECDBF00E0BF
:1047C000102F1F5F612FCE0101960E942739202FE5
:1047D000332785E290E0289FA001299F500D389F44
:1047E000500D1124FA01E95CFB4F89819927982F1C
:1047F00088272A81820F911D938B828B8B818683E0
:10480000888580878C818583DA01AD5BBB4F888D7D
:104810008C93898D81878D819E81918F808F8F81EF
:10482000848F012F123260F280E699E00E94603797
:104830008EE699E00E94803781E299E00E94D439A7
:1048400083E399E00E94F439EDECFDE0A5ECBAE0D9
:1048500088E090E021E08030920719F40E94816E98
:1048600003C0182E0E94816E8091CD0D9091CE0DC7
:10487000892B19F48FEF8093CF0D8091D00D9091FB
:10488000D10D892B19F48FEF8093D20D00E016E043
:10489000BE01665E7F4F802F0E94C937802F992707
:1048A0009C0122953295307F3227207F3227F901F3
:1048B000E756F64F8A8D582F51708081482F4C7FD4
:1048C0008B8D8170982F990F842F852B892B808356
:1048D000F901E756F64F8C8D82838D8D87838E8DFF
:1048E00080878F8D8187D901AD55B64FFE01B09677
:1048F000812F01900D928A95E1F70F5F053040F20C
:10490000E1ECFDE0AEEABEE088E090E021E080303E
:10491000920719F40E94816E03C0182E0E94816EC6
:1049200000E074E143E050E0642F0F2EF5EDEF2E30
:10493000FDE0FF2EF02DFE01F596079FC00111242A
:10494000DC01A253B14F4115510551F081E04030D7
:10495000580719F40E94816E03C0162E0E94816EC2
:10496000202F3327C901880F991F280F391FF901FC
:10497000EE0DFF1D8DA980838FA98183F901E95276
:10498000F24F8EA9982F977080818078892B808331
:104990000F5F043080F2E7960FB6F894DEBF0FBECB
:1049A000CDBFDF91CF911F910F91FF90EF900895B0
:1049B000CF93DF93EC01862F0E942130833240F5A4
:1049C000282F332785E290E0289FA001299F500DD2
:1049D000389F500D1124FA01ED5BFB4F8F89982F02
:1049E0009F7780818078892B80839F8990788F77CB
:1049F000892B8083FA01E95CFB4F88819927982FE6
:104A000088272981820F911D938B828B8A818683CF
:104A1000DF91CF9108951F93CF93C0E01C2F909109
:104A20006E09892F8150803238F4892F0E94381303
:104A30008823B1F011E014C090916E09892F815242
:104A4000843138F4892F0E94025E882349F011E0F6
:104A500007C080916E090E94024A813009F4182F24
:104A600090918309892F8150803220F4892F0E94F0
:104A700038130EC090918309892F8152843120F41C
:104A8000892F0E94025E04C0809183090E94024A1D
:104A90008E3FF1F08130B9F48091EA09843020F43E
:104AA0008F5F8093EA0909C01092EA098091EB09AF
:104AB000882319F081508093EB098091EB098823BA
:104AC00059F4C1E009C0809184098093EB0904C0C6
:104AD000809184098093EB09113021F4812F0E9489
:104AE000C71E0CC0C13021F48C2F0E94E71E06C0E7
:104AF00080E00E94C71E80E00E94E71ECF911F91B8
:104B00000895FC018481982F986080EF82838785C7
:104B100086798787168A892F8F7D84838485882369
:104B20007CF48F77282F332786E990E0289FA00117
:104B3000299F500D389F500D11245687458763C01B
:104B400084858F77992796878587892B59F4918556
:104B50009F3F09F458C085E0989FC00111249387B6
:104B6000828751C084858F77282F3327C9018F71A1
:104B7000907096878587207630702034310541F11A
:104B8000213431053CF42115310541F02032310545
:104B900089F039C02036310549F135C02585368583
:104BA000C901880F991F880F991F820F931F96873D
:104BB000858729C08585968529E130E0829FA001FF
:104BC000839F500D929F500D1124568745871BC01F
:104BD0008585968526E930E0829FA001839F500D50
:104BE000929F500D1124568745870DC08585968567
:104BF00028EE33E0829FA001839F500D929F500DBD
:104C000011245687458783E0878308951F93CF93A8
:104C1000C0E015E2C19FC0011124FC01E95CFB4F1B
:104C20008785992783FD02C080FF03C0CF010E94C2
:104C30008125CF5FC23270F3CF911F9108959927DC
:104C40008C33910509F466C08D339105A4F4883343
:104C50009105A1F1893391051CF4C79721F1A7C0F3
:104C600089339105B1F18A33910509F43DC0CB97A1
:104C700009F445C09CC08034910509F477C08134A3
:104C8000910544F48E33910509F45AC0CF970CF086
:104C900062C04BC08134910509F473C08234910520
:104CA00009F47AC084C08091D70D8077803119F4DF
:104CB00081E090E0089580E090E008958091D70D24
:104CC0008077803219F481E090E0089580E090E0F0
:104CD00008958091D70D8077803319F481E090E0BA
:104CE000089580E090E008958091DA0D807780311A
:104CF00019F481E090E0089580E090E008958091BB
:104D0000DA0D8077803219F481E090E0089580E038
:104D100090E008958091DA0D8077803319F481E076
:104D200090E0089580E090E008958091DD0D807717
:104D3000803119F481E090E0089580E090E00895DA
:104D40008091DD0D8077803219F481E090E0089544
:104D500080E090E008958091DD0D8077803319F434
:104D600081E090E0089580E090E008958091E00D6A
:104D70008077803119F481E090E0089580E090E040
:104D800008958091E00D8077803219F481E090E001
:104D9000089580E090E008958091E00D8077803361
:104DA00019F481E090E0089580E090E0089580E0BB
:104DB00090E00895FF920F931F93CF93DF9310E03D
:104DC0000F2EFFE0FF2EF02D82E00E94A84A85E220
:104DD000189FC0011124EC01C95CDB4F8885882332
:104DE00061F48981803F09F017C18C8188608C83D0
:104DF0008F85867B8F87FA820FC12885822F81500D
:104E0000803208F045C08F85992783FD2FC080FD33
:104E10002DC0822F0E943813882341F089818F3062
:104E200009F0FAC0CE010E948125F6C08981803F39
:104E300009F0F2C089858F3F09F4EEC08A859B8511
:104E4000892B09F0E9C08C85882344F48D859E85E3
:104E5000009721F001979E878D87DEC08C81886046
:104E60008C838F85867B8F87FA82D6C088850E9447
:104E70003813882309F0D0C08981803F09F0CCC065
:104E80008C8188608C838F85867B8F87FA82C4C0F3
:104E90002885822F8152843108F045C08F8599275B
:104EA00083FD2FC080FD2DC0822F0E94025E8823CB
:104EB00041F089818F3009F0AFC0CE010E94812579
:104EC000ABC08981803F09F0A7C089858F3F09F475
:104ED000A3C08A859B85892B09F09EC08C85882379
:104EE00044F48D859E85009721F001979E878D87DC
:104EF00093C08C8188608C838F85867B8F87FA82B4
:104F00008BC088850E94025E882309F085C0898154
:104F1000803F09F081C08C8188608C838F85867B7F
:104F20008F87FA8279C000E08885853371F490918B
:104F3000B90D892F8350823020F0913011F09630D6
:104F400011F491E01DC090E01BC08885863351F4B8
:104F50008091B90D853011F0823011F491E010C0CC
:104F600090E00EC09885892F87538C3028F4892FC4
:104F70000E941F26982F04C088850E94024A982FFD
:104F80009E3FA9F08885803C21F49130A1F4092F3F
:104F900012C08D81813021F4913011F4092F0BC0A2
:104FA0008D81803141F4992331F401E004C088857A
:104FB0008F3F09F401E0002369F089818F3061F5AA
:104FC0008F85992783FD28C080FD26C0CE010E94D1
:104FD000812522C08981803F31F08F85992783FD0B
:104FE00002C080FF19C089858F3FB1F08A859B85FB
:104FF000892B91F48C85882344F48D859E850097B8
:1050000021F001979E878D8707C08C8188608C83F3
:105010008F85867B8F87FA8289818F3079F48F859F
:10502000992789709070892B49F48091110181171B
:1050300029F482E2809311011092E10D1F5F123278
:1050400008F4C2CEDF91CF911F910F91FF90089588
:1050500060933304623019F48FEF809357090895F9
:10506000CF93DF93EC0188818150823218F080E089
:1050700090E03BC088810E942130282F89819927A8
:105080008F30910521F0803F9105A1F02CC033278E
:1050900085E290E0289FA001299F500D389F500D78
:1050A0001124FA01E95CFB4F8FE081838785867FBD
:1050B000878719C0332785E290E0289FA001299FA8
:1050C000500D389F500D1124FA01E95CFB4F80EF21
:1050D00081838785867F8787168AFA01E55CFB4F87
:1050E00080818F7D808381E090E0DF91CF91089572
:1050F0006F927F928F929F92AF92BF92CF92DF92E8
:10510000EF92FF920F931F93CF93DF93CDB7DEB74C
:1051100021970FB6F894DEBF0FBECDBFBB24B98276
:105120009B2CAB2C8B2C1092590910925809B092E1
:105130005C09B0925E09B0925D090E9426058093D9
:105140005B0980913304882309F0A8C4B9828B2DB0
:10515000823208F03FC77724689471F80F2EF3E08D
:105160006F2EF02D82E00E94A84A9924998185E251
:10517000989FC00111240F2EF7E3CF2EF4E0DF2E0D
:10518000F02DC80ED91EF601858D9927807F90706D
:10519000803A910529F40F2EF1E4AF2EF02D18C0BE
:1051A000F601858D9927807F9070803B910529F4C9
:1051B0000F2EF2E4AF2EF02D0BC000E021E0AE0187
:1051C0004F5F5F4F6AE478E082E191E00E94233410
:1051D000F601118A108A248122FDC4C28081992798
:1051E0008130910509F460C18034910509F0C7C28E
:1051F000818199278F30910509F4D5C0803F9105B1
:1052000009F0BDC2822F837019F4878585FF26C0FF
:1052100089818A3039F48091CA0D882319F07092FF
:10522000CA0D13C089818B3039F48091BA0D88235F
:1052300019F07092BA0D09C089818C3031F48091D7
:10524000BE0D882311F07092BE0DF601858D41A12F
:105250006A2D8F700E940E42992473C0F6018485D6
:1052600088232CF085859685892B09F06AC0F60184
:10527000878580FD66C089818A30E1F48091CA0DFE
:105280008823C1F0823048F4858D41A16A2D8F704A
:105290000E9483419924939454C08091CA0D813017
:1052A00009F04FC06092CA0D1092C00D1092BF0D50
:1052B000992447C089818B30E1F48091BA0D88230D
:1052C000C1F0823050F4F601858D41A16A2D8F70B6
:1052D0000E9483419924939434C08091BA0D813007
:1052E00081F56092BA0D1092CC0D1092CB0D9924DD
:1052F00028C089818C30E1F48091BE0D8823C1F0F3
:10530000823050F4F601858D41A16A2D8F700E9484
:1053100083419924939415C08091BE0D813089F406
:105320006092BE0D1092BC0D1092BB0D992409C065
:10533000F601858D41A16A2D8F700E9483419924C9
:105340009394F601848183FF1AC2877F84838281CC
:105350008F3009F014C289818A3039F48091CA0DE6
:10536000882319F07092CA0D13C089818B3039F4EB
:105370008091BA0D882319F07092BA0D09C0898105
:105380008C3031F48091BE0D882311F07092BE0DE7
:105390008FE0F6018183858D41A16A2D8F700E9477
:1053A0000E429924ECC1F601848183FFE8C1877F16
:1053B00084838281803F09F0E2C1818384858823D0
:1053C0002CF085859685892B09F0D9C1F601848159
:1053D000837009F0D4C189818A30E1F48091CA0DCB
:1053E0008823C1F0823048F4858D41A16A2D8F70E9
:1053F0000E94834199249394C2C18091CA0D823046
:1054000009F0BDC16092CA0D1092C00D1092BF0D7F
:105410009924B5C189818B30E9F48091BA0D882334
:10542000C9F0823050F4F601858D41A16A2D8F704C
:105430000E94834199249394A2C18091BA0D823035
:1054400009F09DC16092BA0D1092CC0D1092CB0D57
:10545000992495C189818C30E9F48091BE0D88230F
:10546000C9F0823050F4F601858D41A16A2D8F700C
:105470000E9483419924939482C18091BE0D823011
:1054800009F07DC16092BE0D1092BC0D1092BB0D53
:10549000992475C1F601858D41A16A2D8F700E94F6
:1054A0008341992493946BC1F601818199278F30B0
:1054B000910509F4D8C0803F910509F060C184814D
:1054C000837019F4878585FF26C089818A3039F475
:1054D0008091CA0D882319F07092CA0D13C089817A
:1054E0008B3039F48091BA0D882319F07092BA0D7F
:1054F00009C089818C3031F48091BE0D882311F070
:105500007092BE0DF601858D41A16A2D8F700E94AB
:105510000E42992476C0F601848588232CF0858577
:105520009685892B09F06DC0F6018785992780FD46
:1055300068C083FD66C089818A30E1F48091CA0D1C
:105540008823C1F0823048F4858D41A16A2D8F7087
:105550000E9483419924939454C08091CA0D823053
:1055600009F04FC06092CA0D1092C00D1092BF0D8D
:10557000992447C089818B30E1F48091BA0D88234A
:10558000C1F0823050F4F601858D41A16A2D8F70F3
:105590000E9483419924939434C08091BA0D823043
:1055A00081F56092BA0D1092CC0D1092CB0D99241A
:1055B00028C089818C30E1F48091BE0D8823C1F030
:1055C000823050F4F601858D41A16A2D8F700E94C2
:1055D00083419924939415C08091BE0D823089F443
:1055E0006092BE0D1092BC0D1092BB0D992409C0A3
:1055F000F601858D41A16A2D8F700E948341992407
:105600009394F601848183FFBAC0877F848382816B
:105610008F3009F0B4C089818A3039F48091CA0D85
:10562000882319F07092CA0D13C089818B3039F428
:105630008091BA0D882319F07092BA0D09C0898142
:105640008C3031F48091BE0D882311F07092BE0D24
:105650008FE0F6018183858D41A16A2D8F700E94B4
:105660000E4299248CC0F601848183FF88C0877F15
:1056700084838281803F09F082C08183848588236E
:105680002CF085859685892B09F079C0F6018481F7
:10569000837009F074C089818A30E1F48091CA0D69
:1056A0008823C1F0823048F4858D41A16A2D8F7026
:1056B0000E9483419924939462C08091CA0D8230E4
:1056C00009F05DC06092CA0D1092C00D1092BF0D1E
:1056D000992455C089818B30E1F48091BA0D8823DB
:1056E000C1F0823050F4F601858D41A16A2D8F7092
:1056F0000E9483419924939442C08091BA0D8230D4
:10570000F1F56092BA0D1092CC0D1092CB0D992448
:1057100036C089818C30E1F48091BE0D8823C1F0C0
:10572000823050F4F601858D41A16A2D8F700E9460
:1057300083419924939423C08091BE0D8230F9F463
:105740006092BE0D1092BC0D1092BB0D992417C033
:10575000F601858D41A16A2D8F700E9483419924A5
:1057600093940DC0F601818199278F30910531F016
:10577000803F910521F49924939401C09924F60166
:105780008181803F09F058C082A18F3F09F454C045
:105790000E94F1037C0100271127F601F4A2E3A285
:1057A00089819927FC01EF5DF64F80819927AA270F
:1057B000BB278E159F05A007B10724F0EE24FF2418
:1057C00087010AC089819927FC01EF5DF64F80812E
:1057D000E81AF10801091109F3E0EF16F1040105D7
:1057E0001105CCF089819927880F991FFC01ED5C88
:1057F000F64F808191819C0144275527C801B7014C
:105800000E94B36D20EE31E040E050E00E94276E30
:1058100079018A0103C0EE24FF248701F601F18A91
:10582000E08A80915809909159098E0D9F1D90939F
:1058300059098093580903C0F601118A108A9920EA
:1058400039F4F601828D938D892B11F0138E128E0F
:10585000F60187859927AC014870507083FD70C0B0
:10586000208931898289938982179307E0F5828D97
:10587000938D892B11F0538F428FF601848185FF20
:1058800026C084899589892B09F05AC0878588604C
:10589000878780915C098F5F80935C09808181306C
:1058A00071F4858D41A16A2D8F700E940E4299245A
:1058B000898180931101F60186818093E9098981AC
:1058C000F601608971898F5F0E94983639C0F601B0
:1058D000848180628483968185E0989FC001112431
:1058E000958B848B2DC0F60184818F7D8483208DE0
:1058F000318D2115310521F19920A1F080899189FF
:105900008217930778F4828D938D892BC9F487854C
:1059100086FD16C0948D85E0989FC0011124938F59
:10592000828F0EC0F601828D938D892B49F02089DC
:105930003189808D918D8217930710F4138E128E0A
:105940008981803129F48091CF0D883008F489C095
:105950008981813129F48091D20D883008F481C089
:10596000F601868D9927807F9070803A910529F401
:105970000F2EF1E48F2EF02D18C0F601868D992799
:10598000807F9070803B910529F40F2EF2E48F2EDA
:10599000F02D0BC000E021E0AE014F5F5F4F69E0EA
:1059A0007AE082E191E00E942334F601868D41A1E4
:1059B000682D8F700E94A742282FF6018181803FB9
:1059C00009F04FC08785992783FD4BC080FD49C0F2
:1059D00090915B0980911001891708F042C0F1E0B5
:1059E0009F16E9F52223D9F5F60187818823C9F5A9
:1059F0008485882324F085859685892B91F5F60189
:105A00008181803F71F587898F3F11F08F5F878B90
:105A1000F6018789833028F18689982F9F5F968BBE
:105A20008091B50D8F77891750F0858D41A16A2D32
:105A30008F700E940E42F601178A678212C0F6012B
:105A4000858D41A16A2D8F700E940E42F6018785D7
:105A50008160878789818F5F0E94D03602C0F601FE
:105A6000178AF601878580FF05C080915E098F5FE8
:105A700080935E09F601878583FF05C080915C09EC
:105A80008F5F80935C09F60187858111B3948981CA
:105A90008F5F8983823208F465CB9CC28091330486
:105AA000813009F0CAC119828981482F823208F0F9
:105AB00091C2242F332785E290E0289FB001299FCF
:105AC000700D389F700D1124FB01E95CFB4F878539
:105AD0008F7D878785E2489FC00111240F2EF7E351
:105AE000CF2EF4E0DF2EF02DC80ED91EF601858DE5
:105AF0009927807F9070803A910529F40F2EF1E468
:105B0000AF2EF02D0CC0F601858D9927807F907007
:105B1000803B910521F40F2EF2E4AF2EF02DF6011B
:105B2000848182FD4FC0808199278130910569F180
:105B30008034910509F046C0818199278F30910505
:105B400061F0803F9105F1F5858D41A16A2D8F703F
:105B50000E9483419924939435C08981282F33274B
:105B600085E290E0289FA001299F500D389F500D9D
:105B70001124FA01E95CFB4F858DF60141A16A2DE4
:105B80008F700E940E4299241DC0F60181819927D1
:105B90008F30910561F0803F9105A1F4858D41A181
:105BA0006A2D8F700E948341992493940BC0F60153
:105BB000858D41A16A2D8F700E940E428FE0F60103
:105BC00081839924F6018181803F09F057C082A129
:105BD0008F3F09F453C00E94F1037C010027112775
:105BE000F601F4A2E3A289819927FC01EF5DF64F4B
:105BF00080819927AA27BB278E159F05A007B1078B
:105C000024F0EE24FF2487010AC089819927FC0132
:105C1000EF5DF64F8081E81AF10801091109F3E000
:105C2000EF16F10401051105CCF089819927880F41
:105C3000991FFC01ED5CF64F808191819C01442706
:105C40005527C801B7010E94B36D20EE31E040E056
:105C500050E00E94276E79018A0103C0EE24FF24E0
:105C60008701F601F18AE08A8091580990915909DB
:105C70008E0D9F1D9093590980935809F601208934
:105C80003189828993898217930788F5848185FFFA
:105C900022C084899589892B81F5878588608787CB
:105CA00080915C098F5F80935C098081813059F419
:105CB000858D41A16A2D8F700E940E4299248FE03C
:105CC000F601818382838981F601608971898F5F02
:105CD0000E94983612C0F601848180628483968186
:105CE00085E0989FC0011124958B848B06C0F60136
:105CF00084818F7D8483158A148A8981803129F477
:105D00008091CF0D883008F47AC08981813129F4DF
:105D10008091D20D883008F472C0F601868D9927E3
:105D2000807F9070803A910529F40F2EF1E48F2E38
:105D3000F02D0CC0F601868D9927807F9070803BF6
:105D4000910521F40F2EF2E48F2EF02DF601868DB1
:105D500041A1682D8F700E94A742282FF6018785E8
:105D6000992783FD4CC080FD4AC090915B098091CA
:105D70001001891708F043C0F1E09F16F1F52223C6
:105D8000E1F5F60187818823D1F58485882324F005
:105D900085859685892B99F5F6018181803F79F576
:105DA00087898F3F11F08F5F878BF601878983305A
:105DB00030F18689982F9F5F968B8091B50D8F77F4
:105DC000891758F0858D41A16A2D8F700E940E426F
:105DD000F601178A83E0878312C0F601858D41A101
:105DE0006A2D8F700E940E42F60187858160878739
:105DF00089818F5F0E94D03602C0F601178AF601B2
:105E0000878580FF05C080915E098F5F80935E0962
:105E1000F601878583FF05C080915C098F5F8093C1
:105E20005C09F60187858111B39489818F5F89832D
:105E3000482F823208F43DCECDC0809133048230A9
:105E400009F0C8C019828981982F823208F0C2C037
:105E500085E2989FC00111240F2EF7E3CF2EF4E0C6
:105E6000DF2EF02DC80ED91EF601858D9927807F73
:105E70009070803A910529F40F2EF1E4AF2EF02DA9
:105E80000CC0F601858D9927807F9070803B91052D
:105E900021F40F2EF2E4AF2EF02D40915709442348
:105EA000D1F0898199279C012F5F3F4F842F99273B
:105EB0002817390741F4F601858D41A16A2D8F70AD
:105EC0000E9483410FC0F601858D41A16A2D8F701C
:105ED0000E940E4207C0F601858D41A16A2D8F7088
:105EE0000E948341F60182A18F3F09F46CC00E9499
:105EF000F1037C0100271127F601F4A2E3A28091AF
:105F0000320480FF1CC089819927FC01EF5DF64FA8
:105F100080819927AA27BB278E159F05A007B10767
:105F200024F0EE24FF2487010AC089819927FC010F
:105F3000EF5DF64F8081E81AF10801091109F3E0DD
:105F4000EF16F1040105110574F18091320481FF0F
:105F500019C089819927880F991FFC01ED5CF64FC4
:105F6000808191819C0144275527C801B7010E9477
:105F7000B36D20EE31E040E050E00E94276E7901E1
:105F80008A0114C0C801B70128EB31E040E050E0BD
:105F90000E94B36D20EE31E040E050E00E94276E99
:105FA00079018A0103C0EE24FF248701F601F18AFA
:105FB000E08A80915809909159098E0D9F1D909308
:105FC00059098093580989818F5F8983982F82327C
:105FD00008F43ECFBB2031F4B0925D09B0925E0967
:105FE000B0925F090E941A05982F80935A098091F8
:105FF0003404891710F49093340420915809309197
:10600000590980913504909136048217930720F442
:10601000309336042093350421960FB6F894DEBFF2
:106020000FBECDBFDF91CF911F910F91FF90EF90E9
:10603000DF90CF90BF90AF909F908F907F906F90A8
:106040000895815099270895CF93DF93EC01862F0F
:106050000E942130833278F4282F332785E290E0A4
:10606000289FA001299F500D389F500D1124FA013F
:10607000E95CFB4FC683DF91CF910895EF92FF92C9
:106080001F93CF937C01C0E080EC0E94024A8111F3
:10609000C1E081EC0E94024A8111C26082EC0E9440
:1060A000024A8111C46081ED0E94024A8111C860D8
:1060B00084EC0E94024A8111C06185EC0E94024A70
:1060C0008111C06286EC0E94024A8111C06487EC93
:1060D0000E94024A8111C06810E083EC0E94024ACB
:1060E000811111E082ED0E94024A8111126083ED5C
:1060F0000E94024A81111460F701C0831183C0E03D
:1061000081E00E9438138111C1E082E00E943813BF
:106110008111C26083E00E9438138111C46084E061
:106120000E9438138111C86085E00E9438138111E4
:10613000C06186E00E9438138111C06287E00E942E
:1061400038138111C06488E00E9438138111C0683F
:10615000F701C283C0E089E00E9438138111C1E0D9
:106160008AE00E9438138111C2608BE00E943813CC
:106170008111C4608CE00E9438138111C8608DE0E9
:106180000E9438138111C0618EE00E943813811182
:10619000C0628FE00E9438138111C06480E10E94C8
:1061A00038138111C068F701C383C0E081E10E9408
:1061B00038138111C1E082E10E9438138111C2605D
:1061C00083E10E9438138111C46084E10E94381376
:1061D0008111C86085E10E9438138111C06186E198
:1061E0000E9438138111C06287E10E943813811127
:1061F000C06488E10E9438138111C068F701C4832C
:10620000C0E089E10E9438138111C1E08AE10E9457
:1062100038138111C2608BE10E9438138111C46070
:106220008CE10E9438138111C8608DE10E943813FF
:106230008111C0618EE10E9438138111C0628FE12B
:106240000E9438138111C06480E20E9438138111CA
:10625000C068F701C583CF911F91FF90EF9008951B
:106260001F93CF93DF93182FEB010E942130482F0B
:10627000833218F080E090E0A6C0282F332785E213
:1062800090E0289FB001299F700D389F700D112458
:10629000FB01E55CFB4F808182FD52C0DB01A95C04
:1062A000BB4FFD018181803FD1F5FB01ED5BFB4FD1
:1062B000808188232CF0FD0185859685892B61F5E9
:1062C000242F332785E290E0289FB001299F700D8D
:1062D000389F700D1124FB01E55CFB4F808181FF2D
:1062E00004C0809133048823B9F0242F332785E23A
:1062F00090E0289FF001299FF00D389FF00D1124A8
:106300009F01E55CFB4F808180FD06C0F901E95CDF
:10631000FB4F878585FF03C08FE088833AC0242F19
:10632000332785E290E0289FB001299F700D389FA8
:10633000700D1124FB01E95CFB4F8181888329C02A
:1063400030E0232F822F992782959295907F98276E
:10635000807F9827DC01A756B64FFD0181818130EF
:1063600099F490E06FE050EFFD01E90FF11D828597
:10637000841739F431E08C9182FF02C0688301C038
:1063800058839F5F963080F32F5F253010F43323BE
:10639000C9F2242F332785E290E0289FA001299F8E
:1063A000500D389F500D1124FA01E95CFB4F878591
:1063B0008983808991899C838B83812F0E941B37DD
:1063C0008A8381E090E0DF91CF911F9108950E9430
:1063D0002130833218F080E090E00895282F332791
:1063E00085E290E0289FA001299F500D389F500D15
:1063F0001124FA01E95CFB4F8181803F59F4FA01D5
:10640000E55CFB4F208121FD05C020FD03C081E03C
:1064100090E0089580E090E008950E94213083325A
:1064200018F080E090E00895282F332785E290E06F
:10643000289FA001299F500D389F500D1124FA016B
:10644000E95CFB4F2785283011F0213019F481E0F9
:1064500090E0089580E090E00895FC018091580953
:10646000909159099183808380915A098283809108
:106470005B09838380915C09848380915D098583B6
:1064800080915E09868380915F0987830895982FA4
:106490008150823238F485E2989FC00111248E5ECB
:1064A0009B4F089580E090E008959EEF81B189238D
:1064B00081B982B1892382B917B818B891EF8AB12E
:1064C00089238AB98BB189238BB981E080938000BD
:1064D0008DE0809381001092880010928A000895C8
:1064E0000F930E942130282F833168F000E0202F85
:1064F00040E050E066EA7CE082E191E00E942334D3
:1065000080E090E007C081E299E0FC01E20FF11D1C
:10651000808199270F9108950F930E942130833134
:1065200068F000E0202F40E050E064EB7CE082E186
:1065300091E00E94233480E692E212C09927880FEE
:10654000991FFC01ED5CF64F2081318184E190E0E0
:10655000289FA001299F500D389F500D1124CA017A
:106560000F9108950F93CF93DF93EB010E94213099
:10657000833158F000E0202F40E050E063EC7CE0F5
:1065800082E191E00E94233412C0992723E339E08D
:10659000880F991FFC01E20FF31FCE0164E170E048
:1065A0000E94DE6D71836083C9010E94E439DF912E
:1065B000CF910F9108950E942130833118F080E02F
:1065C00090E00895282F332785E290E0289FA001CE
:1065D000299F500D389F500D1124FA01E95CFB4FA3
:1065E0008089918908950E942130833118F080E0DC
:1065F00090E00895282F332785E290E0289FA0019E
:10660000299F500D389F500D1124FA01E95CFB4F72
:1066100083A194A10895809332046093570908954B
:106620001F93CF93C0E015E2C19FC0011124FC016C
:10663000E95CFB4F82A18F3F41F00E94F1032C2FB8
:106640003327F901EF5DF64F8083CF5FC23160F3EE
:1066500081E299E00E94C439CF911F910895CF93B0
:1066600080913304833059F083E080933304C0E099
:1066700061E08C2F0E944B1ECF5FC232C8F3CF91D6
:106680000895CF93DF93CDB7DEB723970FB6F89475
:10669000DEBF0FBECDBFFE013196A0EEB0E083E0BD
:1066A00090E021E08030920719F40E94816E03C0CF
:1066B000182E0E94816E43E050E060E571E0CE014B
:1066C00001960E94AA5A882391F00E948133E0E546
:1066D000F1E0A0EEB0E083E090E021E080309207AE
:1066E00019F40E94926E03C0182E0E94926E279891
:1066F00023960FB6F894DEBF0FBECDBFDF91CF91CA
:106700000895CF93DF93CDB7DEB76E970FB6F894A9
:10671000DEBF0FBECDBF84E1FE013B9611928A958C
:10672000E9F740E064E124E130E0522FFE013B96BE
:10673000469FC0011124DC01AC51BF4F211531052A
:1067400051F081E02030380719F40E94926E03C0A6
:10675000152E0E94926EA8954F5F483038F319822B
:10676000FE013196A3EEB0E081E090E021E08030C0
:10677000920719F40E94926E03C0182E0E94926E26
:106780006E960FB6F894DEBF0FBECDBFDF91CF91EE
:106790000895CF93DF93CDB7DEB721970FB6F89466
:1067A000DEBF0FBECDBFFE013196A3EEB0E081E0AB
:1067B00090E021E08030920719F40E94816E03C0BE
:1067C000182E0E94816E8981893010F088E08983BB
:1067D0008981992721960FB6F894DEBF0FBECDBFF1
:1067E000DF91CF910895CF93DF93CDB7DEB7649754
:1067F0000FB6F894DEBF0FBECDBF9B01FE013196F0
:1068000094E1899FD0011124A053BF4F84E190E00F
:1068100041E08030940719F40E94816E03C0182E65
:106820000E94816E84E1FE013196D90101900D92A2
:106830008A95E1F764960FB6F894DEBF0FBECDBF20
:10684000DF91CF9108956F927F928F929F92AF9236
:10685000BF92CF92DF92EF92FF920F931F93CF934D
:10686000DF93CDB7DEB7A9970FB6F894DEBF0FBEA2
:10687000CDBF6C015B013A01022FFE01B996A3EE78
:10688000B0E081E090E021E08030920719F40E94AE
:10689000816E03C0182E0E94816E89A5883008F091
:1068A000D4C09924FE01759684E1DF011D928A957A
:1068B000E9F7B601CF010E94AC6D192D89A5981694
:1068C00008F05EC00F2EF4E18F2EF02D0F2EF4E1B4
:1068D000EF2EFF24F02DFE013196189DC0011124EA
:1068E000DC01AC51BF4FE114F10459F020E0E21695
:1068F00021E0F20619F40E94816E03C01E2C0E9452
:10690000816E8D859E858A159B0599F546E050E040
:10691000B601CE0101960E94AA5A882351F5992406
:1069200093948F858A3008F090C0890D8F87053049
:1069300008F004E0198A1A8A1B8A1C8A802F99277A
:10694000AC01B301CE0141960E94956DFE013196D6
:10695000189DD0011124AC51BF4F84E190E021E09B
:106960008030920719F40E94926E03C0182E0E9484
:10697000926E1F5F89A5181718F4992009F4ABCF00
:10698000992009F052C089A5883008F04EC08F5F69
:1069900089A78CE0FE01319611928A95E9F7F601FC
:1069A00001900020E9F731972E2F2C192C3008F098
:1069B0002BE010E0121780F4AE014F5F5F4F812F84
:1069C0009927DC01A40FB51FF601E80FF91F80819C
:1069D0008C931F5F121798F3BE86AD8681E08F8778
:1069E000053008F004E0088B198A1A8A1B8A1C8A71
:1069F000802F9927AC01B301CE0141960E94956D7D
:106A0000FE01319699A584E1989FD0011124A053ED
:106A1000BF4F84E190E021E08030920719F40E949A
:106A2000926E03C0182E0E94926EFE01B996A3EEDC
:106A3000B0E081E090E021E08030920719F40E94FC
:106A4000926E03C0182E0E94926EA9960FB6F8940B
:106A5000DEBF0FBECDBFDF91CF911F910F91FF9091
:106A6000EF90DF90CF90BF90AF909F908F907F90EE
:106A70006F900895089582E1E2EEFDE011928A950B
:106A8000E9F780E1E4EFFDE011928A95E9F7E6E1AC
:106A9000FEE0A8E9B0E082E190E021E080309207DA
:106AA00019F40E94816E03C0182E0E94816EE8E2E4
:106AB000FEE0AAEAB0E082E190E021E080309207B7
:106AC00019F40E94816E03C0182E0E94816EEAE3C1
:106AD000FEE0ACEBB0E080E190E021E08030920796
:106AE00019F40E94816E03C0182E0E94816EE4E0AA
:106AF000FEE0ADECB0E082E190E021E08030920772
:106B000019F40E94816E03C0182E0E94816EEFEE70
:106B1000F9E0A5E9B0E081E090E021E08030920763
:106B200019F40E94816E03C0182E0E94816EE0EF5E
:106B3000F9E0A6E9B0E082E090E021E08030920741
:106B400019F40E94816E0895182E0E94816E089596
:106B5000CF93DF93CDB7DEB762970FB6F894DEBF61
:106B60000FBECDBFFE01319682E1DF011D928A95F5
:106B7000E9F7A8E9B0E082E190E021E080309207F7
:106B800019F40E94926E03C0182E0E94926EA8956E
:106B9000FE013196AAEAB0E082E190E021E0803087
:106BA000920719F40E94926E03C0182E0E94926EF2
:106BB000FE013196ACEBB0E080E190E021E0803066
:106BC000920719F40E94926E03C0182E0E94926ED2
:106BD000FE013196ADECB0E082E190E021E0803042
:106BE000920719F40E94926E03C0182E0E94926EB2
:106BF000A8950E943B3562960FB6F894DEBF0FBE93
:106C0000CDBFDF91CF9108950E940C1F982F8091E6
:106C1000EF09891790F49093EF09EFEEF9E0A5E9F9
:106C2000B0E081E090E021E08030920719F40E940A
:106C3000926E03C0182E0E94926E0E94071F9C0144
:106C40008091F0099091F10982179307A0F4309395
:106C5000F1092093F009E0EFF9E0A6E9B0E082E065
:106C600090E021E08030920719F40E94926E08951E
:106C7000182E0E94926E08958091EF099927089529
:106C80008091F0099091F109089590E042EE5DE065
:106C9000292F3327F901E40FF51F808180FF17C0EA
:106CA0008E7F8083D901A856BF4FF901EA5EF14F6C
:106CB0008081082E0E94866ED901A655BF4FF9012A
:106CC000E85DF14F8081082E0E94866E0895E92FBD
:106CD000FF27DF01A40FB51F8C9181FF0CC08D7FB2
:106CE0008C93DF01A353BF4FEC5FF14F8081082EDF
:106CF0000E94866E08959F5F923150F290E024EFDB
:106D00003DE0E92FFF27DF01A20FB31F8C918130F7
:106D100059F41C92DF01A454BF4FE65CF14F80810F
:106D2000082E0E94866E08959F5F903150F308955B
:106D3000282F2150223198F586E19EE0FC01E20FD8
:106D4000F11D3081832F9927929582958F70892725
:106D50009F7089278F30910514F5482F4F5F942F2E
:106D60009295907F832F8F70890F8083CB018370E2
:106D70009070892B11F041E001C040E03327F90108
:106D8000E85DF14FCB019695879596958795840F91
:106D90008083F901EE51F24F8081816080830895F4
:106DA000E82FE150E231C0F4FF27DF01AA5EB14FC6
:106DB0002C91822F99278F7090700F971CF5822F3E
:106DC0008F708F5F922F907F890F8C93EE51F24FCF
:106DD00080818160808308958351803198F4E82F09
:106DE000FF27DF01A65CB14F2C91822F99278F706E
:106DF00090700F973CF4822F8F5F8C93EC50F24F82
:106E000081E08083089581508231A0F4E82FFF272C
:106E1000DF01AC5FB14F2C91822F99278F7090705A
:106E20000F9744F4822F8F5F8C93EE51F24F808145
:106E3000826080830895E82FE150E23188F42E2F9C
:106E40003327F901EA5EF14F8081882331F4F9019B
:106E5000EC5FF14F8081882391F081E090E008950C
:106E6000282F2351203158F48AE39EE0FC01E20FE1
:106E7000F11D8081882319F081E090E0089580E081
:106E800090E00895CF93DF93EC01FC0120E931E01D
:106E90008EE090E041E08030940721F4D9010E9417
:106EA000926E04C0D901182E0E94926ECE010296F5
:106EB000AC01698188810E94101FDF91CF910895F4
:106EC000FC01A0E9B1E08EE090E021E08030920783
:106ED00019F40E94816E0895182E0E94816E089503
:106EE000FC01AEE9B1E08BE290E021E08030920756
:106EF00019F40E94926E0895182E0E94926E0895C1
:106F0000FC01AEE9B1E08BE290E021E08030920735
:106F100019F40E94816E0895182E0E94816E0895C2
:106F20000F93CF93DF93CDB7DEB721970FB6F894C9
:106F3000DEBF0FBECDBF8983853060F000E021E069
:106F4000AE014F5F5F4F6DE370E084E591E00E941A
:106F5000233415C089819BE1899FC0011124FB0165
:106F6000DC01A95DB14F8BE190E021E08030920718
:106F700019F40E94926E03C0182E0E94926E219600
:106F80000FB6F894DEBF0FBECDBFDF91CF910F914A
:106F900008950F93CF93DF93CDB7DEB721970FB648
:106FA000F894DEBF0FBECDBF8983853060F000E06E
:106FB00021E0AE014F5F5F4F6AE470E084E591E04D
:106FC0000E94233415C089819BE1899FC00111244F
:106FD000FB01DC01A95DB14F8BE190E021E0803045
:106FE000920719F40E94816E03C0182E0E94816ED0
:106FF00021960FB6F894DEBF0FBECDBFDF91CF91C3
:107000000F9108950F93CF93DF93CDB7DEB72197FC
:107010000FB6F894DEBF0FBECDBF8983803260F01B
:1070200000E021E0AE014F5F5F4F66E570E084E570
:1070300091E00E94233414C0FB0199818CE2989F57
:10704000D0011124AD54BD4F8CE290E021E080309E
:10705000920719F40E94926E03C0182E0E94926E3D
:1070600021960FB6F894DEBF0FBECDBFDF91CF9152
:107070000F9108950F93CF93DF93CDB7DEB721978C
:107080000FB6F894DEBF0FBECDBF8983803260F0AB
:1070900000E021E0AE014F5F5F4F60E670E084E505
:1070A00091E00E94233414C0FB0199818CE2989FE7
:1070B000D0011124AD54BD4F8CE290E021E080302E
:1070C000920719F40E94816E03C0182E0E94816EEF
:1070D00021960FB6F894DEBF0FBECDBFDF91CF91E2
:1070E0000F9108950F93CF93DF93CDB7DEB721971C
:1070F0000FB6F894DEBF0FBECDBF8983843160F038
:1071000000E021E0AE014F5F5F4F6AE670E084E58A
:1071100091E00E94233414C0FB01998188E1989F7B
:10712000D0011124AB5CB74F88E190E021E08030C2
:10713000920719F40E94926E03C0182E0E94926E5C
:1071400021960FB6F894DEBF0FBECDBFDF91CF9171
:107150000F9108950F93CF93DF93CDB7DEB72197AB
:107160000FB6F894DEBF0FBECDBF8983843160F0C7
:1071700000E021E0AE014F5F5F4F64E770E084E51F
:1071800091E00E94233414C0FB01998188E1989F0B
:10719000D0011124AB5CB74F88E190E021E0803052
:1071A000920719F40E94816E03C0182E0E94816E0E
:1071B00021960FB6F894DEBF0FBECDBFDF91CF9101
:1071C0000F910895CF93DF93CDB7DEB769970FB6D0
:1071D000F894DEBF0FBECDBFFC01862F81508232F6
:1071E00018F080E090E02AC061508081898381811D
:1071F0008A8382818B8383818C8387818887878937
:10720000888F808D898F848195819E838D838681EF
:107210008F83DF0118968FE0FE0139960D90019261
:107220008A95E1F789E1689FC00111248B52954F3F
:10723000BC01CE0101960E94B339992769960FB619
:10724000F894DEBF0FBECDBFDF91CF9108950F93AD
:107250001F93CF93DF93CDB7DEB769970FB6F8943E
:10726000DEBF0FBECDBF8C01962F91509232B0F58C
:1072700089E1989FC00111249E012F5F3F4FDC01DF
:10728000AB52B54F89E190E041E08030940721F4A2
:10729000F9010E94816E04C0F901182E0E94816ECE
:1072A0008981F80180838A8181838B8182838C81AB
:1072B000838388858783888D878B898D808F8D8157
:1072C0009E81958384838F818683D80118968FE071
:1072D000FE01399601900D928A95E1F769960FB6F5
:1072E000F894DEBF0FBECDBFDF91CF911F910F91FC
:1072F000089581508B30C8F4FB01A82FBB27CD0126
:1073000082959295907F9827807F9827DC01AB5ECD
:10731000B54F80E190E021E08030920719F40E949F
:10732000926E0895182E0E94926E089581508B30AF
:10733000C8F4FB01A82FBB27CD0182959295907FC1
:107340009827807F9827DC01AB5EB54F80E190E005
:1073500021E08030920719F40E94816E0895182E62
:107360000E94816E0895FC01DB0189E190E021E03B
:107370008030920719F40E94926E03C0182E0E946A
:10738000926E81E090E00895FC01A0E1B0E082E11E
:1073900090E021E08030920719F40E94926E0895E7
:1073A000182E0E94926E0895FC01A0E1B0E082E1E7
:1073B00090E021E08030920719F40E94816E0895D8
:1073C000182E0E94816E0895FC01A0E3B0E084E2D3
:1073D00090E021E08030920719F40E94926E0895A7
:1073E000182E0E94926E0895FC01A0E3B0E084E2A2
:1073F00090E021E08030920719F40E94816E089598
:10740000182E0E94816E0895FC01A9ECB1E088E17C
:1074100090E021E08030920719F40E94926E089566
:10742000182E0E94926E0895FC01A9ECB1E088E14B
:1074300090E021E08030920719F40E94816E089557
:10744000182E0E94816E08950F93FC01808188237D
:1074500019F481EE91E016C08081813019F487E241
:1074600092E010C08081823019F48DE692E00AC06B
:1074700000E021E0AF016FE371E084E591E00E945C
:1074800023340DC0DC0186E490E021E080309207D7
:1074900019F40E94926E03C0182E0E94926E0F91F2
:1074A00008950F93CF93DF93CDB7DEB721970FB633
:1074B000F894DEBF0FBECDBF8983882319F481EE17
:1074C00091E018C08981813019F487E292E012C0FE
:1074D0008981823019F48DE692E00CC000E021E051
:1074E000AE014F5F5F4F68E571E084E591E00E9477
:1074F00023340EC0FB01DC0186E490E021E0803003
:10750000920719F40E94816E03C0182E0E94816EAA
:1075100021960FB6F894DEBF0FBECDBFDF91CF919D
:107520000F910895CF93DF93CDB7DEB760970FB675
:10753000F894DEBF0FBECDBFFE013196A0E0B0E0F3
:1075400080E190E021E08030920719F40E94816E82
:1075500003C0182E0E94816E8B858F3119F48FE144
:1075600090E008C08B85803219F480E290E002C080
:107570008FE190E060960FB6F894DEBF0FBECDBFEE
:10758000DF91CF9108950F931F93CF93DF93CDB7E2
:10759000DEB76E970FB6F894DEBF0FBECDBFFE010B
:1075A0003196A0E0B0E084E090E021E080309207E6
:1075B00019F40E94816E03C0182E0E94816E44E06F
:1075C00050E068E671E0CE0101960E94AA5A882335
:1075D00009F44DC08E010F5F1F4F8EE1D8011D923F
:1075E0008A95E9F785E0E8E6F1E0D80101900D928F
:1075F0008A95E1F71D821E821F82188619861A86D7
:107600001B860E944D22F801A0E0B0E080E190E0EE
:1076100021E08030920719F40E94926E03C0182E68
:107620000E94926EFE013196A0E0B0E084E090E00E
:1076300021E08030920719F40E94926E03C0182E48
:107640000E94926EFE01319684E1DF011D928A95BF
:10765000E9F7AEE1BFE084E190E021E080309207FD
:1076600019F40E94926E03C0182E0E94926EFE01C1
:107670003196A0E8B1E08AE090E021E08030920706
:1076800019F40E94816E03C0182E0E94816E4AE098
:1076900050E06FE871E0CE0101960E94AA5A88235B
:1076A000D1F10E946D220E94CB120E947D5C0E944B
:1076B00032060E943511AE014F5F5F4F8EE1DA0155
:1076C0001D928A95E9F789E02DE631E0FA01D901AA
:1076D0000D9001928A95E1F7FA01A0E7B0E080E110
:1076E00090E021E08030920719F40E94926E03C06E
:1076F000182E0E94926EEFE8F1E0A0E8B1E08AE077
:1077000090E021E08030920719F40E94926E03C04D
:10771000182E0E94926EFE013196A0EEB0E083E03A
:1077200090E021E08030920719F40E94816E03C03E
:10773000182E0E94816E43E050E066E771E0CE01B2
:1077400001960E94AA5A882391F00E948133E6E7AD
:10775000F1E0A0EEB0E083E090E021E0803092071D
:1077600019F40E94926E03C0182E0E94926EFE01C0
:107770003196A0E9B0E085E090E021E0803092070A
:1077800019F40E94816E03C0182E0E94816E45E09C
:1077900050E06AE771E0CE0101960E94AA5A882360
:1077A00009F475C0FE0131968EE1DF011D928A95C4
:1077B000E9F7ACECB0E081E090E021E080309207A6
:1077C00019F40E94926E03C0182E0E94926EFE0160
:1077D0003196A5E9B0E081E090E021E080309207A9
:1077E00019F40E94926E03C0182E0E94926EFE0140
:1077F0003196A6E9B0E082E090E021E08030920787
:1078000019F40E94926E03C0182E0E94926EFE011F
:107810003196A8E9B0E082E190E021E08030920763
:1078200019F40E94926E03C0182E0E94926EFE01FF
:107830003196ACEBB0E080E190E021E0803092073F
:1078400019F40E94926E03C0182E0E94926EFE01DF
:107850003196ADECB0E082E190E021E0803092071B
:1078600019F40E94926E03C0182E0E94926EEAE7ED
:10787000F1E0A0E9B0E085E090E021E080309207FF
:1078800019F40E94926E03C0182E0E94926EFE019F
:107890003196AEE1BFE089E090E021E080309207D0
:1078A00031F40E94816E06C00E94926E30C0182E84
:1078B0000E94816E90E09E012F5F3F4F89811816D4
:1078C00034F5AE014F5F5F4FF901E90FF11D808183
:1078D00080538A3090F089E0F90111928A95E9F796
:1078E000F901AEE1BFE089E090E021E0803092074D
:1078F000D9F2182E0E94926E0AC09F5F983038F419
:107900009A01FA01E90FF11D80811816ECF2FE01CF
:107910003196A7E2BFE089E090E021E08030920755
:1079200031F40E94816E06C00E94926E30C0182E03
:107930000E94816E90E09E012F5F3F4F8981181653
:1079400034F5AE014F5F5F4FF901E90FF11D808102
:1079500080538A3090F089E0F90111928A95E9F715
:10796000F901A7E2BFE089E090E021E080309207D2
:10797000D9F2182E0E94926E0AC09F5F983038F498
:107980009A01FA01E90FF11D80811816ECF26E964A
:107990000FB6F894DEBF0FBECDBFDF91CF911F9120
:1079A0000F910895CFEFD0E1DEBFCDBF80E990E029
:1079B00090934B0E80934A0E8EE490E090934B0E82
:1079C00080934A0E80EA90E090934B0E80934A0E8B
:1079D0008BE290E090934B0E80934A0E87E890E004
:1079E00090934B0E80934A0E82E39FE090934B0E50
:1079F00080934A0E0E947E590E946D3F0E94321F62
:107A00000E945D050E9490590E944E4B0E94413396
:107A10000E94C33AE6EAFDE0A0E8B0E080E190E031
:107A200021E08030920719F40E94816E03C0182E65
:107A30000E94816E8091A60D9091A70D8A3F9105BD
:107A400071F18B3F910538F484369105A1F08D37A3
:107A50009105D9F04AC023E0883E9207A1F123E0C6
:107A6000893E920720F4845F914019F13EC085530E
:107A7000954099F13AC086E28093E20084E08093D9
:107A8000E30083E18093E40030C08EE18093E20064
:107A900084E08093E30083E18093E40026C08EE0DD
:107AA0008093E20084E08093E30083E18093E4002C
:107AB0001CC086E08093E20084E08093E30083E1D1
:107AC0008093E40012C082E08093E20084E080931F
:107AD000E30083E18093E40008C01092E20088E0B4
:107AE0008093E30084E28093E4008091B30D8436B8
:107AF00018F4880F8093B30D0E946E118091A80D29
:107B00009091A90D059738F485E090E09093A90D28
:107B10008093A80D0DC08091A80D9091A90D815D55
:107B2000974030F080ED97E09093A90D8093A80DD9
:107B30008091AA0D9091AB0D28E08030920738F02B
:107B40008959994021F01092AB0D1092AA0D8091A5
:107B5000B20D80FF04C082E08093BA0D02C0109283
:107B6000BA0D8091B20D81FF04C082E08093BE0DFA
:107B700002C01092BE0D8091B20D82FF04C082E05F
:107B80008093CA0D02C01092CA0D8091B30D8A5025
:107B9000813F18F08AE98093B30D8091B50D8F77FE
:107BA00011F08F3130F08091B50D80788461809331
:107BB000B50D0E94E5420E942C5C0E94D1230E94D8
:107BC000934A87E00E94116878940E940658A8950D
:107BD00080E00E94A84A0E94594BFACF1F93162FAB
:107BE000A398992787709070880F991F81640E94CD
:107BF0008959812F0E94895980E00E948959A39A4E
:107C000099271F9108950F931F93162F042FA39860
:107C1000992787709070880F991F80640E948959F6
:107C2000812F0E948959802F0E948959A39A1F9100
:107C30000F910895CF93C091F209CC2309F041C070
:107C400081E08093F2094CE16AE08C2F0E94033EB0
:107C50004C2F8091CF0D883010F0269802C04061E3
:107C6000269A8091D20D883010F0259802C0486085
:107C7000259A60E0862F0E94033E4FEF61E080E08E
:107C80000E94033E40E062E0842F0E94033E40E0F9
:107C900063E0842F0E94033E40E064E0842F0E9452
:107CA000033E40E065E0842F0E94033E40E06CE02C
:107CB000842F0E94033E40E06DE0842F0E94033E2B
:107CC0000AC1C091F209C13089F54CE16AE08C2FFC
:107CD0000E94033E40E0642F8C2F0E94033E4FEF32
:107CE0006C2F8C2F0E94033E40E062E08C2F0E949C
:107CF000033E40E063E08C2F0E94033E40E064E0DE
:107D00008C2F0E94033E40E065E08C2F0E94033ED2
:107D100040E06CE08C2F0E94033E40E06DE08C2F31
:107D20000E94033E82E08093F209D5C0C091F2091F
:107D3000C23089F54CE16AE08C2F0E94033E40E09E
:107D4000642F8C2F0E94033E4FEF61E08C2F0E9426
:107D5000033E40E06C2F8C2F0E94033E40E063E026
:107D60008C2F0E94033E40E064E08C2F0E94033E73
:107D700040E065E08C2F0E94033E40E06CE08C2FD9
:107D80000E94033E40E06DE08C2F0E94033E83E0A2
:107D90008093F209A0C0C091F209C33089F54CE18B
:107DA0006AE08C2F0E94033E40E0642F8C2F0E94DB
:107DB000033E4FEF61E08C2F0E94033E40E062E003
:107DC0008C2F0E94033E40E06C2F8C2F0E94033EBC
:107DD00040E064E08C2F0E94033E40E065E08C2F81
:107DE0000E94033E40E06CE08C2F0E94033E40E086
:107DF0006DE08C2F0E94033E84E08093F2096BC0FB
:107E0000C091F209C43089F54CE16AE08C2F0E94E0
:107E1000033E4CEF60E08C2F0E94033E4FEF61E089
:107E20008C2F0E94033E40E062E08C2F0E94033EB4
:107E300040E063E08C2F0E94033E40E06C2F8C2FCB
:107E40000E94033E40E065E08C2F0E94033E40E02C
:107E50006CE08C2F0E94033E40E06DE08C2F0E946E
:107E6000033E85E08093F20936C0C091F209C53027
:107E700081F54CE16AE08C2F0E94033E40E0642FC4
:107E80008C2F0E94033E40EF61E08C2F0E94033E46
:107E900040E062E08C2F0E94033E40E063E08C2FC4
:107EA0000E94033E40E064E08C2F0E94033E40E0CD
:107EB0006C2F8C2F0E94033E40E06CE08C2F0E94C0
:107EC000033E40E06DE08C2F0E94033E1092F209C9
:107ED00002C01092F209CF9108959B9AA39A4CE1A7
:107EE0006AE080E00E94033E40E064E1842F0E944B
:107EF000033E40E08091CF0D883010F0269802C0FC
:107F00004061269A8091D20D883010F0259802C0E9
:107F10004860259A60E0862F0E94033E4FEF61E0A3
:107F200080E00E94033E40E062E0842F0E94033E16
:107F300040E063E0842F0E94033E40E064E0842F31
:107F40000E94033E40E065E0842F0E94033E40E033
:107F50006CE0842F0E94033E40E06DE0842F0E947D
:107F6000033E4CE16AE081E00E94033E40E064E1B0
:107F700081E00E94033E40E0642F81E00E94033EC6
:107F80004FEF61E0862F0E94033E40E062E081E017
:107F90000E94033E40E063E081E00E94033E40E037
:107FA00064E081E00E94033E40E065E081E00E94E1
:107FB000033E40E06CE081E00E94033E40E06DE063
:107FC00081E00E94033E4CE16AE082E00E94033EB1
:107FD00040E064E182E00E94033E40E0642F82E0E2
:107FE0000E94033E4FEF61E082E00E94033E40E0CA
:107FF00062E0862F0E94033E40E063E082E00E9440
:10800000033E40E064E082E00E94033E40E065E021
:1080100082E00E94033E40E06CE082E00E94033E6A
:1080200040E06DE082E00E94033E4CE16AE083E0C4
:108030000E94033E40E064E183E00E94033E40E092
:10804000642F83E00E94033E4FEF61E083E00E94D3
:10805000033E40E062E083E00E94033E40E063E0D4
:10806000862F0E94033E40E064E083E00E94033ECE
:1080700040E065E083E00E94033E40E06CE083E086
:108080000E94033E40E06DE083E00E94033E4CE12D
:108090006AE084E00E94033E40E064E184E00E94E4
:1080A000033E4CEF60E084E00E94033E4FEF61E04E
:1080B00084E00E94033E40E062E084E00E94033ED0
:1080C00040E063E084E00E94033E40E064E0862FED
:1080D0000E94033E40E065E084E00E94033E40E0F1
:1080E0006CE084E00E94033E40E06DE084E00E948A
:1080F000033E4CE16AE085E00E94033E40E064E11B
:1081000085E00E94033E40E065E185E00E94033E79
:1081100040E0642F85E00E94033E40EF61E085E08F
:108120000E94033E40E062E085E00E94033E40E0A2
:1081300063E085E00E94033E40E064E085E00E9449
:10814000033E40E065E0862F0E94033E40E06CE085
:1081500085E00E94033E40E06DE085E00E94033E22
:1081600008950F931F93CF93082FC62F142F20E04D
:1081700030E0613611F421E030E080E090E0C1347D
:1081800011F481E090E0822B932B892B91F060E039
:10819000812F0E94EE3D21E030E0002E02C0220F30
:1081A000331F0A94E2F7482F422B60E0812F0E9490
:1081B000033E20E030E0C23611F421E030E080E000
:1081C00090E0C23411F481E090E0822B932B892B54
:1081D00089F061E0812F0E94EE3D21E030E002C095
:1081E000220F331F0A95E2F7482F422B61E0812FBF
:1081F0000E94033ECF911F910F9108950F931F93FB
:10820000CF93082FC62F142F20E030E0613611F4F1
:1082100021E030E080E090E0C13411F481E090E0B2
:10822000822B932B892BA1F060E0812F0E94EE3DE1
:1082300021E030E0002E02C0220F331F0A94E2F743
:10824000922F9095482F492360E0812F0E94033E92
:1082500020E030E0C23611F421E030E080E090E030
:10826000C23411F481E090E0822B932B892B99F09A
:1082700061E0812F0E94EE3D21E030E002C0220F3C
:10828000331F0A95E2F7922F9095482F492361E01A
:10829000812F0E94033ECF911F910F9108950F935C
:1082A0001F93CF93182FC62F042F20E030E06136A4
:1082B00011F421E030E080E090E0C13411F481E07D
:1082C00090E0822B932B892B29F0412F64E1802FA2
:1082D0000E94033E20E030E0C23611F421E030E09D
:1082E00080E090E0C23411F481E090E0822B932B87
:1082F000892B29F0412F65E1802F0E94033ECF9109
:108300001F910F910895FF920F931F93CF93082F02
:10831000C62F142F50E0F52E20E030E0613611F426
:1083200021E030E080E090E0C13411F481E090E0A1
:10833000822B932B892B09F448C062E1812F0E9484
:10834000EE3D21E030E0002E02C0220F331F0A94E0
:10835000E2F7582F522B1123C1F50430E1F480913C
:10836000CF0D8830C0F480918A00882351F080912D
:10837000B80D882331F08091800080628093800066
:1083800006C0809180008F7D809380002E98FF240E
:10839000F394F092B80D0330C1F48091D20D88307F
:1083A000A0F480918800882331F08091800080685B
:1083B0008093800006C0809180008F77809380003A
:1083C0002D98FF24F394F092C90D20E030E0C236DE
:1083D00011F421E030E080E090E0C23411F481E05B
:1083E00090E0822B932B892B69F063E1812F0E940F
:1083F000EE3D21E030E002C0220F331F0A95E2F784
:10840000582F522BFF2029F4412F6C2F852F0E94CB
:108410004F41CF911F910F91FF9008950F931F939C
:10842000CF93082FC62F142F50E020E030E06136A4
:1084300011F421E030E080E090E0C13411F481E0FB
:1084400090E0822B932B892B31F162E1812F0E94E6
:10845000EE3D21E030E0002E02C0220F331F0A94CF
:10846000E2F7922F9095582F59231123A1F404304D
:1084700041F42E98809180008F7D8093800010932E
:10848000B80D033041F42D98809180008F77809350
:1084900080001092C90D20E030E0C23611F421E0D6
:1084A00030E080E090E0C23411F481E090E0822B73
:1084B000932B892B79F063E1812F0E94EE3D21E01F
:1084C00030E002C0220F331F0A95E2F7922F9095F9
:1084D000582F5923412F6C2F852F0E944F41CF9148
:1084E0001F910F9108951F93CF93C82F162F40E02F
:1084F00020E030E0813611F421E030E080E090E0CF
:10850000C13411F481E090E0822B932B892B29F068
:1085100062E1812F0E94EE3D482F20E030E0C2361C
:1085200011F421E030E080E090E0C23411F481E009
:1085300090E0822B932B892B29F063E1812F0E94FD
:10854000EE3D482F842F9927CF911F9108950F93C7
:108550001F93CF93182FC62F042F40E020E030E068
:10856000613611F421E030E080E090E0C13411F494
:1085700081E090E0822B932B892B29F062E1802F00
:108580000E94EE3D482F20E030E0C23611F421E099
:1085900030E080E090E0C23411F481E090E0822B82
:1085A000932B892B29F063E1802F0E94EE3D482F09
:1085B00081E090E002C0880F991F1A95E2F78423AA
:1085C0009927CF911F910F9108950E94071780E579
:1085D0009AE09093E70A8093E60A1092E80A1092D4
:1085E000DF0A1092E00A8FED9AE00E940F178823AD
:1085F000D1F71092DE0A88E59AE09093F30A80930F
:10860000F20A1092F40A1092EB0A1092EC0A8BEE26
:108610009AE00E940F178823D1F71092EA0A80E6A9
:108620009AE09093FF0A8093FE0A1092000B10923A
:10863000F70A1092F80A87EF9AE00E940F17882332
:10864000D1F71092F60A88E69AE090930B0B80938C
:108650000A0B10920C0B1092030B1092040B83E088
:108660009BE00E940F178823D1F71092020B80E045
:108670009AE09093780A8093770A1092790A109280
:10868000700A82E08093710A80E79AE00E940F17D7
:108690008823D1F788E09AE09093830A8093820A36
:1086A0001092840A10927B0A82E080937C0A8BE706
:1086B0009AE00E940F178823D1F780E19AE0909307
:1086C0008E0A80938D0A10928F0A1092860A82E099
:1086D0008093870A86E89AE00E940F178823D1F7D3
:1086E00088E19AE09093990A8093980A10929A0AE6
:1086F0001092910A82E08093920A81E99AE00E94A6
:108700000F178823D1F780E29AE09093A40A809310
:10871000A30A1092A50A10929C0A82E080939D0AF7
:108720008CE99AE00E940F178823D1F788E29AE03B
:108730009093AF0A8093AE0A1092B00A1092A70AE3
:1087400082E08093A80A87EA9AE00E940F178823A4
:10875000D1F780E39AE09093BA0A8093B90A109215
:10876000BB0A1092B20A82E08093B30A82EB9AE0CD
:108770000E940F178823D1F788E39AE09093C50AE7
:108780008093C40A1092C60A1092BD0A82E08093B8
:10879000BE0A8DEB9AE00E940F178823D1F780E480
:1087A0009AE09093D00A8093CF0A1092D10A109247
:1087B000C80A82E08093C90A88EC9AE00E940F17E9
:1087C0008823D1F788E49AE09093DB0A8093DA0A51
:1087D0001092DC0A1092D30A82E08093D40A83EDCF
:1087E0009AE00E940F178823D1F708958091DE0A3E
:1087F0008823E1F08091DE0A813059F48EED9AE011
:1088000001960E940F17882389F482E08093DE0A84
:108810000DC08091DE0A823049F48EED9AE0019617
:108820000E942118882311F48093DE0A8091EA0ABD
:108830008823E1F08091EA0A813059F48AEE9AE0C7
:1088400001960E940F17882389F482E08093EA0A38
:108850000DC08091EA0A823049F48AEE9AE00196CE
:108860000E942118882311F48093EA0A8091F60A65
:108870008823E1F08091F60A813059F486EF9AE07E
:1088800001960E940F17882389F482E08093F60AEC
:108890000DC08091F60A823049F486EF9AE0019685
:1088A0000E942118882311F48093F60A8091020B0C
:1088B0008823E1F08091020B813059F482E09BE043
:1088C00001960E940F17882389F482E08093020B9F
:1088D00008958091020B823049F482E09BE001967A
:1088E0000E942118882311F48093020B0895CF93DE
:1088F000DF93EC0180E79AE00E942118882309F0B9
:1089000046C08091720A9091730AAA27BB27888378
:108910009983AA83BB83E091770AF091780A8081DA
:108920008D83E091770AF091780A81818E83E091BE
:10893000770AF091780A82818F83E091770AF0912B
:10894000780A83818887E091770AF091780A848198
:108950008987E091770AF091780A85818A87E0918A
:10896000770AF091780A86818B87E091770AF091F7
:10897000780A87818C878091760A8C8380E79AE0D9
:108980000E940F178823D1F781E090E0BBC28BE7EC
:108990009AE00E942118882309F046C080917D0A40
:1089A00090917E0AAA27BB2788839983AA83BB83D9
:1089B000E091820AF091830A80818D83E091820A9E
:1089C000F091830A81818E83E091820AF091830A7B
:1089D00082818F83E091820AF091830A8381888764
:1089E000E091820AF091830A84818987E091820A6A
:1089F000F091830A85818A87E091820AF091830A47
:108A000086818B87E091820AF091830A87818C8727
:108A10008091810A8C838BE79AE00E940F1788234C
:108A2000D1F781E090E06EC286E89AE00E942118BA
:108A3000882309F046C08091880A9091890AAA2764
:108A4000BB2788839983AA83BB83E0918D0AF09129
:108A50008E0A80818D83E0918D0AF0918E0A81814A
:108A60008E83E0918D0AF0918E0A82818F83E0914E
:108A70008D0AF0918E0A83818887E0918D0AF091AA
:108A80008E0A84818987E0918D0AF0918E0A858112
:108A90008A87E0918D0AF0918E0A86818B87E0911A
:108AA0008D0AF0918E0A87818C8780918C0A8C8345
:108AB00086E89AE00E940F178823D1F781E090E0C2
:108AC00021C281E99AE00E942118882309F046C05A
:108AD0008091930A9091940AAA27BB27888399834F
:108AE000AA83BB83E091980AF091990A80818D83D3
:108AF000E091980AF091990A81818E83E091980A19
:108B0000F091990A82818F83E091980AF091990AF5
:108B100083818887E091980AF091990A84818987F6
:108B2000E091980AF091990A85818A87E091980AE4
:108B3000F091990A86818B87E091980AF091990AC1
:108B400087818C878091970A8C8381E99AE00E94C3
:108B50000F178823D1F781E090E0D4C18CE99AE027
:108B60000E942118882309F046C080919E0A9091A6
:108B70009F0AAA27BB2788839983AA83BB83E09196
:108B8000A30AF091A40A80818D83E091A30AF09159
:108B9000A40A81818E83E091A30AF091A40A8281C4
:108BA0008F83E091A30AF091A40A83818887E091E2
:108BB000A30AF091A40A84818987E091A30AF09125
:108BC000A40A85818A87E091A30AF091A40A86818C
:108BD0008B87E091A30AF091A40A87818C8780910A
:108BE000A20A8C838CE99AE00E940F178823D1F7A0
:108BF00081E090E087C187EA9AE00E9421188823EB
:108C000009F046C08091A90A9091AA0AAA27BB2719
:108C100088839983AA83BB83E091AE0AF091AF0A5F
:108C200080818D83E091AE0AF091AF0A81818E83BD
:108C3000E091AE0AF091AF0A82818F83E091AE0A93
:108C4000F091AF0A83818887E091AE0AF091AF0A74
:108C500084818987E091AE0AF091AF0A85818A8785
:108C6000E091AE0AF091AF0A86818B87E091AE0A5F
:108C7000F091AF0A87818C878091AD0A8C8387EA57
:108C80009AE00E940F178823D1F781E090E03AC163
:108C900082EB9AE00E942118882309F046C0809157
:108CA000B40A9091B50AAA27BB2788839983AA831F
:108CB000BB83E091B90AF091BA0A80818D83E0917B
:108CC000B90AF091BA0A81818E83E091B90AF091D4
:108CD000BA0A82818F83E091B90AF091BA0A83813E
:108CE0008887E091B90AF091BA0A84818987E09176
:108CF000B90AF091BA0A85818A87E091B90AF091A0
:108D0000BA0A86818B87E091B90AF091BA0A878105
:108D10008C878091B80A8C8382EB9AE00E940F17AF
:108D20008823D1F781E090E0EDC08DEB9AE00E94BE
:108D30002118882309F046C08091BF0A9091C00A8B
:108D4000AA27BB2788839983AA83BB83E091C40A9F
:108D5000F091C50A80818D83E091C40AF091C50A23
:108D600081818E83E091C40AF091C50A82818F834C
:108D7000E091C40AF091C50A83818887E091C40A12
:108D8000F091C50A84818987E091C40AF091C50AEF
:108D900085818A87E091C40AF091C50A86818B8714
:108DA000E091C40AF091C50A87818C878091C30A3B
:108DB0008C838DEB9AE00E940F178823D1F781E016
:108DC00090E0A0C088EC9AE00E942118882309F066
:108DD00046C08091CA0A9091CB0AAA27BB278883F4
:108DE0009983AA83BB83E091CF0AF091D00A808156
:108DF0008D83E091CF0AF091D00A81818E83E0913A
:108E0000CF0AF091D00A82818F83E091CF0AF0914E
:108E1000D00A83818887E091CF0AF091D00A8481BB
:108E20008987E091CF0AF091D00A85818A87E09105
:108E3000CF0AF091D00A86818B87E091CF0AF0911A
:108E4000D00A87818C878091CE0A8C8388EC9AE047
:108E50000E940F178823D1F781E090E053C083ED83
:108E60009AE00E942118882309F046C08091D50A13
:108E70009091D60AAA27BB2788839983AA83BB83AC
:108E8000E091DA0AF091DB0A80818D83E091DA0AC1
:108E9000F091DB0A81818E83E091DA0AF091DB0A9E
:108EA00082818F83E091DA0AF091DB0A83818887DF
:108EB000E091DA0AF091DB0A84818987E091DA0A8D
:108EC000F091DB0A85818A87E091DA0AF091DB0A6A
:108ED00086818B87E091DA0AF091DB0A87818C87A3
:108EE0008091D90A8C8383ED9AE00E940F17882322
:108EF000D1F781E090E006C0188219821A821B82A5
:108F000080E090E0DF91CF910895CF93DF93DC0173
:108F10008091DE0A882339F48EED9AE090930F0B4E
:108F200080930E0B21C08091EA0A882339F48AEEDF
:108F30009AE090930F0B80930E0B16C08091F60A67
:108F4000882339F486EF9AE090930F0B80930E0BF1
:108F50000BC08091020B882309F072C082E09BE075
:108F600090930F0B80930E0BE0910E0BF0910F0B73
:108F70000084F185E02DED018D818083E0910E0B61
:108F8000F0910F0B0084F185E02D8E818183E091BB
:108F90000E0BF0910F0B0084F185E02D8F81828301
:108FA000E0910E0BF0910F0B0084F185E02D888588
:108FB0008383E0910E0BF0910F0B0084F185E02D7F
:108FC00089858483E0910E0BF0910F0B0084F1856D
:108FD000E02D8A858583E0910E0BF0910F0B0084C4
:108FE000F185E02D8B858683E0910E0BF0910F0BC0
:108FF0000084F185E02D8C858783E0910E0BF09144
:109000000F0B8C818783E0910E0BF0910F0B8D91EC
:109010009C9194838383E0910E0BF0910F0B128649
:10902000E0910E0BF0910F0B1182E0910E0BF0917D
:109030000F0B1282E0910E0BF0910F0B81E08083F9
:10904000DF91CF91089583EF99E00E9477448823C0
:1090500061F183EF99E00E94051483EF99E00E948B
:109060007744882311F183EF99E00E94051483EF80
:1090700099E00E9477448823C1F083EF99E00E9431
:10908000051483EF99E00E947744882371F083EF01
:1090900099E00E94051483EF99E00E9477448823A9
:1090A00021F083EF99E00E9405140895FF920F9339
:1090B0001F93CF93DF93CDB7DEB760970FB6F894C9
:1090C000DEBF0FBECDBF20E0822F99278C01005F4D
:1090D000144FF80180818C7F8083F22EF394BE01BF
:1090E0006F5F7F4F8F2D0E94963988898170982FEE
:1090F000990F990F990FF80180818370892B8083D4
:109100002F2D2B3008F360960FB6F894DEBF0FBEFC
:10911000CDBFDF91CF911F910F91FF900895FC017A
:10912000808183709927009719F0019731F0089595
:1091300080818D728162808308959081892F807FE4
:1091400001F593FD11C0892F83708230D1F0892FF2
:109150008C7F8260808382FF03C08B7F8083089531
:109160008081846080830895808182FF03C08B7F2B
:10917000808303C080818460808380818C7F826053
:1091800080830895FC018081837099278130910547
:10919000BCF0833091051CF0039731F00895808175
:1091A0008F708362808308959081892F807F41F43E
:1091B000892F8C7F808393FF03C0892F887F8083D2
:1091C00008959927853C910509F457C0863C91057F
:1091D000ACF4823C9105C9F1833C91053CF4803CA0
:1091E000910519F1813C910541F17AC0833C9105CB
:1091F00009F45EC0843C9105C1F172C0813D9105C6
:1092000061F1823D910544F4863C9105F1F1873C82
:10921000910509F442C064C0823D910509F450C033
:10922000833D910509F454C05BC0309B03C081E0CD
:1092300090E0089580E090E00895319903C081E0C6
:1092400090E0089580E090E00895329903C081E0B5
:1092500090E0089580E090E00895499903C081E08E
:1092600090E0089580E090E00895349903C081E093
:1092700090E0089580E090E00895359903C081E082
:1092800090E0089580E090E00895369903C081E071
:1092900090E0089580E090E0089586B1992787FDD9
:1092A0009095809590958827990F881F9927089504
:1092B000339903C081E090E0089580E090E0089544
:1092C0004A9903C081E090E0089580E090E008951D
:1092D0004B9903C081E090E0089580E090E008950C
:1092E00080E090E0089530E0832F9927FC01E05F53
:1092F000F44F2081822F807F41F0822F807F982F32
:109300009051822F8F70892B80833F5F3B3060F3B9
:10931000E0E1FBE0309B04C0CF010E948F4803C016
:10932000CF010E94C248E1E1FBE0319904C0CF01C6
:109330000E948F4803C0CF010E94C248E2E1FBE0D7
:10934000329904C0CF010E948F4803C0CF010E9410
:10935000C248E3E1FBE0499904C0CF010E948F4875
:1093600003C0CF010E94C248E4E1FBE0349904C08D
:10937000CF010E948F4803C0CF010E94C248E5E19F
:10938000FBE0359904C0CF010E948F4803C0CF0194
:109390000E94C248E6E1FBE0369904C0CF010E947A
:1093A0008F4803C0CF010E94C248E7E1FBE0379934
:1093B00004C0CF010E948F4803C0CF010E94C24861
:1093C000E8E1FBE0339904C0CF010E948F4803C05D
:1093D000CF010E94C248E9E1FBE04A9904C0CF01F5
:1093E0000E948F4803C0CF010E94C248EAE1FBE01F
:1093F0004B9904C0CF010E948F480895CF010E946D
:10940000C24808959927853C910509F451C0863CCE
:109410009105ACF4823C9105B1F1833C91053CF49B
:10942000803C910511F1813C910531F16BC0833C89
:10943000910509F452C0843C910599F163C0813DC6
:10944000910541F1823D91053CF4863C9105B9F1CD
:10945000873C9105D9F156C0823D910509F444C07D
:10946000833D910509F447C04DC08091100B86954E
:1094700086958170992708958091110B8695869520
:109480008170992708958091120B86958695817039
:10949000992708958091130B869586958170992759
:1094A00008958091140B869586958170992708956B
:1094B0008091150B869586958170992708958091E6
:1094C000160B869586958170992708958091170BC4
:1094D000869586958170992708958091180B8695B9
:1094E00086958170992708958091190B86958695A8
:1094F00081709927089580911A0B869586958170C1
:10950000992708958EEF90E008951092B60087E0B5
:109510008093B0001092B2008EE48093B30082E09A
:109520008093700008950E94854A10921D0B10923E
:109530001E0B10921F0B1092200B1092250B1092F5
:10954000260B0E9456480E94DB050E943B35089579
:10955000CF93C82F80911B0B882311F010921B0B07
:10956000A8950E942348C23011F00E94F643C230F1
:1095700009F471C080911C0B882309F446C08091C6
:109580001C0B815080931C0B0E94071980911D0BAE
:109590008F5F80931D0B823040F010921D0B0E9454
:1095A00073490E94791A0E94160780911E0B8F5FE3
:1095B00080931E0B843040F010921E0B0E94F31A11
:1095C0000E94B15C0E949D5980911F0B8F5F809318
:1095D0001F0B8A3030F010921F0BC13011F00E9427
:1095E000ED138091200B8F5F8093200B843168F006
:1095F0001092200B8091250B8F5F8093250B0E948A
:109600001A3E0E94711C0E9466138091250B8A30BD
:1096100010F11092250B8091210B9091220BA091BB
:10962000230BB091240B0196A11DB11D8093210B3A
:109630009093220BA093230BB093240B0E944536EA
:109640008091260B8F5F8093260B8C3320F0109235
:10965000260B0E940436CF9108958091210B9091A2
:10966000220BA091230BB091240BBC01CD010895D6
:109670001F920F920FB60F9211248F931092B20087
:1096800081E080931B0B80911C0B8F5F80931C0BE0
:109690008F910F900FBE0F901F9018950E945D58EC
:1096A0000E94EF5960E076E980E090E00E940A5A5B
:1096B000089504C00E9482580E94D5580E946C5898
:1096C0008823C1F70895FC0190E061506F3F21F0BD
:1096D000819198276150E0F7892F992708950F937A
:1096E0001F938C01FC0181818150682FC801019674
:1096F0000E94634BF801808381819927BC01C801D6
:109700000E949D581F910F910895AF92BF92CF92E2
:10971000DF92EF92FF920F931F93CF93DF93CDB71A
:10972000DEB7C35ED0400FB6F894DEBF0FBECDBF2C
:109730006C01FC0181818150682FC60101960E9455
:10974000634BD6019C91981711F00C94EB57F601DE
:109750008281882309F0F8C083819927813591059A
:1097600009F449C0823591053CF48033910589F0B4
:109770008035910561F1E8C08335910509F48EC00B
:10978000833591050CF478C08435910509F4B2C095
:10979000DBC08E01035D1F4F80E5D8011D928A95C5
:1097A000E9F785E18EA71FA680E888ABF6018481E2
:1097B00089AB992796012B5F3F4FAC01B901CE01D0
:1097C000C2960E94956DC8010E946F4BBDC08E016C
:1097D000035D1F4F80E5D8011D928A95E9F785E06A
:1097E0008EA71FA680EA88AB0E94C93389ABC80147
:1097F0000E946F4BA9C0F601B4800F2EFDE2EF2E40
:10980000FF24F02DEC0EFD1E80E5D7011D928A95F8
:10981000E9F789E18EA71FA681EA88AB8E0103587C
:109820001F4FB8018B2D0E94F333B9AA8CE0FE01C3
:10983000F296D8010D9001928A95E1F7F80184859E
:1098400095859FAF8EAF8685FE01E05CFF4F8083DC
:10985000F8018785FE01EF5BFF4F80839927AC01FC
:10986000BE0163577F4FCE018E5B9F4F0E94956D67
:10987000C7010E946F4B68C00E948133FE01BD96F4
:1098800080E5DF011D928A95E9F784E08EA71FA687
:1098900082EA88ABCF010E946F4B56C0F60145812A
:1098A00056818481FE01ED51FF4F8083813108F0A4
:1098B0004BC080E5FE01BD9611928A95E9F787E1DC
:1098C0008EA71FA683EA88AB5BAB4AABFE01ED51C6
:1098D000FF4F808189ABFE01F4969927DA01019749
:1098E00024F00E94796E0192FACFCE018D960E94EB
:1098F0006F4B2AC0F601458156818481FE01ED51EE
:10990000FF4F8083813100F5F60137969927DA0100
:10991000019724F001900E94866EFACFDE019D9699
:1099200080E5FD0111928A95E9F787E08EA71FA6D1
:1099300084EA88AB5BAB4AABFE01ED51FF4F8081FF
:1099400089ABCD010E946F4BF6018281813011F00D
:109950000C94F45783819927AA27BB27FC013197E0
:10996000EB36F10510F00C94DD57E65BFF4FEE0F80
:10997000FF1F0590F491E02D09940E942F33F6010A
:10998000B4808B2D8150823210F00C94F45720E07B
:10999000AE01475F5F4F822F9927DA01A80FB91FE9
:1099A000F601E80FF91F82858C932F5F2F3098F313
:1099B000F6018581898386818A8387818B83838D64
:1099C000948D9E838D83858D8F8380858887818507
:1099D0008C83818D888F828D898F6B2DCE0101962E
:1099E0000E94E2386B2DCE0101960E94D8241DA65C
:1099F00085E08EA711E01FA781E888AB19AACE01E8
:109A00008D960E946F4B812F0E94A84A0C94F457A8
:109A1000F601B4808B2D8150823208F047C06B2D47
:109A2000CE0101960E9427398EE18EA781E08FA793
:109A300082E888ABB9AA89818AAB8A818BAB8B819A
:109A40008CAB8C818EAB8D819E81FE01E85BFF4FDC
:109A5000918380838F81FE01E65BFF4F808320E04E
:109A6000BE016F5F7F4FAE01475F5F4F822F992727
:109A7000DC01A60FB71FFA01E80FF91F8081FD0175
:109A800086AB2F5F2F3090F388858DAB888DFE01DC
:109A9000EA5BFF4F8083898DFE01E95BFF4F808386
:109AA000CE018D960E946F4B0C94F457FFEFBF16BA
:109AB00011F00C94F457FE01ED51FF4F1082FE019E
:109AC000ED51FF4F8081982F823210F00C94F457A3
:109AD0000F2EF3EEEF2EFF24F02DEC0EFD1E6E0187
:109AE0000894C11CD11C8E01075F1F4F0F2EF6E496
:109AF000AF2EBB24F02DAC0EBD1E892F8F5F682FBB
:109B0000CE0101960E9427398EE18EA781E08FA7B2
:109B100082E888ABD7018C918F5F89AB89818AAB52
:109B20008A818BAB8B818CAB8C818EAB8D819E813E
:109B3000FE01E85BFF4F918380838F81FE01E65B2E
:109B4000FF4F808320E0822F9927DC01AC0DBD1DE3
:109B5000F801E80FF91F8081FD0186AB2F5F2F30E0
:109B600090F388858DAB888DD5018C93898DFE010E
:109B7000E95BFF4F8083CE018D960E946F4B81E0A1
:109B80000E94A84AF70180818F5F8083982F8232DC
:109B900008F4B3CF0C94F4570E942F33F601B4802D
:109BA000AE0143585F4F96012B5F3F4F8FE0DA01C4
:109BB000F90101900D928A95E1F7F6018489FA0185
:109BC0008787BA018B2D0E94793981E08FA783E8BE
:109BD00088ABB9AA85E08EA7CE018D960E946F4B07
:109BE0000C94F457F601B4808B2D81508A3010F517
:109BF00081E08FA784E888ABB9AA8E0103581F4F74
:109C0000B8018B2D0E9496398FE0FE01F296D801A3
:109C10000D9001928A95E1F7F8018785FE01EF5BCF
:109C2000FF4F808385E18EA7CE018D960E946F4BFA
:109C30000C94F457FFEFBF1611F00C94F457FE018B
:109C4000ED51FF4F1082FE01ED51FF4F8081982FA3
:109C50008B3010F00C94F457BB24B3948E0103584E
:109C60001F4F0F2EFFE0AF2EF02D0F2EF1E4EF2E41
:109C7000FF24F02DEC0EFD1E0F2EF3EECF2EDD2473
:109C8000F02DCC0EDD1EBFA684E888AB892F8F5F38
:109C900089ABB8010E949639FE01F296D8012A2DAF
:109CA0000D9001922A95E1F7F8018785D7018C93F1
:109CB00085E18EA7CE018D960E946F4B8B2D0E9461
:109CC000A84AF60180818F5F8083982F8B30D8F26D
:109CD0000C94F457A8950E942F330E94321FA89528
:109CE0000E946D22A8950E94D123A8950E94CB12B4
:109CF000A8950E947D5CA8950E943206A8950E94B6
:109D0000A8350E94351181E08FA786E888AB84E0F2
:109D10008EA7CE018D960E946F4B0C94F457F601DE
:109D20008181863011F00C94F45784E18EA781E094
:109D30008FA787E888AB8DE0A2E8B1E0FE01F1963D
:109D40000D9001928A95E1F70E942D4B9B01AC0189
:109D5000AA27BB278EAFBB27A52F942F832F8FAFAA
:109D6000FE01E05CFF4F2083CE018D960E946F4B79
:109D70000C94F4570C9400000C94F457F6013496AC
:109D8000A5ECBAE088E090E021E08030920719F479
:109D90000E94926E03C0182E0E94926E81E08FA7DF
:109DA00089E888AB84E08EA7CE018D960E946F4B28
:109DB0000C94F45781E08FA78AE888AB8CE08EA7DB
:109DC000FE01F196A5ECBAE088E090E021E0803059
:109DD000920719F40E94816E03C0182E0E94816EB2
:109DE000CE018D960E946F4B0C94F457CE0187964E
:109DF0000E943E3081E08FA781EA88AB8FA189ABBA
:109E000088A58AAB89A58BAB8AA58CAB8BA58DABBE
:109E10008CA58EAB8AE08EA7CE018D960E946F4BEB
:109E20000C94F457F601B480F1E2FB15B8F1BE01D1
:109E30006E5D7F4F8B2D0E94303181E08FA782EACB
:109E400088ABB9AA8BA18BAB8CA18EAB8AA18AAB54
:109E50008DA19EA1892F99278CAB8DA18DAB21E17E
:109E6000B21641F48091CF0D883020F480918A00A1
:109E70008FAB0CC082E1B81641F48091D20D8830CE
:109E800020F4809188008FAB01C01FAA8BE08EA7C1
:109E9000CE018D960E946F4B0C94F457AFEFBA161B
:109EA00011F00C94F457FE01ED51FF4F1082FE01AA
:109EB000ED51FF4F8081982F823210F00C94F457AF
:109EC0008F01BE016E5D7F4F892F8F5F0E94303101
:109ED00081E08FA782EA88ABF8012081822F8F5F13
:109EE00089AB8BA18BAB8CA18EAB8AA18AAB8DA1E8
:109EF0009EA1892F99278CAB8DA18DAB203141F488
:109F00008091CF0D883020F480918A008FAB0DC0F6
:109F1000D8018C91813141F48091D20D883020F4A8
:109F2000809188008FAB01C01FAA8BE08EA7CE0165
:109F30008D960E946F4B81E00E94A84AF8018081B3
:109F40008F5F8083982F823208F4BBCF0C94F45734
:109F5000CE014A960E942D328AE08EA781E08FA71B
:109F600080EA88AB88A189AB8E8D8AAB8A8D9B8D68
:109F7000892F99278BAB8A8D8CAB8D8D8DAB8C8D7A
:109F80008EABCE018D960E946F4B0C94F457F60168
:109F9000648180E00E94282884E08EA781E08FA75A
:109FA00083EA88ABCE018D960E946F4B0C94F457D8
:109FB000DE01A353BF4FF60184818C938581FD019F
:109FC0008183F6018681FD018283F6018781FD018F
:109FD0008383F6018085FD018483F6018185FD017F
:109FE0008583F6018285FD018683F6018385FD0167
:109FF0008783CD010E94302884E08EA781E08FA75F
:10A0000084EA88ABCE018D960E946F4B0C94F45776
:10A01000FE01E358FF4FA0E0B0E080E190E021E0D6
:10A020008030920719F40E94816E03C0182E0E949E
:10A03000816EF60184819581A681B781FE01EF577B
:10A04000FF4F80839183A283B383DE01A358BF4F68
:10A05000F6018085FD018087F6018185FD018187FC
:10A06000F6018285FD018287A0E0B0E080E190E00A
:10A0700021E08030920719F40E94926E03C0182EDE
:10A080000E94926E84E08EA781E08FA780EC88AB5F
:10A09000CE018D960E946F4BA7C7FE01E358FF4F7C
:10A0A000A0E0B0E080E190E021E08030920719F478
:10A0B0000E94816E03C0182E0E94816E8BE08EA7D5
:10A0C00081E08FA781EC88ABFE01EF57FF4F8081C5
:10A0D0009181A281B38189AB9AABABABBCABFE01E2
:10A0E000E358FF4F80858DAB81858EAB82858FAB2A
:10A0F000CE018D960E946F4B77C78AE38EA781E0D1
:10A100008FA780ED88ABFE01F196A8E9B0E082E16F
:10A1100090E021E08030920719F40E94816E03C024
:10A12000182E0E94816EFE01ED5BFF4FAAEAB0E09F
:10A1300082E190E021E08030920719F40E94816E64
:10A1400003C0182E0E94816EFE01EB5AFF4FADEC4A
:10A15000B0E082E190E021E08030920719F40E94A3
:10A16000816E03C0182E0E94816ECE018D960E94D2
:10A170006F4B3AC784E18EA781E08FA78EED88AB45
:10A18000FE01F196ACEBB0E080E190E021E08030A0
:10A19000920719F40E94816E03C0182E0E94816EEE
:10A1A000CE018D960E946F4B1FC70E94A83584E098
:10A1B0008EA781E08FA781ED88ABCE018D960E949E
:10A1C0006F4B12C788E08EA781E08FA78FED88AB19
:10A1D0000E943C368BAB0E9440369AAB89ABFE01A5
:10A1E000ED51FF4FACECB0E081E090E021E0803039
:10A1F000920719F40E94816E03C0182E0E94816E8E
:10A20000FE01ED51FF4F80818CABCE018D960E94F7
:10A210006F4BEAC6FE01E358FF4F80E5DF011D9258
:10A220008A95E9F7ACECB0E081E090E021E0803085
:10A23000920719F40E94926E03C0182E0E94926E2B
:10A24000FE01E358FF4FA5E9B0E081E090E021E096
:10A250008030920719F40E94926E03C0182E0E945B
:10A26000926EFE01E358FF4FA6E9B0E082E090E075
:10A2700021E08030920719F40E94926E03C0182EDC
:10A280000E94926E84E08EA781E08FA780EE88AB5B
:10A29000CE018D960E946F4BA7C6F60185819681EF
:10A2A0009093A70D8093A60D878190859093A90D1B
:10A2B0008093A80D818592859093AB0D8093AA0D14
:10A2C00083858093AC0D84858093AD0D85858093C7
:10A2D000AE0D878590899093B10D8093B00D8685E2
:10A2E0008093AF0D81898093B20D82898093B30DE5
:10A2F00083898093B40D8489982F9F778091B50DC1
:10A300008078892B8093B50D948990788F77892BED
:10A310008093B50DE6EAFDE0A0E8B0E080E190E0D2
:10A3200021E08030920719F40E94926E03C0182E2B
:10A330000E94926E85E08EA791E09FA785EA88AB88
:10A3400099ABCE018D960E946F4B4EC685E18EA7CC
:10A3500081E08FA786EA88AB19AA8091E200863255
:10A3600069F48091E300843049F48091E400833102
:10A3700029F484E690E09BAB8AAB57C08091E20061
:10A380008E3169F48091E300843049F48091E400D7
:10A39000833129F48DE790E09BAB8AAB46C0809176
:10A3A000E2008E3069F48091E300843049F48091BA
:10A3B000E400833129F48AEF90E09BAB8AAB35C08F
:10A3C0008091E200863069F48091E300843049F4A2
:10A3D0008091E400833129F484EF91E09BAB8AAB58
:10A3E00024C08091E200823069F48091E3008430DF
:10A3F00049F48091E400833129F488EE93E09BAB2B
:10A400008AAB13C08091E200882369F48091E30055
:10A41000883049F48091E400843229F485E395E0A2
:10A420009BAB8AAB02C01BAA1AAA8091A80D90917F
:10A43000A90D9DAB8CAB8091AA0D9091AB0D9FABFC
:10A440008EAB8091AC0D88AF8091AD0D89AF8091BE
:10A45000AE0D8AAF8091B00D9091B10D9DAF8CAFD4
:10A460008091AF0D8BAF8091B20D8EAF8091B30D07
:10A470008FAF8091B40DFE01E05CFF4F808380912F
:10A48000B50DFE01EF5BFF4F8083CE018D960E94DC
:10A490006F4BAAC5DE01AB52BF4FF60184818C938E
:10A4A0008581FD018183D60116968CE0FE01E9527B
:10A4B000FF4F0D9001928A95E1F7FE01ED51FF4F9C
:10A4C0001082FE01ED51FF4F8081982F8C30A0F457
:10A4D0009E012B523F4FDF01F901E90FF11D8281EF
:10A4E000882321F08F3F11F0815082838C918F5F00
:10A4F0008C93982F8C3080F3CE018B529F4F0E940B
:10A50000423784E08EA781E08FA787EA88ABCE012F
:10A510008D960E946F4B68C58E010B521F4FC8016C
:10A520000E94603782E18EA781E08FA788EA88AB1E
:10A53000D8018C9189ABF80181818AABFE01ED5184
:10A54000FF4F1082FE01ED51FF4F8081982F8C301C
:10A5500080F49801DF01F901E90FF11D82818F3F3D
:10A5600011F08F5F82838C918F5F8C93982F8C304A
:10A5700090F38CE0DE01A952BF4FFE01F3960D90DF
:10A5800001928A95E1F7CE018D960E946F4B2CC502
:10A59000F6018481FE01E358FF4F8083D6011596B2
:10A5A00084E1FE01E258FF4F0D9001928A95E1F798
:10A5B000FE01ED51FF4F1082FE01ED51FF4F8081F2
:10A5C000982F8431A0F49E0123583F4FDF01F901F9
:10A5D000E90FF11D8181882321F08F3F11F0815017
:10A5E00081838C918F5F8C93982F843180F3DE016F
:10A5F000A358BF4FF601818DFD01858BF601828D39
:10A60000FD01868BD6015B9684E1FE01EC56FF4F7F
:10A610000D9001928A95E1F7FE01ED51FF4F1082F6
:10A62000FE01ED51FF4F8081982F8431A0F49E01EF
:10A6300023583F4FDF01F901E90FF11D8789882376
:10A6400021F08F3F11F08150878B8C918F5F8C931D
:10A65000982F843180F3CE0183589F4F0E9470372A
:10A6600084E08EA781E08FA789EA88ABCE018D9622
:10A670000E946F4BB9C48E0103581F4FC8010E943E
:10A6800080378FE28EA781E08FA78AEA88ABD80156
:10A690008C9189ABFE01ED51FF4F1082FE01ED510F
:10A6A000FF4F8081982F843180F49801DF01F901F8
:10A6B000E90FF11D81818F3F11F08F5F81838C91B4
:10A6C0008F5F8C93982F843190F384E1DE01A25840
:10A6D000BF4FFE01F2960D9001928A95E1F7DE01DF
:10A6E000A358BF4FFD018589FE01EA5BFF4F8083C0
:10A6F000FD018689FE01E95BFF4F8083FE01ED517C
:10A70000FF4F1082FE01ED51FF4F8081982F843161
:10A7100080F49D01DF01F901E90FF11D87898F3F69
:10A7200011F08F5F878B8C918F5F8C93982F843182
:10A7300090F384E1DE01AC56BF4FFE01E85BFF4FB2
:10A740000D9001928A95E1F7CE018D960E946F4B94
:10A750004BC4F601B48085819927982F88272681DC
:10A76000820F911DBC018B2D0E94B23285E08EA715
:10A7700081E08FA782EC88ABB9AACE018D960E94AA
:10A780006F4B32C4F601B4808CE08EA781E08FA7B6
:10A7900083EC88ABB9AA8B2D0E9470328AAB8B2DCB
:10A7A0000E948C32892F99278BAB8B2D0E948C3283
:10A7B0008CAB8B2D0E94DB32892F99278DAB8B2D93
:10A7C0000E94DB328EAB8B2D0E94F332892F9927AA
:10A7D0008FAB8B2D0E94F33288AFCE018D960E94F5
:10A7E0006F4B02C420E0F601848181FD21E0F60177
:10A7F000848182FD2260F6018181863029F46581A1
:10A80000822F0E940B33F0C360E0822F0E940B3333
:10A81000EBC30E94103384E08EA781E08FA785EC04
:10A8200088ABCE018D960E946F4BDEC3F601B480DB
:10A830009E0123583F4F9581492F4170D9018C913A
:10A84000887F9670842B892B8C9386819781F90160
:10A8500092838183F60180859185F90194838383B6
:10A86000F6018685F9018187F6018785F9018287DE
:10A87000F60182859385F90196838583F6018485A7
:10A880009585F90190878783F6018089F90183878F
:10A89000F6018189F9018487F6018289F9018587AA
:10A8A000F6018389F9018687D60154968FE0FE016F
:10A8B000E457FF4F0D9001928A95E1F7F60183A1CD
:10A8C000F901868FF60184A1F901878FF60185A130
:10A8D000F90180A3F60186A1F90181A315E0D60153
:10A8E0009796FE01E156FF4F812F0D9001928A95B8
:10A8F000E1F7F60184A595A5A6A5B7A5F90187A35B
:10A9000090A7A1A7B2A7F60180A9F90183A7B90171
:10A910008B2D0E94023881E08FA782ED88AB1EA7A5
:10A92000B9AACE018D960E946F4B5EC3F601B4802A
:10A930008E0103581F4FB8018B2D0E943A3881E0D9
:10A940008FA783ED88AB81E38EA7B9AAD8019C912C
:10A95000292F21708AA9887F9670822B892B8AAB38
:10A96000F801818192819CAB8BAB838194819EABFA
:10A970008DAB81858BAF82858CAF8581968198AFB9
:10A980008FAB878190859AAF89AF83858DAF8485A2
:10A990008EAF85858FAF8685FE01E05CFF4F80839B
:10A9A0008FE0DE01A457BF4FFE01EF5BFF4F0D901C
:10A9B00001928A95E1F7F801868DFE01E05BFF4F79
:10A9C0008083F801878DFE01EF5AFF4F8083F801E5
:10A9D00080A1FE01EE5AFF4F8083F80181A1FE01A4
:10A9E000ED5AFF4F808385E0DE01A156BF4FFE0187
:10A9F000EC5AFF4F0D9001928A95E1F7F80187A17B
:10AA000090A5A1A5B2A5FE01E75AFF4F80839183CF
:10AA1000A283B383F80183A5FE01E35AFF4F80832D
:10AA2000CE018D960E946F4BDFC2F601B480AE015D
:10AA300043585F4F828DDA018C93838DFA018183B5
:10AA4000F601848DFA018283F6018681FA018383FF
:10AA5000F6018781FA018483F6018085FA018583F6
:10AA6000F6018185FA018683F6018285FA018783E2
:10AA7000F601858DFA01878BC6010B962FE0FE014A
:10AA8000EB57FF4FDC010D9001922A95E1F7BA01D7
:10AA90008B2D0E94723881E08FA784ED88AB85E012
:10AAA0008EA7B9AACE018D960E946F4B9DC2F6016A
:10AAB000B4808E0103581F4FB8018B2D0E94AA3815
:10AAC00081E08FA785ED88AB8FE18EA7B9AAD80169
:10AAD0008C91FE01E95BFF4F8083F8018181FE01CB
:10AAE000E85BFF4F8083F8018281FE01E75BFF4F47
:10AAF0008083F80183818BAB84818CAB85818DABA6
:10AB000086818EAB87818FAB8789FE01E65BFF4F25
:10AB100080838FE0DE01AB57BF4FFE01F8960D90AA
:10AB200001928A95E1F7CE018D960E946F4B5CC22F
:10AB3000F6013496A3E3B8E082E090E021E08030B3
:10AB4000920719F40E94926E03C0182E0E94926E12
:10AB500081E08FA783EE88AB84E08EA7CE018D962F
:10AB60000E946F4B41C281E08FA784EE88AB84E1E5
:10AB70008EA7FE01F196A3E3B8E082E090E021E029
:10AB80008030920719F40E94816E03C0182E0E9433
:10AB9000816ECE018D960E946F4B26C2F601B48065
:10ABA000C6010596BC018B2D0E94903781E08FA7CE
:10ABB00088ED88AB85E08EA7B9AACE018D960E945C
:10ABC0006F4B12C2F601B48081E08FA789ED88AB8C
:10ABD00080E28EA7B9AABE016E5C7F4F8B2D0E94CA
:10ABE000C937CE018D960E946F4BFEC1F60184815C
:10ABF0008093C10D85818093C20D86818093C30DA2
:10AC000087818093C40D80858093C50D8185809355
:10AC1000C60D82858093C70D83858093C80DE1ECB6
:10AC2000FDE0AEEABEE088E090E021E080309207EF
:10AC300019F40E94926E03C0182E0E94926E81E059
:10AC40008FA785EE88AB84E08EA7CE018D960E94FB
:10AC50006F4BCAC181E08FA786EE88AB8CE08EA7D0
:10AC60008091C10D89AB8091C20D8AAB8091C30DDB
:10AC70008BAB8091C40D8CAB8091C50D8DAB809159
:10AC8000C60D8EAB8091C70D8FAB8091C80D88AF7C
:10AC9000CE018D960E946F4BA7C1F6013496AEECA3
:10ACA000BEE080E590E021E08030920719F40E9438
:10ACB000926E03C0182E0E94926EF60184818093DA
:10ACC000D50D8581982F97708091D70D887F892B1E
:10ACD0008093D70D86818093D60D808D8093D80D7B
:10ACE000818D982F97708091DA0D887F892B8093C2
:10ACF000DA0D828D8093D90D84A58093DB0D85A517
:10AD0000982F97708091DD0D887F892B8093DD0DC2
:10AD100086A58093DC0DE05CFF4F80818093DE0D83
:10AD2000F601EF5BFF4F8081982F97708091E00DC7
:10AD3000887F892B8093E00DF601EE5BFF4F8081C9
:10AD40008093DF0D81E08FA787EE88AB84E08EA72C
:10AD5000CE018D960E946F4B47C181E08FA788EE90
:10AD600088AB84E58EA7FE01F196AEECBEE080E5EF
:10AD700090E021E08030920719F40E94816E03C0B8
:10AD8000182E0E94816ECE018D960E946F4B2CC1B1
:10AD9000F6013496AEE1BFE089E090E021E080303A
:10ADA000920719F40E94926E03C0182E0E94926EB0
:10ADB000F6013D96A7E2BFE089E090E021E0803017
:10ADC000920719F40E94926E03C0182E0E94926E90
:10ADD00081E08FA789EE88AB84E08EA7CE018D96A7
:10ADE0000E946F4B01C181E08FA78AEE88AB87E19B
:10ADF0008EA7FE01F196AEE1BFE089E090E021E090
:10AE00008030920719F40E94816E03C0182E0E94B0
:10AE1000816EFE01FA96A7E2BFE089E090E021E0B2
:10AE20008030920719F40E94816E03C0182E0E9490
:10AE3000816ECE018D960E946F4BD6C0C6010596DD
:10AE40000E94043A81E08FA786ED88AB85E08EA74B
:10AE5000CE018D960E946F4BC7C081E08FA787ED12
:10AE600088AB8DE18EA7CE01C2960E94143ACE0126
:10AE70008D960E946F4BB8C0F601B480C60104964F
:10AE80000E94243A81E08FA78AED88AB85E08EA7E7
:10AE9000B9AACE018D960E946F4BA6C0F601B48070
:10AEA00081E08FA78BED88AB8AE48EA7BE016F5C33
:10AEB0007F4F8B2D0E94513AB9AACE018D960E94E8
:10AEC0006F4B92C0F601B4808B2D0E94351381E048
:10AED0008FA78CED88ABB9AA85E08EA7CE018D96A1
:10AEE0000E946F4B81C0F6014481558181E08FA79C
:10AEF0008DED88AB86E18EA75AAB49ABFE01ED51D3
:10AF0000FF4F1082FE01ED51FF4F8081982F80315D
:10AF1000C8F48E010F5F1F4FBF01892F99279C0135
:10AF2000200F311F840F951FAA27BB27ABBFFC0141
:10AF30008791F90182ABDB018C918F5F8C93982F05
:10AF4000803158F3CE018D960E946F4B4DC0F601B3
:10AF50003496A0E7B0E080E190E021E080309207F5
:10AF600019F40E94926E03C0182E0E94926E81E026
:10AF70008FA781EE88AB84E08EA7CE018D960E94CC
:10AF80006F4B32C081E08FA782EE88AB84E18EA741
:10AF9000FE01F196A0E7B0E080E190E021E0803092
:10AFA000920719F40E94816E03C0182E0E94816ED0
:10AFB000CE018D960E946F4B17C081E08FA780E86D
:10AFC00088AB85E08EA7F601838189ABCE018D9693
:10AFD0000E946F4B09C085E08EA71FA681E088AB59
:10AFE000CE018D960E946F4BCD51DF4F0FB6F89476
:10AFF000DEBF0FBECDBFDF91CF911F910F91FF90AC
:10B00000EF90DF90CF90BF90AF900895CF93DF93F4
:10B01000CDB7DEB72A970FB6F894DEBF0FBECDBF0F
:10B0200081E08B8388E88C8384E08A83CE0101965B
:10B030000E946F4B2A960FB6F894DEBF0FBECDBFAD
:10B04000DF91CF9108950F931F93CF93DF93CDB7E7
:10B05000DEB7C055D0400FB6F894DEBF0FBECDBFEF
:10B060008A0121E02B832DE52C839E838D836F83C2
:10B0700020E0261780F4AE01485F5F4F822F9927AA
:10B08000DA01A80FB91FF801E80FF91F80818C932E
:10B090002F5F261798F38FE08A83CE0101960E94D6
:10B0A0006F4BC05BDF4F0FB6F894DEBF0FBECDBF56
:10B0B000DF91CF911F910F91089548EC50E060E02F
:10B0C00070E08CE49EE00E94A26D1092160F109228
:10B0D000150F1092140F08959091150F8091160F6F
:10B0E000981738F08091150F9091160F891B9927AA
:10B0F00008959091150F8091160F981B892F8853F2
:10B10000992708952091160F8CE49EE0FC01E20F30
:10B11000F11DE0818091160F8F5F8093160F809153
:10B12000140F81508093140F8091160F883C10F0FB
:10B130001092160F8E2F992708950F931F93CF9378
:10B14000DF93EC018B0180EC0E94305A01501040DB
:10B150008FEF0F3F180709F188819927803C9105EF
:10B1600021F08B3D910541F00EC08BED0E94305ACD
:10B170008CED0E94305A0AC08BED0E94305A8DED42
:10B180000E94305A03C088810E94305A2196015093
:10B1900010408FEF0F3F1807F9F680EC0E94305AED
:10B1A000DF91CF911F910F9108950F931F93382F27
:10B1B0008091270B9927009719F00197C1F059C08A
:10B1C000303C09F056C01092280B2091280B8AE2DF
:10B1D0009BE0FC01E20FF11D30832F5F2093280BD1
:10B1E00081E08093270B84E68093290B42C0303C9A
:10B1F00099F58091280B8230F0F08091280B0AE2BB
:10B200001BE0F801E80FF11D30838F5F8093280B5E
:10B2100082E08093270B1092290BA8016091280BE4
:10B22000C8010E944459C8010E94854B1092270B07
:10B230001092280B1EC01092280B2091280B8AE236
:10B240009BE0FC01E20FF11D30832F5F2093280B60
:10B2500084E68093290B0DC02091280B8AE29BE0A5
:10B26000FC01E20FF11D30838091280B8F5F8093EA
:10B27000280B8091280B893620F01092270B109212
:10B28000280B1F910F910895FC01DA0161506F3F67
:10B29000F1F02081822F9927803C910521F08B3D90
:10B2A000910519F010C0319610C031962081822F7F
:10B2B00099278C3D910521F08D3D910519F003C032
:10B2C00020EC01C02BED2D933196615010F70895BD
:10B2D0008091290B882389F08091290B81508093DC
:10B2E000290B9091290B992341F48091270B8130F0
:10B2F00021F49093280B9093270B089585B1807FBC
:10B3000085B984B1876084B981E58CBD81E08DBD4C
:10B3100008958EBD0DB407FEFDCF8EB59927089513
:10B320000E94ED599C9AA4988FE08093940BA49866
:10B330006A9862980895A4980895CF93DF93CDB743
:10B34000DEB728970FB6F894DEBF0FBECDBFA49B23
:10B3500018C0629914C08091930B853050F0A49866
:10B360000E94062682E2809311011092E10D109254
:10B37000B60D8091930B8F5F8093930B02C0109258
:10B38000930BCE0101960E942D3229813A8181E5ED
:10B3900090E0289FA001299F500D389F500D112447
:10B3A000CA01880F892F881F990B91950E94EE5929
:10B3B0008D81882319F48F81882311F0A49A01C00C
:10B3C000A49828960FB6F894DEBF0FBECDBFDF91CC
:10B3D000CF9108958093940B089508950895109245
:10B3E000960B1092950B86E08093C20088E98093BB
:10B3F000C10060E875E280E090E00E940A5A81E0B6
:10B400008093170F1092180F08959093960B8093C6
:10B41000950B08959B01AC01DC01CB01689412F8F7
:10B42000880F991FAA1FBB1F1694D1F780509C4DFF
:10B43000AB40BF4F689413F8220F331F441F551FB2
:10B440001694D1F7BC01CD010E94056EDA01C90145
:10B450000197292F33272093C5008093C4000895B6
:10B46000982F8091C00085FFFCCF9093C60008956F
:10B470000F931F93CF93DF938C01EB0121978FEFF5
:10B48000CF3FD80751F0F80181918F010E94305AC7
:10B490002197FFEFCF3FDF07B1F781E090E0DF9129
:10B4A000CF911F910F9108951F920F920FB60F9297
:10B4B00011242F933F934F935F936F937F938F93B9
:10B4C0009F93AF93BF93EF93FF932091150F8CE45D
:10B4D0009EE0FC01E20FF11D8091C60080832F5F8A
:10B4E0002093150F8091140F8F5F8093140F92B1EA
:10B4F00084E0892782B98091140F883C18F00E945B
:10B500005D5806C08091150F883C10F01092150F01
:10B51000FF91EF91BF91AF919F918F917F916F912B
:10B520005F914F913F912F910F900FBE0F901F9001
:10B530001895DC01FB01415050408FEF4F3F5807F9
:10B5400041F081918D93415050408FEF4F3F58070C
:10B55000C1F70895DC01FB01415050408FEF4F3F90
:10B56000580769F091918D91891719F081E090E069
:10B570000895415050408FEF4F3F580799F780E0B2
:10B5800090E00895CF93DF93DC01FB0160E0462F4C
:10B5900091E0562F8081803231F4692F9F5F319680
:10B5A00080818032D1F38081882379F0808180325C
:10B5B00019F4442309F4492F8081803209F040E0D6
:10B5C0009F5F31968081882389F7442331F48081FD
:10B5D000882311F4492F01C0462F262F3327E90174
:10B5E000C91BD109EC0FFD1F3196842F9927821BAF
:10B5F000930B01971816190624F4942F961B91505B
:10B6000001C090E091509F3F29F081918D935F5F41
:10B610009150D8F71C925F5F852F9927DF91CF91CA
:10B620000895FC0190E08191882331F09F5F819122
:10B63000882311F09F3FD1F7892F99270895DC01C6
:10B64000FB018081882329F081918D93808188235B
:10B65000D9F71C9208950F931F93CF93DF93082F70
:10B66000162FFA0141E0C0E1D7E2C901BE010E94F4
:10B67000F26D6115710581F06C9FC0016D9F900D99
:10B680007C9F900D1124281B390B862F805D8193A0
:10B69000440F01E015E00AC0153040F0002319F016
:10B6A00080E3819302C080E281934F5FC8EED3E0D4
:10B6B000C901BE010E94F26D6115710581F06C9F98
:10B6C000C0016D9F900D7C9F900D1124281B390B9C
:10B6D000862F805D81934F5F01E014E00AC0143033
:10B6E00040F0002319F080E3819302C080E281934F
:10B6F0004F5FC4E6D0E0C901BE010E94F26D611542
:10B70000710581F04F5F6C9FC0016D9F900D7C9F14
:10B71000900D1124281B390B862F805D819301E049
:10B7200013E00AC0133040F04F5F002319F080E3AC
:10B73000819302C080E28193C9016AE070E00E94B7
:10B74000F26D6115710591F04F5FCB01880F991F64
:10B75000880F991F880F991F860F971F860F971FB5
:10B76000281B390B862F805D81930AC0123040F070
:10B770004F5F002319F080E3819302C080E2819340
:10B78000822F805D81931082842F9927DF91CF9142
:10B790001F910F910895FC01262F862F82958F709F
:10B7A0008A3038F06AE00E94D26D892F8F5B8193D6
:10B7B00009C0862F82958F706AE00E94D26D892F12
:10B7C000805D8193822F8F708A3038F06AE00E940A
:10B7D000D26D892F8F5B80830895822F8F706AE0EE
:10B7E0000E94D26D892F805D80830895EF92FF9231
:10B7F0000F931F937C018B01872F9927682FC70117
:10B800000E94CB5BC8019070682FC7010E94CB5B80
:10B810001F910F91FF90EF900895CF92DF92EF92DA
:10B82000FF920F931F936C017A018B01CB01AA2722
:10B83000BB27BC01C6010E94F65BD801C701A070FE
:10B84000B070BC01C6010E94F65B1F910F91FF9082
:10B85000EF90DF90CF9008951F93CF93DF93CDB7F4
:10B86000DEB768970FB6F894DEBF0FBECDBF10E00D
:10B87000BE016F5F7F4F812F0E94AA38412F55274D
:10B88000CA01880F991F880F991F880F991F9C0163
:10B89000241B350BF901E956F44F898184838A8191
:10B8A00085838B8186838C8180838D8181838E814A
:10B8B0008283F901E656F44F8F81382F33708885E3
:10B8C0008370282F220F220F888D982F9295907FBA
:10B8D000822F832B892B8083FA01E356F34F10824A
:10B8E0001F5F143128F268960FB6F894DEBF0FBEC2
:10B8F000CDBFDF91CF911F9108951F93CF93DF9319
:10B90000CDB7DEB768970FB6F894DEBF0FBECDBFD8
:10B9100010E0A89519821A821B821C821D821E8249
:10B920001F821886188E8FE0189FC0011124885836
:10B93000994FBC01CE0109960E94816DBE016F5FD7
:10B940007F4F812F0E9472381F5F143110F3689669
:10B950000FB6F894DEBF0FBECDBFDF91CF911F9120
:10B960000895CF93C0E086E0C89FC0011124FC0178
:10B97000EB5DF34FF093240CE093230C80819181D5
:10B98000009719F0019791838083E091230CF09147
:10B99000240C82819381009719F00197938382830D
:10B9A000E091230CF091240C84819581009719F08B
:10B9B0000197958384832C2F3327C901880F991F02
:10B9C000880F991F880F991F821B930BFC01E95662
:10B9D000F44F8081882319F48181882321F08C2FF2
:10B9E0008F5D0E94025ECF5FC43108F4BCCFCF915F
:10B9F000089599278730910509F466C0883091052C
:10BA0000ACF48430910509F43EC08530910534F4DE
:10BA10008230910511F1039759F198C08530910555
:10BA200009F43CC0069709F444C090C08A309105DF
:10BA300009F46BC08B30910544F48830910509F40A
:10BA40004EC0099709F456C081C08B30910509F4A6
:10BA500067C00C9709F46FC079C080EC0E94024A5D
:10BA6000882319F081E090E0089580E090E0089547
:10BA700081EC0E94024A882319F081E090E0089549
:10BA800080E090E0089582EC0E94024A882319F039
:10BA900081E090E0089580E090E0089581ED0E94BB
:10BAA000024A882319F081E090E0089580E090E058
:10BAB000089584EC0E94024A882319F081E090E006
:10BAC000089580E090E0089585EC0E94024A882362
:10BAD00019F081E090E0089580E090E0089586EC10
:10BAE0000E94024A882319F081E090E0089580E0E6
:10BAF00090E0089587EC0E94024A882319F081E0C3
:10BB000090E0089580E090E0089583EC0E94024A5E
:10BB1000882319F081E090E0089580E090E0089596
:10BB200082ED0E94024A882319F081E090E0089596
:10BB300080E090E0089583ED0E94024A882319F086
:10BB400081E090E0089580E090E0089580E090E04A
:10BB500008950F93CF93DF93CDB7DEB721970FB63C
:10BB6000F894DEBF0FBECDBF89838150843170F061
:10BB700000E021E0AE014F5F5F4F69E071E089E9CD
:10BB800091E00E94233480E090E007C089819927EA
:10BB9000FC01E456F34F8081992721960FB6F89463
:10BBA000DEBF0FBECDBFDF91CF910F9108950F93F0
:10BBB000CF93DF93CDB7DEB721970FB6F894DEBFF2
:10BBC0000FBECDBF8983843160F000E021E0AE017B
:10BBD0004F5F5F4F64E171E089E991E00E94233497
:10BBE00007C089812DE93CE0F901E80FF11D608370
:10BBF00021960FB6F894DEBF0FBECDBFDF91CF9177
:10BC00000F910895EF92FF920F931F93CF93DF93BD
:10BC1000CDB7DEB721970FB6F894DEBF0FBECDBF0C
:10BC20001982FF240F2D813209F46EC0823219F47B
:10BC300081E0898369C0833219F482E0898364C01A
:10BC4000843219F483E089835FC0853219F484E07B
:10BC500089835AC0863219F485E0898355C08732BA
:10BC600019F486E0898350C0883219F487E089830B
:10BC70004BC0893219F488E0898346C08A3219F4AE
:10BC800089E0898341C08B3219F48AE089833CC002
:10BC90008C3219F48BE0898337C08D3219F48CE033
:10BCA000898332C08E3219F48DE089832DC08F32A2
:10BCB00019F48EE0898328C0803319F48FE08983DA
:10BCC00023C0813319F480E189831EC0823319F4C3
:10BCD00081E1898319C0833319F482E1898314C017
:10BCE000843319F483E189830FC000E021E0AE01C1
:10BCF0004F5F5F4F69E471E089E991E00E9423346E
:10BD000080E090E00C94046810E0F12EE12E29818F
:10BD100086E0289FC00111248B5D934F9093240CE3
:10BD20008093230C3327C901880F991F880F991F0F
:10BD3000880F991F821B930BFC01E956F44F8081F9
:10BD4000882309F43CC28981282F3327C901880F31
:10BD5000991F880F991F880F991F821B930BFC0155
:10BD6000E956F44F80818F3F19F4FF24F39427C2E2
:10BD70008981282F3327C901880F991F880F991FA0
:10BD8000880F991F821B930BFC01E956F44FE08149
:10BD90008E2F82508B3008F04EC08E2F0E94F95C9F
:10BDA000082F8981282F3327C901880F991F880FF1
:10BDB000991F880F991F821B930BFC01E656F44FC5
:10BDC000808182958F7080FF02C081E00827002368
:10BDD00069F0E091230CF091240C80819181892BF2
:10BDE00019F4FF24F394EBC1FF24E9C1A091230CC3
:10BDF000B091240C8981282F3327C901880F991FFE
:10BE0000880F991F880F991F821B930BFC01E9561D
:10BE1000F44F948185E0989FC00111248D939C93E9
:10BE2000E091230CF091240C808191810196918303
:10BE30008083FF24C4C18981282F3327C901880F3B
:10BE4000991F880F991F880F991F821B930BFC0164
:10BE5000E956F44FE0818E2F8D50803208F04EC0AD
:10BE60008F5F0E943813082F8981282F3327C9013B
:10BE7000880F991F880F991F880F991F821B930B9A
:10BE8000FC01E656F44F808182958F7080FF02C0DE
:10BE900081E00827002369F0E091230CF091240C45
:10BEA00080819181892B19F4FF24F39488C1FF24A8
:10BEB00086C1A091230CB091240C8981282F3327AF
:10BEC000C901880F991F880F991F880F991F821B1E
:10BED000930BFC01E956F44F948185E0989FC001D3
:10BEE00011248D939C93E091230CF091240C80817C
:10BEF0009181019691838083FF2461C18981282FDC
:10BF00003327C901880F991F880F991F880F991F20
:10BF1000821B930BFC01E956F44FE0818E2F8D526A
:10BF2000823208F04EC08F5F0E94E731082F89816E
:10BF3000282F3327C901880F991F880F991F880F51
:10BF4000991F821B930BFC01E656F44F808182956A
:10BF50008F7080FF02C081E00827002369F0E09124
:10BF6000230CF091240C80819181892B19F4FF24FA
:10BF7000F39425C1FF2423C1A091230CB091240C7C
:10BF80008981282F3327C901880F991F880F991F8E
:10BF9000880F991F821B930BFC01E956F44F948183
:10BFA00085E0989FC00111248D939C93E091230C10
:10BFB000F091240C80819181019691838083FF24EC
:10BFC000FEC08981282F3327C901880F991F880F48
:10BFD000991F880F991F821B930BFC01E956F44FA0
:10BFE000E0818E2F8F54843108F04EC08F5F0E9405
:10BFF000A95D082F8981282F3327C901880F991F30
:10C00000880F991F880F991F821B930BFC01E6561E
:10C01000F44F808182958F7080FF02C081E00827F5
:10C02000002369F0E091230CF091240C8081918130
:10C03000892B19F4FF24F394C2C0FF24C0C0A0913F
:10C04000230CB091240C8981282F3327C901880F34
:10C05000991F880F991F880F991F821B930BFC0152
:10C06000E956F44F948185E0989FC00111248D9387
:10C070009C93E091230CF091240C80819181019696
:10C0800091838083FF249BC08981282F3327C90196
:10C09000880F991F880F991F880F991F821B930B78
:10C0A000FC01E956F44FE0818E2F83568E3008F064
:10C0B00086C000E0E33661F49091B90D892F83507A
:10C0C000823020F0913011F0963081F501E02EC0E1
:10C0D0008981282F3327C901880F991F880F991F3D
:10C0E000880F991F821B930BFC01E956F44F808146
:10C0F000843641F48091B90D853011F08230B1F46D
:10C1000001E014C08981282F3327C901880F991FA6
:10C11000880F991F880F991F821B930BFC01E9560A
:10C12000F44F80818E520E941F26082F8981282F6C
:10C130003327C901880F991F880F991F880F991FEE
:10C14000821B930BFC01E656F44F808182958F7021
:10C1500080FF02C081E00827002369F0E091230CF2
:10C16000F091240C80819181892B19F4FF24F394A0
:10C1700026C0FF2424C0A091230CB091240C8981F7
:10C18000282F3327C901880F991F880F991F880FFF
:10C19000991F821B930BFC01E956F44F948185E0B3
:10C1A000989FC00111248D939C93E091230CF091F2
:10C1B000240C80819181019691838083FF244981A1
:10C1C000842F99279C01220F331F220F331F220F28
:10C1D000331F281B390BF901E956F44F808188235E
:10C1E00069F08181882351F48281882339F4602F9A
:10C1F000842F0E94D75D802F992706C78981282F19
:10C200003327C901880F991F880F991F880F991F1D
:10C21000821B930BFC01E956F44F8181882311F4B2
:10C22000182F3BC28981282F3327C901880F991FF6
:10C23000880F991F880F991F821B930BFC01E956E9
:10C24000F44F81818F3F11F411E027C28981282F9B
:10C250003327C901880F991F880F991F880F991FCD
:10C26000821B930BFC01E956F44F9181892F825078
:10C270008B3008F04EC0892F0E94F95C082F89810D
:10C28000282F3327C901880F991F880F991F880FFE
:10C29000991F821B930BFC01E656F44F8081829517
:10C2A0008F7081FF02C081E00827002361F0E091D8
:10C2B000230CF091240C82819381892B11F411E0DD
:10C2C000ECC110E0EAC1A091230CB091240C89814B
:10C2D000282F3327C901880F991F880F991F880FAE
:10C2E000991F821B930BFC01E956F44F958185E061
:10C2F000989FC0011124FD0193838283E091230C58
:10C30000F091240C8281938101969383828310E0C3
:10C31000C4C18981282F3327C901880F991F880F2D
:10C32000991F880F991F821B930BFC01E956F44F4C
:10C330009181892F8D50803208F04EC08F5F0E940E
:10C340003813082F8981282F3327C901880F991F97
:10C35000880F991F880F991F821B930BFC01E656CB
:10C36000F44F808182958F7081FF02C081E00827A1
:10C37000002361F0E091230CF091240C82819381E1
:10C38000892B11F411E089C110E087C1A091230C21
:10C39000B091240C8981282F3327C901880F991F58
:10C3A000880F991F880F991F821B930BFC01E95678
:10C3B000F44F958185E0989FC0011124FD0193837E
:10C3C0008283E091230CF091240C82819381019669
:10C3D0009383828310E061C18981282F3327C901AB
:10C3E000880F991F880F991F880F991F821B930B25
:10C3F000FC01E956F44F9181892F8D52823208F069
:10C400004EC08F5F0E94E731082F8981282F332784
:10C41000C901880F991F880F991F880F991F821BC8
:10C42000930BFC01E656F44F808182958F7081FF5B
:10C4300002C081E00827002361F0E091230CF09115
:10C44000240C82819381892B11F411E026C110E024
:10C4500024C1A091230CB091240C8981282F33276B
:10C46000C901880F991F880F991F880F991F821B78
:10C47000930BFC01E956F44F958185E0989FC0012C
:10C480001124FD0193838283E091230CF091240C0D
:10C490008281938101969383828310E0FEC089811B
:10C4A000282F3327C901880F991F880F991F880FDC
:10C4B000991F821B930BFC01E956F44F9181892F40
:10C4C0008F54843108F04EC08F5F0E94A95D082F01
:10C4D0008981282F3327C901880F991F880F991F39
:10C4E000880F991F821B930BFC01E656F44F808145
:10C4F00082958F7081FF02C081E00827002361F0E0
:10C50000E091230CF091240C82819381892B11F40A
:10C5100011E0C3C010E0C1C0A091230CB091240C65
:10C520008981282F3327C901880F991F880F991FE8
:10C53000880F991F821B930BFC01E956F44F9581DC
:10C5400085E0989FC0011124FD0193838283E091CF
:10C55000230CF091240C8281938101969383828332
:10C5600010E09BC08981282F3327C901880F991FAC
:10C57000880F991F880F991F821B930BFC01E956A6
:10C58000F44F9181892F83568E3008F086C000E0E9
:10C59000933661F49091B90D892F8350823020F049
:10C5A000913011F0963081F501E02EC08981282F5D
:10C5B0003327C901880F991F880F991F880F991F6A
:10C5C000821B930BFC01E956F44F8181843641F4C0
:10C5D0008091B90D853011F08230B1F401E014C0C2
:10C5E0008981282F3327C901880F991F880F991F28
:10C5F000880F991F821B930BFC01E956F44F818130
:10C600008E520E941F26082F8981282F3327C901A7
:10C61000880F991F880F991F880F991F821B930BF2
:10C62000FC01E656F44F808182958F7081FF02C035
:10C6300081E00827002361F0E091230CF091240CA5
:10C6400082819381892B11F411E027C010E025C06D
:10C65000A091230CB091240C8981282F3327C90184
:10C66000880F991F880F991F880F991F821B930BA2
:10C67000FC01E956F44F958185E0989FC001112493
:10C68000FD0193838283E091230CF091240C82813D
:10C69000938101969383828310E08981282F332729
:10C6A000C901880F991F880F991F880F991F821B36
:10C6B000930BFC01E956F44F8281882311F4E82E94
:10C6C00041C28981282F3327C901880F991F880FFC
:10C6D000991F880F991F821B930BFC01E956F44F99
:10C6E00082818F3F19F4EE24E3942CC28981282F94
:10C6F0003327C901880F991F880F991F880F991F29
:10C70000821B930BFC01E956F44F9281892F8250D2
:10C710008B3008F04FC0892F0E94F95C082F898167
:10C72000282F3327C901880F991F880F991F880F59
:10C73000991F821B930BFC01E656F44F8081829572
:10C740008F7082FF02C081E00827002369F0E0912A
:10C75000230CF091240C84819581892B19F4EE240B
:10C76000E394F0C1EE24EEC1A091230CB091240C0F
:10C770008981282F3327C901880F991F880F991F96
:10C78000880F991F821B930BFC01E956F44F968189
:10C7900085E0989FC0011124FD0195838483E09179
:10C7A000230CF091240C84819581019695838483D8
:10C7B000EE24C8C18981282F3327C901880F991F0A
:10C7C000880F991F880F991F821B930BFC01E95654
:10C7D000F44F9281892F8D50803208F04FC08F5FC7
:10C7E0000E943813082F8981282F3327C901880F09
:10C7F000991F880F991F880F991F821B930BFC01AB
:10C80000E656F44F808182958F7082FF02C081E0EE
:10C810000827002369F0E091230CF091240C848117
:10C820009581892B19F4EE24E3948CC1EE248AC1FE
:10C83000A091230CB091240C8981282F3327C901A2
:10C84000880F991F880F991F880F991F821B930BC0
:10C85000FC01E956F44F968185E0989FC0011124B0
:10C86000FD0195838483E091230CF091240C848155
:10C870009581019695838483EE2464C18981282F54
:10C880003327C901880F991F880F991F880F991F97
:10C89000821B930BFC01E956F44F9281892F8D5234
:10C8A000823208F04FC08F5F0E94E731082F8981E4
:10C8B000282F3327C901880F991F880F991F880FC8
:10C8C000991F821B930BFC01E656F44F80818295E1
:10C8D0008F7082FF02C081E00827002369F0E09199
:10C8E000230CF091240C84819581892B19F4EE247A
:10C8F000E39428C1EE2426C1A091230CB091240C0E
:10C900008981282F3327C901880F991F880F991F04
:10C91000880F991F821B930BFC01E956F44F9681F7
:10C9200085E0989FC0011124FD0195838483E091E7
:10C93000230CF091240C8481958101969583848346
:10C94000EE2400C18981282F3327C901880F991F40
:10C95000880F991F880F991F821B930BFC01E956C2
:10C96000F44F9281892F8F54843108F04FC08F5F2C
:10C970000E94A95D082F8981282F3327C901880FBC
:10C98000991F880F991F880F991F821B930BFC0119
:10C99000E656F44F808182958F7082FF02C081E05D
:10C9A0000827002369F0E091230CF091240C848186
:10C9B0009581892B19F4EE24E394C4C0EE24C2C0FF
:10C9C000A091230CB091240C8981282F3327C90111
:10C9D000880F991F880F991F880F991F821B930B2F
:10C9E000FC01E956F44F968185E0989FC00111241F
:10C9F000FD0195838483E091230CF091240C8481C4
:10CA00009581019695838483EE249CC08981282F8B
:10CA10003327C901880F991F880F991F880F991F05
:10CA2000821B930BFC01E956F44F9281892F8356A8
:10CA30008E3008F087C000E0933661F49091B90D14
:10CA4000892F8350823020F0913011F0963081F59B
:10CA500001E02EC08981282F3327C901880F991F33
:10CA6000880F991F880F991F821B930BFC01E956B1
:10CA7000F44F8281843641F48091B90D853011F0F4
:10CA80008230B1F401E014C08981282F3327C90115
:10CA9000880F991F880F991F880F991F821B930B6E
:10CAA000FC01E956F44F82818E520E941F26082F06
:10CAB0008981282F3327C901880F991F880F991F53
:10CAC000880F991F821B930BFC01E656F44F80815F
:10CAD00082958F7082FF02C081E00827002369F0F1
:10CAE000E091230CF091240C84819581892B19F419
:10CAF000EE24E39427C0EE2425C0A091230CB0912E
:10CB0000240C8981282F3327C901880F991F880F8A
:10CB1000991F880F991F821B930BFC01E956F44F54
:10CB2000968185E0989FC0011124FD01958384833F
:10CB3000E091230CF091240C8481958101969583DA
:10CB40008483EE242981822F9927AC01440F551F3D
:10CB5000440F551F440F551F481B590BDA01A956A6
:10CB6000B44F8C91882309F47FC1FD018181882312
:10CB700009F47AC18281882309F476C1FA01E65664
:10CB8000F44FE0818E2F837009F084C0FF2009F4F8
:10CB90003EC01123E1F18E2F86958695837061F456
:10CBA0006E2D822F0E94D75DEE2019F081E090E07B
:10CBB0002BC280E090E028C28981282F3327C90149
:10CBC000880F991F880F991F880F991F821B930B3D
:10CBD000FC01E656F44F80818695869583708230FD
:10CBE00079F460E0FE1409F461E089810E94D75D68
:10CBF000FE1419F481E090E007C280E090E004C2E6
:10CC000061E089810E94D75D81E090E0FDC14981AA
:10CC1000242F3327C901880F991F880F991F880F68
:10CC2000991F821B930BFC01E656F44F8081869579
:10CC300086958370823049F4EE2039F461E0842FC8
:10CC40000E94D75D81E090E0DFC14981242F332726
:10CC5000C901880F991F880F991F880F991F821B80
:10CC6000930BFC01E656F44F808186958695682FDC
:10CC70006370613041F4EE2031F0842F0E94D75D63
:10CC800081E090E0C1C160E089810E94D75D80E0D1
:10CC900090E0BAC14981242F3327C901880F991F19
:10CCA000880F991F880F991F821B930BFC01E65672
:10CCB000F44FE0818E2F8370823009F045C0F11669
:10CCC000E1F58E2F86958695837061F46E2D842F05
:10CCD0000E94D75DEE2019F081E090E095C180E0E0
:10CCE00090E092C18981282F3327C901880F991FAD
:10CCF000880F991F880F991F821B930BFC01E65622
:10CD0000F44F8081869586958370823079F460E057
:10CD1000FE1409F461E089810E94D75DFE1419F4C4
:10CD200081E090E071C180E090E06EC161E08981B6
:10CD30000E94D75D81E090E067C160E089810E9438
:10CD4000D75D80E090E060C1FF2019F4112309F461
:10CD500048C04981242F3327C901880F991F880FA4
:10CD6000991F880F991F821B930BFC01E656F44F05
:10CD7000808186958695837061F46E2D842F0E9444
:10CD8000D75DEE2019F081E090E03EC180E090E0B8
:10CD90003BC14981242F3327C901880F991F880F70
:10CDA000991F880F991F821B930BFC01E656F44FC5
:10CDB0008081869586958370823061F46E2D842FF4
:10CDC0000E94D75DEE2019F081E090E01DC180E067
:10CDD00090E01AC161E089810E94D75D81E090E016
:10CDE00013C14981242F3327C901880F991F880F48
:10CDF000991F880F991F821B930BFC01E656F44F75
:10CE0000808186958695682F6370613041F4EE20AD
:10CE100021F1842F0E94D75D81E090E0F5C0498127
:10CE2000242F3327C901880F991F880F991F880F56
:10CE3000991F821B930BFC01E656F44F8081869567
:10CE400086958370823049F4EE2039F461E0842FB6
:10CE50000E94D75D81E090E0D7C060E089810E94A8
:10CE6000D75D80E090E0D0C02981822F9927AC0166
:10CE7000440F551F440F551F440F551F481B590B96
:10CE8000DA01A956B44F8C91882309F452C0FD01F0
:10CE90008181882309F44DC0FA01E656F44F808160
:10CEA000837091F4FF2049F0112339F061E0822F63
:10CEB0000E94D75D81E090E0A7C060E089810E9478
:10CEC000D75D80E090E0A0C04981242F3327C901BD
:10CED000880F991F880F991F880F991F821B930B2A
:10CEE000FC01E656F44F80818370823081F4F116A4
:10CEF00039F461E0842F0E94D75D81E090E084C026
:10CF000060E089810E94D75D80E090E07DC0FF20D5
:10CF100011F4112339F061E089810E94D75D81E02D
:10CF200090E072C060E089810E94D75D80E090E06F
:10CF30006BC02981822F9927AC01440F551F440FE4
:10CF4000551F440F551F481B590BDA01A956B44F02
:10CF5000FD018181882309F455C08281882309F469
:10CF600051C0FA01E656F44F80818695869583700C
:10CF700091F4FF2049F0112339F061E0822F0E94E3
:10CF8000D75D81E090E040C060E089810E94D75D7C
:10CF900080E090E039C04981242F3327C901880FF0
:10CFA000991F880F991F880F991F821B930BFC01F3
:10CFB000E656F44F8081869586958370823081F4A1
:10CFC000F11639F461E0842F0E94D75D81E090E092
:10CFD0001BC060E089810E94D75D80E090E014C0B2
:10CFE000FF2011F4112339F061E089810E94D75D9F
:10CFF00081E090E009C060E089810E94D75D80E017
:10D0000090E002C080E090E021960FB6F894DEBF79
:10D010000FBECDBFDF91CF911F910F91FF90EF9089
:10D020000895CF93DF93CDB7DEB721970FB6F8946D
:10D03000DEBF0FBECDBF282F04B603FE28C0FE0101
:10D040003196ACECB0E081E090E031E080309307C5
:10D0500019F40E94816E03C0182E0E94816E89818E
:10D06000843190F48F5F8983FE013196ACECB0E09F
:10D0700081E090E031E08030930719F40E94926ED5
:10D0800003C0182E0E94926E84B7877F84BF809160
:10D090006000886180936000209360008091600050
:10D0A00088608093600021960FB6F894DEBF0FBEB3
:10D0B000CDBFDF91CF910895EF92FF920F931F9311
:10D0C0007B018C0120E030E040E05FE40E94C06A18
:10D0D00088239CF020E030E040E05FECC801B7011D
:10D0E0000E94AA69DC01CB01BC01CD010E945A6BF0
:10D0F000605070408040904804C0C801B7010E9451
:10D100005A6B1F910F91FF90EF900895A0E0B0E04F
:10D11000ECE8F8E60C94426E8C017B015A01DC01CC
:10D120008C91823058F0FB019081923010F4A7016D
:10D130000BC1843029F4943009F4A6C0A80104C1BD
:10D140009430A9F3923009F4A9C0823081F3F80138
:10D15000C280D380FB0162817381F8012481358113
:10D1600046815781F7016480758086809780C6016B
:10D17000861B970B97FDD8C080970CF46CC06C157C
:10D180007D050CF0ADC0662477244301F801618170
:10D19000F7018181681709F499C0662309F491C0E9
:10D1A000621A730A840A950AA401930157FDC0C04C
:10D1B000F5011182B60119012A0179018A013901AB
:10D1C0004A0108946108710881089108FFEF6F1601
:10D1D000FFEF7F06FFEF8F06FFE39F06F0F4A80145
:10D1E0009701220F331F441F551F19012A01B60151
:10D1F000615070406B0179018A0139014A0108943C
:10D2000061087108810891088FEF68168FEF780622
:10D210008FEF88068FE3980610F383E0D5018C9397
:10D2200057FC64C0F5012483358346835783738399
:10D230006283A50189C06F5F7F4FD401C3018170F4
:10D240009070A070B0709694879477946794682AD1
:10D25000792A8A2A9B2A6C157D056CF311C00894E3
:10D26000C11CD11CDA01C90181709070A070B0702E
:10D270005695479537952795282B392B4A2B5B2BAD
:10D28000C616D70664F382CFF8019181FB01818134
:10D29000981709F453CF4CEA51E056C0823009F098
:10D2A0004DCF88E0DA01F80101900D928A95E1F7FF
:10D2B000F8018181FB0191818923FA018183A50114
:10D2C00043C0261937094809590970CFF501618310
:10D2D000B601260D371D481D591D19012A019DCF84
:10D2E0006B0120E030E040E050E050CFD201C101BE
:10D2F000B695A7959795879521E030E040E050E0FE
:10D300002222332244225522282A392A4A2A5B2AF9
:10D31000F50124823582468257820894C11CD11CB3
:10D32000D382C282A50110C0909581959F4F24CFD2
:10D3300081E0F5018183B6015095409530952195A6
:10D340003F4F4F4F5F4F37CFCA01E2E1CDB7DEB756
:10D350000C945E6EA0E2B0E0E0EBF9E60C94506E47
:10D36000DC01CB01898F9A8FAB8FBC8F2D8F3E8FC5
:10D370004F8F58A3BE016F5F7F4FCE0149960E9429
:10D38000946C8E01075F1F4FB801CE014D960E942D
:10D39000946CAE014F5E5F4FB801CE0101960E94C2
:10D3A00086680E94AC6BDC01CB01BC01CD01E4E0DE
:10D3B000A0960C946C6EA0E2B0E0E1EEF9E60C945D
:10D3C000506EDC01CB01898F9A8FAB8FBC8F2D8F74
:10D3D0003E8F4F8F58A3BE016F5F7F4FCE0149969E
:10D3E0000E94946C8E01075F1F4FB801CE014D96CD
:10D3F0000E94946C8A8591E089278A87AE014F5EEE
:10D400005F4FB801CE0101960E9486680E94AC6B06
:10D41000DC01CB01BC01CD01E4E0A0960C946C6E64
:10D42000A8E1B0E0E6E1FAE60C944A6EDC01CB013B
:10D43000898B9A8BAB8BBC8B2D8B3E8B4F8B588FF4
:10D44000BE016F5F7F4FCE0141960E94946C8E01AA
:10D45000075F1F4FB801CE0145960E94946CFE01F4
:10D4600031962981223008F45FC03985323010F4BA
:10D47000B8017BC081819A8589278183243009F492
:10D4800055C0223009F452C0343009F454C032304F
:10D4900009F458C06B817C818B859C85681B790B56
:10D4A0002D813E814F815885ED84FE840F8518893A
:10D4B0002E153F054007510730F4220F331F441F3C
:10D4C000551F615070407C836B8380E090E0A0E04A
:10D4D000B0E4AA24BB2465012E153F05400751077F
:10D4E00040F0A82AB92ACA2ADB2A2E193F09400B84
:10D4F000510BB695A79597958795220F331F441F1B
:10D50000551F0097A105B10539F7D601C5018F77E1
:10D510009070A070B07080349105A105B105A9F09C
:10D52000A482B582C682D782BF011FC02317E1F74C
:10D530006CEA71E01AC01D821E821F8218861C824E
:10D540001B82F2CF84E08983EFCFA7FC05C02115B1
:10D5500031054105510521F380E490E0A0E0B0E001
:10D56000A80EB91ECA1EDB1EDBCFCB010E94AC6B1E
:10D57000DC01CB01BC01CD01EAE068960C94666E3B
:10D58000A8E1B0E0E6ECFAE60C94506EDC01CB01C9
:10D59000898B9A8BAB8BBC8B2D8B3E8B4F8B588F93
:10D5A000BE016F5F7F4FCE0141960E94946C8E0149
:10D5B000075F1F4FB801CE0145960E94946C898188
:10D5C000823018F08985823018F42FEF3FEF09C0C0
:10D5D000B801CE0101960E940E6D282F332727FD3A
:10D5E0003095C901E4E068960C946C6EA8E0B0E058
:10D5F000ECEFFAE60C944E6E9B01AC017B018C01C2
:10D60000EE2417FDE394FF2400271127EA82211559
:10D6100031054105510539F482E08983CE01019637
:10D620000E94AC6B43C083E089836EE170E0CB0164
:10D63000EE2031F579018A01A80197012030E0E060
:10D640003E07E0E04E07E0E45E0798F479018A01C6
:10D65000EE0CFF1C001F111F0197BC01A8019701D0
:10D66000E0E0EE16E0E0FE06E0E00E07E0E41E0774
:10D6700068F3ED82FE820F8318877C836B83CECFA5
:10D680002030E0E03E07E0E04E07E0E85E0741F0D2
:10D69000EE24FF248701E21AF30A040B150BCCCF0A
:10D6A0007C836B8360E070E080E09FECE6E028968E
:10D6B0000C946A6EACE0B0E0E0E6FBE60C94526ECF
:10D6C000DC01CB0189879A87AB87BC87BE016F5F7E
:10D6D0007F4FCE0109960E94946C8981823011F0AF
:10D6E000823028F460E070E080E090E031C0843067
:10D6F00039F02B813C8137FDF5CF2F3131056CF0AE
:10D700008A81882329F060E070E080E090E820C002
:10D710006FEF7FEF8FEF9FE71BC08EE190E0821BE2
:10D72000930B2D813E814F81588504C056954795B6
:10D73000379527958A95D2F78A81882339F05095B5
:10D740004095309521953F4F4F4F5F4FCA01B9012A
:10D75000E2E02C960C946E6EA0E0B0E0E2EBFBE60B
:10D760000C94486E882499245401DC01FC01248126
:10D770003581468157818181082F112760E070E053
:10D780008C91823020F46FEF70E04061A4C084304F
:10D7900009F464C0823009F463C0211531054105E4
:10D7A000510509F498C0FD0182819381FFEF823811
:10D7B0009F070CF050C0A2E8EA2EAFEFFA2EE81A4D
:10D7C000F90A8AE1E816F1040CF06BC06B0181E004
:10D7D00090E0A0E0B0E00E2C04C0880F991FAA1FB3
:10D7E000BB1F0A94D2F70197A109B10982239323A1
:10D7F000A423B5230097A105B10519F0F1E0CF2EC0
:10D80000D12C04C05695479537952795EA94D2F7C1
:10D81000C601AA2797FDA095BA2F282B392B4A2B92
:10D820005B2BDA01C9018F779070A070B0708034E3
:10D830009105A105B105D1F1215C3F4F4F4F5F4FDD
:10D840002030E0E03E07E0E04E07E0E45E0708F14C
:10D8500061E070E01EC0803891053CF06FEF70E031
:10D8600020E030E040E050E036C0BC0161587F4F1E
:10D87000DA01C9018F779070A070B0708034910583
:10D88000A105B105D1F0215C3F4F4F4F5F4F57FDD0
:10D890001BC097E056954795379527959A95D1F7F0
:10D8A0001AC020E030E040E050E0BBCF27FFC8CFF7
:10D8B000205C3F4F4F4F5F4FC3CF27FFE8CF205C27
:10D8C0003F4F4F4F5F4FE3CF56954795379527957D
:10D8D0006F5F7F4FDECF822E932E942F9F778A2DFE
:10D8E0008078A82EA92A962F9795992797958A2D03
:10D8F0008F77A82EA92A76956795962F9F778B2DDF
:10D900008078B82EB92A902F9795992797958B2DC7
:10D910008F77B82EB92AD501C401BC01CD01ECE046
:10D92000CDB7DEB70C94646ECF93DF93FC01DB01BF
:10D93000408151812281622F6F7770E0221F222760
:10D94000221F9381892F880F822B282F3327991F1D
:10D950009927991FED0199832115310541F441154E
:10D96000510561057105E1F482E08C9354C02F3FAD
:10D97000310509F441C02F573040FD013383228324
:10D9800083E08C9387E0440F551F661F771F8A95AD
:10D99000D1F77064ED014C835D836E837F833BC060
:10D9A00022E83FEFF901C7E0440F551F661F771FBC
:10D9B000CA95D1F783E08C93403080E0580780E02F
:10D9C000680780E4780778F4440F551F661F771FB7
:10D9D00021503040F9014030C0E05C07C0E06C07E6
:10D9E000C0E47C0788F3ED01FB83EA83FD014483F7
:10D9F0005583668377830FC0411551056105710515
:10DA000019F484E08C9307C064FF03C081E08C9319
:10DA1000C1CF1C92BFCFDF91CF9108950F931F9379
:10DA2000CF93DF93FC01DB018081823018F09C9161
:10DA3000923018F461E070E05EC08430C1F0843050
:10DA400001F1943009F447C0823009F44BC08230B0
:10DA500009F44EC09230A9F04181ED018981481747
:10DA6000B9F0442389F08FEF9FEFBC0144C094309C
:10DA700031F7EB018981682F77278181681B710954
:10DA80003AC08181882379F781E090E0BC0133C0FE
:10DA900022813381ED018A819B81821793070CF3E8
:10DAA000281739079CF00481158126813781FD01F3
:10DAB000648175818681978160177107820793075A
:10DAC00080F2061717072807390778F4442359F21C
:10DAD00081E090E0DBCFFD018181882321F281E0AC
:10DAE00090E0D4CF923009F0B2CF60E070E003C094
:10DAF000ED018981F2CFCB01DF91CF911F910F9181
:10DB00000895FB01DC0105900D920020E1F70895D6
:10DB1000FB01DC0104C08D910190801921F441507A
:10DB20005040C8F7881B990B0895FB01DC0140FFAA
:10DB300005C002C001900D9201900D9242505040DC
:10DB4000C8F70895DC0140FF03C001C06D936D93D9
:10DB500042505040D8F70895FB01DC0101900D922E
:10DB60000020E1F70895629FD001739FF001829F2A
:10DB7000E00DF11D649FE00DF11D929FF00D839F5C
:10DB8000F00D749FF00D659FF00D9927729FB00DF9
:10DB9000E11DF91F639FB00DE11DF91FBD01CF010C
:10DBA00011240895991B79E004C0991F961708F075
:10DBB000961B881F7A95C9F780950895AA1BBB1BF1
:10DBC00051E107C0AA1FBB1FA617B70710F0A61B7D
:10DBD000B70B881F991F5A95A9F780959095BC019E
:10DBE000CD01089597FB092E07260AD077FD04D0B2
:10DBF000E5DF06D000201AF4709561957F4F0895F7
:10DC0000F6F7909581959F4F0895A1E21A2EAA1BD1
:10DC1000BB1BFD010DC0AA1FBB1FEE1FFF1FA217DC
:10DC2000B307E407F50720F0A21BB30BE40BF50BD9
:10DC3000661F771F881F991F1A9469F76095709562
:10DC4000809590959B01AC01BD01CF01089597FB94
:10DC5000092E05260ED057FD04D0D7DF0AD0001CB0
:10DC600038F450954095309521953F4F4F4F5F4F79
:10DC70000895F6F790958095709561957F4F8F4F39
:10DC80009F4F08952F923F924F925F926F927F9293
:10DC90008F929F92AF92BF92CF92DF92EF92FF92BC
:10DCA0000F931F93CF93DF93CDB7DEB7CA1BDB0B68
:10DCB0000FB6F894DEBF0FBECDBF09942A8839880D
:10DCC00048885F846E847D848C849B84AA84B98414
:10DCD000C884DF80EE80FD800C811B81AA81B98120
:10DCE000CE0FD11D0FB6F894DEBF0FBECDBFED0134
:10DCF0000895F999FECFB2BDA1BDF89A119600B46E
:10DD00000895F7DF01921A94E1F70895F999FECF8B
:10DD1000B2BDA1BD00BC11960FB6F894FA9AF99A5B
:0EDD20000FBE08950190F2DF1A94E1F7089506
:10DD2E00012E2E2F63616E5F696E7075742E630007
:10DD3E006E222E2E2F6368616E6E656C732E6300DD
:10DD4E0053657175656E636520233100536571757A
:10DD5E00656E63652023320053657175656E63656C
:10DD6E002023330053657175656E6365202334007F
:10DD7E00455233002E2E2F656570726F6D6368618C
:10DD8E006E6E656C732E630050434D3000506F778E
:10DD9E006572426F7800455233004C4F4730340065
:10DDAE00092550434D2076657220392E3437004FA9
:10DDBE00425220383434300B002E2E2F7669727476
:10DDCE0075656C5F696E7075742E630000000000DF
:04DDDE000000000041
:00000001FF
